:100000000C94E94B0C941A4D0C940F4C0C940F4C1F
:100010000C940F4C0C940F4C0C940F4C0C94665E8B
:100020000C940F4C0C94A65D0C940F4C0C940F4C3C
:100030000C940F4C0C941A590C940F4C0C940F4CBC
:100040000C940F4C0C940F4C0C940F4C0C940F4CC4
:100050000C940F4C0C940F4C0C940F4C0C940F4CB4
:100060000C940F4C0C940F4C0C940F4C0C940F4CA4
:10007000090212000101008096090400000000003E
:10008000000012011001FF000008C016DD0500018C
:1000900001020001160351005500490043004B00C6
:1000A0004400450056003100360016036F00700012
:1000B00074006900780078002E006F0072006700FD
:1000C000040309045553425F42554C4B5F55504C55
:1000D0004F41445F494E49543A2025692025690A19
:1000E000005553425F42554C4B5F55504C4F414475
:1000F0005F494E49543A2062616E6B5F73697A655D
:100100003D30782530386C782062616E6B5F636EAD
:10011000743D3078257820656E645F616464723D5B
:1001200030782530386C780A005553425F42554C80
:100130004B5F55504C4F41445F414444523A20720A
:1001400065715F62616E6B3D307825303278206179
:100150006464723D30782530386C782074696D6540
:100160003D25690A005553425F42554C4B5F55503F
:100170004C4F41445F4E4558543A207265715F625E
:10018000616E6B3D30782530327820616464723D59
:1001900030782530386C782074696D653D25690AA2
:1001A000005553425F42554C4B5F55504C4F4144B4
:1001B0005F454E443A0A005553425F4352433A204A
:1001C000616464723D30782530386C78200A0055BF
:1001D00053425F4D4F44455F4156523A0A005553D2
:1001E000425F4D4F44455F534E45533A0A005553C5
:1001F000425F4156525F52455345543A0A005553A7
:10020000425F5345545F4C414F4445523A0A0055B2
:10021000534220706F6C6C0A00506F6C6C20555309
:10022000420A002D2D3E53776974636820544F2095
:100230004156520A004552524F523A757362467502
:100240006E6374696F6E5772697465206D6F726545
:100250002064617461207468616E206578706563E4
:100260007465642072656D61696E3A202569206C41
:10027000656E3A2025690A0075736246756E63746F
:10028000696F6E5772697465205245515F535441CE
:100290005455535F42554C4B5F55504C4F41442091
:1002A000616464723A2030782530386C78206C654F
:1002B0006E3A2025692072785F72656D61696E699A
:1002C0006E673D25690A0075736246756E637469D1
:1002D0006F6E52656164206C656E3D25692074788F
:1002E0005F72656D61696E696E673D2569200A0000
:1002F000737265675F7365743A20616464723D3040
:10030000782530386C7800310030000A0073726153
:100310006D5F62756C6B5F616464725F736176655B
:100320003A20616464723D30782530386C780A0D6B
:10033000007372616D5F62756C6B5F777269746573
:100340005F73746172743A20616464723D30782521
:1003500030386C780A0D007372616D5F62756C6B7A
:100360005F616464725F726573746F72653A206175
:100370006464723D30782530386C780A0D007372F1
:10038000616D5F62756C6B5F726561645F737461F0
:1003900072743A20616464723D30782530386C782C
:1003A0000A0D007372616D5F62756C6B5F726561DF
:1003B000645F656E643A0A007372616D5F726561B5
:1003C000643A20616464723D30782530386C780A74
:1003D0000D007372616D5F62756C6B5F777269742B
:1003E000655F656E643A007372616D5F7772697400
:1003F000653A20616464723D30782530386C78202D
:10040000646174613D25780A0D007372616D5F62ED
:10041000756C6B5F636F70795F66726F6D5F62752D
:10042000666665723A20616464723D3078253038C2
:100430006C78207372633D30782570206C656E3D5A
:10044000256C690A0D007372616D5F62756C6B5F7C
:10045000636F70795F696E746F5F627566666572EF
:100460003A20616464723D30782530386C782064BD
:1004700073743D30782570206C656E3D256C690A7B
:100480000D007372616D5F62756C6B5F7365743ABA
:1004900020616464723D30782530386C78206C655A
:1004A0006E3D256C690A0D007372616D5F62756C3B
:1004B0006B5F7365743A20616464723D30782530F7
:1004C000386C780A0D006372635F636865636B5F05
:1004D00062756C6B5F6D656D6F72793A20626F74D7
:1004E000746F6D5F616464723D30782530386C786C
:1004F00020746F705F616464723D30782530386CB1
:10050000780A006372635F636865636B5F62756C32
:100510006B5F6D656D6F72793A2062616E6B3D3015
:10052000782530327820616464723D307825303827
:100530006C78206372633D3078253034780A00632C
:1005400072635F636865636B5F62756C6B5F6D653B
:100550006D6F72793A2062616E6B3D307825303272
:100560007820616464723D30782530386C7820637F
:1005700072633D3078253034780A002A0A0025302D
:10058000386C783A00202530327800207C002563D2
:10059000002E007C0A000A2530386C783A002025AD
:1005A000303278000A00F5D319755A5D48BA249D97
:1005B00097CE4A3F49DF4AC72487F489F4AEF49ABC
:1005C000F4B2F45F5299B44DDA243D22AD94164B47
:1005D000F3A47BA53BA4A992451A2FA549574B83A9
:1005E000A5FE522F492F692445EBD77AB5FFD19E3E
:1005F000D5FEACFD41FB8DB64A5BA13DA0FD50FB95
:100600008EF675ED2BDA17B5CF689FD4EED06ED687
:1006100016691FD51668976B17691FD2DEAFBD5BD1
:100620007BBB76BA769236433B5E3B5A3B527B9518
:1006300076B03659DB471BAFD56B252DD106357EFD
:100640004D93E60F4D83A656F3ABE627CDF79A6A96
:10065000CD579A2F34159A839AFD9A0F34EF6AFE7C
:10066000A9F987E615CD6ECDF39ABF68EC9AC73528
:10067000DB359B359B34EB358F68566972354B35CE
:100680008B34399AB99A399AD99A999A199A699A56
:10069000C91AAB264393AE19AB49D38CD4A4688650
:1006A0006B066B066AFA69FA681234719A188DA49F
:1006B0001134A0098A2D62B3D8245E14CF8BF56261
:1006C0009DE8167F114F893F8ADF8935E2D7E2978F
:1006D000E217E211D1211E143F153F16DF17F78AEA
:1006E0006F8B6F8AAF89AF8A7BC497C417C4E7C486
:1006F00067C4A7C427C527C41DE23671B3288B453C
:10070000E27A719DB8565C25E6892BC4A5E2C3E266
:100710004231479C273E28CE11EF11EF166789B76B
:100720008B33C4E9E2CDE264D12A668A3789378AFD
:10073000E3C431E268F13A71A478B538421C2E0E58
:1007400011CDE24071809824F61113C578D120C6EE
:100750008AD1A24ED48A8248442604855621205C40
:10076000167C42A3E011FE10CE0B0DC239A14E380B
:100770002BB8855F859F859F8413C20FC277C2B750
:1007800042B5705CF84AF852A8123E178E084EE146
:10079000B070503820EC173E113E123E10DE13F6BA
:1007A0000AEF086F096F0AAF0BFF105E155E11CAE2
:1007B000859785DDC20BC2F3C2B3C233C2D3C25325
:1007C000825D28139E101E137608DB85ADC266A1DC
:1007D0004490854DC246618350283C2AAC15D6080A
:1007E000AB847C214FC815960BCB8425C2626191E6
:1007F000B040C811B28579C25CE101618E709F7012
:100800008F305BB84B9825CC146E176E136E156E37
:1008100011A609538529C264214BB00899428670FC
:100820009370A3902E8C176E10C60AD70BA3855415
:10083000E13A61A470AD703572DC0861B8304C18D3
:10084000220C16CCC22061A03040E82FF413FA0A23
:100850007D84DE422F2141300A06214ED00B3142E9
:10086000B41025488256D0088240052230AAD01004
:100870000DD256DA4203D44F9BE925EAA34DD44B5F
:100880003DF422FD839EA7BFD3FFD0065A4F7FA31E
:1008900075B4969EA567A88BFE4A7FA1A7E9CFF401
:1008A000143D494FD01FE90FF47BFA1DFD1699B690
:1008B0009A7E438FD3AFE957F45FF44B5A45BFA0FC
:1008C0009FD34A7A941EA115D4491DF4303D443F6C
:1008D000A307E8A7743FFD847E4C3FA21FD20FE818
:1008E000FBF43DBA8FEEA5EFD277E8DBF42DFA4F9B
:1008F000FA267D83BE8EBCFD0FFA77FA2AFD1B7D9A
:1009000085EEA1E5F465FA12DD4D5FA42FD0BFD2CC
:10091000E7E973F459FA5FF419FA17FA347D8AEEAD
:10092000A276FA245A19DD499FA08FD3C7E80E5A40
:100930004AB7D36D742BDD82B69996A00AC8B498D5
:100940006EA2457423DA06BA9E16D275F451FA08DF
:100950005D8BB686AEA6AB6801CDA779682B692EF4
:100960005D4197D365684BE912FA305D4C17A12DB4
:10097000A40BE87C9A83964D1FA2F35057E6D2074A
:10098000E903F47E3A07ED3E7A2FBD076D36BD9B35
:10099000DE45EF449B4567D23BD06EA7B7D11968BF
:1009A000B7D25BE874B469742ABD196D0A9D4C27EF
:1009B000A165512B9A8566D2896819F426B409F489
:1009C000469A8E369E8E43BB818E451B43AFA7A3AE
:1009D000D1D2682ADA757414DA487A2DDA35F46AD5
:1009E000B4143A02ED2A3A1C6D181D8A36840E465C
:1009F000335313DA20B48134196D00AA617FDA8F82
:100A000026A1F545EB437BA325D25E680968F1D4A6
:100A10008866408BA3B1687AB4181A8D1685A6A390
:100A2000129A164D8326524C26CA0BA1C08D17214F
:100A30003179D8D8EC7C47C57B25D933470E4B4C50
:100A4000D44112A441315A1ABEE9AE50C9FF2DFF5C
:100A5000DF2AB7C128F39D8F2C5BB862D1E247CD66
:100A6000A3C799EFB97B927914A981298B173CB25E
:100A70006482F9F6F9CBF2602AB977D9A2C5F9E612
:100A80005BEEBA73CD043297689EA4C53855BC5A44
:100A900028E6D367CE9A7DCB9C39E6B58BD7ACEDF3
:100AA0003A35EB9145CBF2613BB979CEECC8CCDD60
:100AB0004463C7995F9061696913C6A4A5A591D3E2
:100AC00044837906CF10CD648177DC9ABFFEFA09A2
:100AD0009A29F8FE3DD1DC8C8D96E2A73113345370
:100AE000F13D916AA66133957F1A3B41331DDF6763
:100AF00053CD2DFC1399BD6CE5E285F98B164F2083
:100B00007388E6A1EC62402FE761C3FDBB63DDFCA7
:100B1000D505E629F397AD99BFE291358BF3BA3A43
:100B2000397BFE82DC65E8F75D387BF5A2C5AB71E9
:100B3000C3854BD73CB2D29CBFC2DCF1BE60FE2263
:100B4000C8219A32CA37D70038E156AA21D8DC81A9
:100B5000B0C2663BBDB970F1C247D62ECB5B62BE58
:100B6000730A0671F2ED53CCA3FFFCF3F5F0059D7B
:100B7000B53A7FC9EAC56BD64C3063194E4E51DD8C
:100B800033B8F476726F7E6EFE236B2790E789266A
:100B9000077DC7706563F3328FCA0D1334B7E24126
:100BA000DF269A19D8FCCA3F8D9BA0B90DDF2F1004
:100BB000CDEDD80C12F0D3F8099A3BF07DA4A099A2
:100BC00089CD43FC53FA04CD2C7CCF1534776223B6
:100BD00036A5344D6C9ADCB4A8695DD3634DBB9ADD
:100BE0007637BDDAB4B7E9E3A6234D5F369D6EAA2A
:100BF0006D4AF4997D237D637C137C59BEE9BE6CFC
:100C0000DFA3BE27BB58B9EF35DFFBBE4F7D9FFB8F
:100C1000BEF69DF4B97CE77D4DFF6BFF03CB6BFE09
:100C2000A1F9A3CB5AC108420CDC00B34090804C20
:100C3000478A25300086C32850E1350A41025330E7
:100C40004917E42E869BF37863C611C076D2629171
:100C50004016B4A3C67CDFEA656B1773F0CABD68A3
:100C6000B19EC05C983C3F77A179324F56D00A893B
:100C7000A08D87EB600A64C32638AEA2FCDF508CDF
:100C8000093B10EE29C8CD9FBF686441EEFCF5E634
:100C900035F9794B78DF4D89B458476002DCBD36B1
:100CA000BF20FC95EFDA9B164711F4F5EEC56BD526
:100CB0008FE635058B172FE2B261E8438BA309ACB1
:100CC00080BBF9E7854BE7E7E52DCE35AF9CBF66E6
:100CD000053F98D49716C710F82BBC09EFC367508F
:100CE000896DD8EE2E5888302BC85FBDD63C7B7DF1
:100CF000C162B8233F6F310700B4631730FFCD33B3
:100D00001F596B86DBF3179927AF5C64E6EEF1DDC4
:100D10006209FC04772D5EFBC8EA3CE0612412EF17
:100D2000614BD59E5EED3DC0FDEE28A44BD3F99DF1
:100D3000909EFDA4EBFFC83FD2D145A0E321E15630
:100D40003542FE276FFFCF2DF96FBE91EE4FFBFEB0
:100D500091B68BBB57D657B65D0FDE35045D23D6F3
:100D6000F31FFFCFE0BF291A2AEAB43A1D15452D1B
:100D70005654238952A4502AE924ECE245C2115A60
:100D80005E772D8246D0EA042D2F1AAD968A5AAA94
:100D9000E3EF229A96BF89B834C1893A11076B7480
:100DA000D8E082B8ACC88B46A715F9F21A2A618D33
:100DB00095A46E83FB69F8B2E13D2345ABEB592462
:100DC0007529BEA4BABD36DC08824694BA7EC0320C
:100DD000AE6566CBD2969296175A3E68F9BAE5B7D9
:100DE00016A505A2FA9021967104449D7E2846C05E
:100DF0001C8E9AC9240AF1F17BA000E616010C258D
:100E00000208460FEF880751E8D56B0F58E1FE0C3A
:100E1000DE3106C6843B7A6187319E8E060430C07F
:100E2000E42E33E2D519AFCC82B9B7F18E2E332040
:100E30002A1E60CC70023A63D264D2B13984F7B012
:100E4000FCD98C187CC62400D1F3CDBBCC68EF0054
:100E50003D9FD1B5A3331568786DB5D6A9751FB57B
:100E6000BE5EAD17A90353D481F7AAC990C06BE346
:100E7000305E9BA7F3DAFA2CAF4B9EE603176EC5E4
:100E80005A18B1146BED3DE3B873C6D5585F357889
:100E90000AD6774DDA8143C46D8FE25A51ABEEC268
:100EA0004DFB4DC67D75E9DB71DF3EEB56E3BE635E
:100EB000EE9982FB2E31EE580464ECE075294097E0
:100EC0004E9E7D2F68C69546258071CDDAA461308F
:100ED00078DAF471D32FB4CADA3679649B3CB14D19
:100EE0009EDC26DFD2262F6D93FBC5214DCC5FB44F
:100EF0007EA479FEBAF9CB544D5E9657F0C8DAEB72
:100F0000A09F11A6E4AFCBE3C4C8BFDE35F3F691D2
:100F1000E6358B17AFE07F96E294C5ABAFBB0E47CB
:100F2000456BE36DFD3FA5C5E638ACC870D03865AC
:100F300067EF588D9361DD2F01A6E63F92B7C8ACED
:100F40001780DC96AF2E11F71C0EBB7DC132BE435D
:100F500047B788BCBFAC67F7736DDD2D07CB2C2C72
:100F6000562C699CEFB118B1901E85F628428F224D
:100F7000F6289A1E45DBA3483DCA4DC1C9C119C117
:100F8000BB830F0617065704D7043706B7049F081C
:100F9000FE25F862F0D5A00DB3D580D9514A45B2EF
:100FA00091F056A3B676AA25F9E1D6C6DB2D542AD0
:100FB0004085029BA053FBB17D2A9BB7A027063E2C
:100FC0000F62E305FE9FC46D525B30180DC85036AA
:100FD0000E1B42B14D2069D8EE0DD6056F88E42571
:100FE000218621B6C47832D496D89B0CB3C51AE2B8
:100FF00087DB627BC55F658B314A236C3189528AFE
:101000002DDE9872B54D671C8ED9D59ECCC8A23600
:1010100023C0005BEFD8A1036C0363AE1F604B36A7
:10102000EA926DD1711C02A1EBFEDB326AE4B5D706
:101030005C9D32E2AAE1C3860E196C360D1A983C0B
:10104000A07FBFA4BE7D7A27F64A88371AE262F5F0
:1010500031D15148491A51A014B8912BE89500EDAF
:1010600066FFF723FE4F8B4E358ECDC17A217188F6
:1010700071E8B0C5E6EDC9AF99BF98F265CAB1B4E1
:101080006B47BF73CBF577AC79F8C175A2D72982CE
:10109000194C452B6EDEF7D09CFCFBD34C70DD70F9
:1010A000FBD5EB260CBABB389BAD6372CE08B730CC
:1010B000FA7680B747AFB983C9A622DDE0B21BD666
:1010C000DC612A8AD58D05133115D1B1D659EE4D83
:1010D0003C3F314B01E51CACFCC1509BF9830EEC4D
:1010E0000EC99D9515566B56F75E3D70F570F3CEA3
:1010F000EB4E87E49A8DF2D36B64F6BFE57F54EE36
:101100009C327A5C977FF7DC3279C6949BEF1D3D69
:10111000AECBC58FE6443D066E39FEF1F57C0C2260
:1011200048B53EF844FE7394D9083EFF17093CBC0D
:101130002000000100ECB5097C5355FA307CEE3DEF
:10114000D9BA26EC01DAE686B5654D81C1A0858461
:10115000566B4510DC661866C606D98A8AB4E06804
:10116000C5DAA4420095D02AFC15B435150992625F
:10117000A18E0B325813CA561068661C87C5A56924
:101180000BB4CAD25B0A346DD3DCEF39F7266DBAE3
:101190008EEFFFF7FEDEEFF7BDDFFF3C39E7DC9CAB
:1011A000E73CCB79565FF193B237AB197B76CABE79
:1011B000B2F85D086DFD3B5D4A2F56C4D86266E209
:1011C000C57172E41A38A724AA54BC388E43A1977B
:1011D0006445DE2B38B6E5EADA37942B1155740AEC
:1011E000C95C15FB620D010676548864BBF062662B
:1011F000D56438E5D95533A578B122A454B2F8B8EE
:10120000C8456BE1B083B406F0445644C711AB3512
:10121000287976662468644344709143E5359A29B9
:10122000906234E3428C0E526611B308954C2D4403
:101230001410E3C54576842E8158BB1199E9601AD4
:101240005428432DCC9DC9D54C315E1C62B2E0C5FB
:10125000FB62832594EE9C39274EAA5C290B8531CD
:10126000CC2C2A8B277CEF257C2FFD26C62DFC0B52
:10127000434C0578B14D5420E1D997971F93BA8616
:10128000AE332C5A2A29952E8E33A250B3B454462D
:101290004C688E2844E8203A8FD91F520EE2381548
:1012A0003287A5C1CA9CA5CCF283780E19FCE14116
:1012B00014F80614512D542C2737AEB5E3AF05B002
:1012C000D708EE5D745532F709EA78183B282F5499
:1012D0007B25224F7E3C2C2FCCA05C1651223E1E3B
:1012E0005642196C618645015D30E8003ABFAE4751
:1012F0006C0CAF8E59BC1B9797DBC4299B37933F6F
:1013000069EF222742AEFA7586DD98FC2FF47180D2
:101310002B2FF7E38E6117BBCE70A913BB83E82197
:10132000CEF82E82876357E3BA16431724D159DCCF
:10133000F126B334A0BF3944B94CAA5C26CE15259A
:1013400042A8D871AE2411FD2A8CB2F80303138190
:101350002C4578BE186493A78AFD528AC0BC293CEC
:10136000DFB4943837364BD3E25096396469583736
:10137000C9C0FE7537C762BB6038B80C325F577999
:10138000E1C48DC561FC19CA522E0B799D5B0F67B4
:10139000284B1CF62E5A1AC64BF9E6374BD15EF194
:1013A0004B41C8CFD38DB557FC72DACF5096F64A71
:1013B000400E0A92F335C8B924F0348BECD9106B87
:1013C000903124D8942BD760883522A4206C715D8D
:1013D0005D79F90991ABB1659D4156164FE209411E
:1013E0000E39448BB3E1FB38728538E8C5D90A0C55
:1013F0002128A4941B52AA2A566B08132588568AC2
:10140000FE286E1347490C927725F749A2441344EE
:10141000E1A262F1F7E281E2F3A2BDA243921CB124
:10142000A19AD9FF77BAF84BDA25B65305E2C5FE83
:10143000FF7B68B6CBFF00BE2C1EFEF3DA9AC59D7B
:10144000F405E9618BCD98F933A4AC4DE2C21FE0FD
:10145000E0CB9DAE9686F079814395CBF0A522C76F
:101460000F12C870C78F12630B6478CFE47DCB1264
:10147000DBE976D598D77107995DBE18529E8B62CD
:101480000EF7A0859DE318358608540413F770CF36
:101490001D05F77A790A0418300726D47F60D2E94F
:1014A0005E3593691799A37BE3593FF3B7F1E415D0
:1014B000FB0DF77AE727181231DABED1BFFF0DDA3C
:1014C0000897C2FAE011FCD7EE24BADB4FF66ABDEA
:1014D000C03DD0BD9737066E801B791E7C0C3C7DCD
:1014E000CEB83FD538DE67845CDBA547D6A1A9D945
:1014F000A74FBB3CF9FB686800247D8CB91FD3D98A
:1015000042EB82A8B653963D3429DFFB20633A7A3A
:101510002260F8AA2FF34E93C6325FCAA0B37D2192
:101520007B2D54165622FD51FA8BF48E143C98BF35
:1015300087067D98E552209A64B1D3F60D96227AFB
:10154000171A6657DEDC43C38F646BF14734948906
:10155000BD10880C140B3AD44C17EF2627A0356227
:10156000942B4D68970859D744670FABABDBECBAA7
:101570009BE2BFFE8672158D8AD24E20574D357381
:10158000F5C558C209842050B52C3E1644173F8D2E
:101590001562A6445A162FA0F2BFA4ED119DB17694
:1015A000DAC2EB070F6756CB883A805882E3287679
:1015B00070F13E1A7A5F9CCEB28FDE7B282A55519D
:1015C0000F174C8B0892E691DA5FBA226702CB388C
:1015D000133BBD2CFE937D7471316F1B18A44F1605
:1015E000BC37D38E220AF26702E650746ACAA1E1C0
:1015F000A9BCE50EA9C8BE37CDBB2B9AE8D88DAEE5
:101600009A39C4A42A57D9416772C4B321876A386A
:101610002C02FD22FDE7F933AB990F3E98196B3090
:1016200074D813CECD9250332A7E1641C5138175DE
:10163000B7AD328B0A15A8B88436CB984619F9FC99
:101640009BF0995F42E7FF8D8E353C2F4379717B8C
:10165000F2EC14B26E9B980DF1637D6F62B60D597A
:10166000B7C34A5BDF815564DD31311B624A86CCEA
:1016700079365AB94C02BD5FA45C06B579B3EB88E4
:1016800081490E613E0B017B5A49A8992CFB79FFD9
:101690002EA5F33FA78B3F868719CD9007CB50D15E
:1016A00052E438DF62346BAB19C745D8EF852A5E48
:1016B000166FA3D99013F4412DBCDF14C36FA75448
:1016C000A864606851D60CE16F91E352B4919444E0
:1016D000E1D2A2DD68E7B695EBCAAF225319FFC984
:1016E00087C052B45492BF93CE7F9FCE2FA0418F1C
:1016F000FC0F69620FDEA6C4062B89547B362FF3DC
:10170000300895805089207468BB50796891B7394A
:10171000BA24853F60D6869E62A0836CD94983C86F
:101720000DA275E5458E511EA20879373A4EE77D28
:10173000B5149CF2C94EC813D0A2D84A0FB358E9C9
:10174000B3BBE93CB11DC341B96947AC416B20AAA9
:10175000018B0EB44129E80BDA42705A69C8AF4BCD
:1017600029ED6F94A4B518F8808EB67C44DB5596AD
:10177000DD74BE8DB61BCD0EB06EF0DB6C420E3A42
:101780009E8A379A4B99BBA1906ACCD4906A068204
:101790009991851964D50CA4408FA4F91F77A78E61
:1017A00025C97A5942CAC2B65585FAE9CCAAC9ED0B
:1017B000095FBC9FB61C8048DCFF215DBA6D25D156
:1017C00051446C35E512AF73CB306290551FD2296E
:1017D0008B4AB7AF4C297D87DCD82B5C0C2D2211AE
:1017E0005E16BF2ECDF2213D774598F617860FF194
:1017F000D0BDCC6B6190717BE853B44B5E7C80D6DE
:101800007C18676425E70ED0730787EDE3DD09E6F2
:1018100062B4E170E723FA1A7C97C5E7D289C8AEB3
:1018200000FB1417D0CAD583137946503817FE86AB
:101830004BC4F6C0AD3D1E42790702E9CD0F218AA7
:10184000DBBDBAEA7DDAF23E7D0A72614A9C14C1C0
:101850002770196629F0C7D1D902BA64989258F155
:101860007DFAA695FC40B0E06F0CA606AD1795C5B5
:10187000A70061511A64E19C3973F642947F106E9F
:101880001C5A42EF2CA1D7C51A8ADFA7438B0E96AC
:1018900002AB6B595BC3E708C30C5CF62354BA6D0B
:1018A0009518176C5B55FAD12A315DF0D12A08EEF4
:1018B0001392B278D7B78655E1CF853F1BFE4CF81F
:1018C000CAF0B4F015E1CBC3295A2453307A130976
:1018D00021D9D2D0A5F07CCFAEBF2389688C788C7B
:1018E000648C342FDE26531AA320B964B610E3703B
:1018F000D8436CA1C661B087DAC28C43610FB3854F
:101900001B95B087DB228C43608F38CD0F45E905EE
:1019100012764BA5BB102A94A0435214C7BA426C4E
:1019200052B63FFF497455AED414AC5F79555A474F
:101930004EE43C3292FF6C476C769D7423E492D85F
:101940003596F52BEBEC11701A4B42B178B63ACEC6
:101950007DCAED8A01C7C2A71422A338517DF61BA8
:10196000DA2586903361CB37B4F54FA9D99096A785
:1019700048052BF27E1851CDF094F9FD6966A1C29D
:1019800076F6F839578BEDD429CA753BD6D016B9FF
:101990005D7E5AFE6F794CE4B8C819FD5EEE773A69
:1019A000B23EB228F2EB482A52117939A231E278DC
:1019B000C4BF2380D569CB6C3544B0CFA2575F3DFF
:1019C000450ABC5E7DCAE712D92933F9C7A3ED6D7C
:1019D000C1C8B62E486F30D2DB8EB47BE0DC2E3629
:1019E00007301E57BAEDB4F93BD23E91B90262AB53
:1019F000A2C8B1C167345738CCB0BAA0DE1CACB8AD
:101A0000F75ECBF7A8BCBC9A3958019CCB614DE47A
:101A1000D72475B9FD16B03BAB57BB5A7BC0350612
:101A20007067BE477947EDCD443268613B1FA237EE
:101A30009F270D6CB63A3F91BCB23558D756BFAE12
:101A40007E23D8BE850A1CB18606BEC56BE887908A
:101A5000C9B28694E9966092968EE71977BDF66FC3
:101A6000F33F365694C583EAF6A2C3BC7C383F6385
:101A70001A73B0A2FC9A1D99C2AE910FFE7C581940
:101A8000036CAA99D32EE1FF4ACC7A53CAE099E5B8
:101A9000E54564B110EDDC1474F471A0C94A631A11
:101AA000DC86BF7952FE76FA7EB075F2D553F642E7
:101AB000CB20DA2EB70CA6991C39497F528814C85E
:101AC000FAC7D4ECD3A75D1ED2B7F3F56A1205ECC2
:101AD00038B0B30E15950EA5CDA74A87D3E66FF99A
:101AE0009039452156E18F1BDB59E54A519CCE7C4C
:101AF000963CA681580CB7FBAAC1B5067CF5CF4E23
:101B0000BEDAC4FB6AF3FF6E5FDD0EF82A19BC650E
:101B1000026FC1B36CE7483B03B5420B86D2B67384
:101B2000829EE7F88297724940A6150CA7D3AA991E
:101B30008261B45DD6EDD2A514E11298A7976B2D02
:101B400002333F2FE1021D7C0112CA763ECE683E71
:101B5000CFA7570A84503A1D502B8DDC9604DFE640
:101B600013B00796A2E04BC0CF41F891D8B100FB6B
:101B7000D3E672C1C04E52699D450E8C8C422EDE5A
:101B8000019B1CD0ABD1A9BBACC82E15526D3A2815
:101B900033DD1F7BC44577D95F4FDD71DDB275E161
:101BA0008190D15CE6A0603D0A25C47CDC924EA702
:101BB00014F72785D985E10969A74E5279500BAFF3
:101BC0001E2B8BD7FE729232D5F3A5BF8C2FF665F4
:101BD000E6327B7F60651723A86EEF5B1F7F2ADBF1
:101BE000DE84AC4F3C956D3B6E7DF2A96CE063FDED
:101BF000C353D97564D82944F007CB08BABC1CF686
:101C0000DFFB31E5E57DE14E385DC7963A9796F901
:101C1000EFD89C3CFB8E1BE0325EEEE34FE5AE4915
:101C200042E4DD1014D3EDD9B92F2421BB28371D90
:101C3000567D6E46120A0E93E24134317678B738FB
:101C400068BF3098BF10D9CB85E221749C94831B68
:101C5000607A45E73BBC4BF71494BE37936F4371F2
:101C600046142247D7887B99B50A81459ECB2B7CA9
:101C7000C41C8F6185B88247E4E6A1ECDCB75176DD
:101C80002192EDDA3691593539D6F0F8804B83063A
:101C90000EFE6C40E840FBC027069C1F12A97C404A
:101CA000691AB267C8E3030260B0534A0B4A3AB8F4
:101CB0001DE4B08F9AEF428FB68893C082DBCD1EB1
:101CC000CB6035FFD162A1936087928193405F938F
:101CD0006510A48F252CF1C45D56054A7856425FE5
:101CE00027976D2D4AF249AE0B6C4CFFF0B3B7EB62
:101CF000DBB9DE0D70F5F4C21538DE5D8928FEA271
:101D0000CDA35CA947FC5581055C2477026C4DFF8F
:101D10007DB6263F5B5310DBFF5D7702EA21EABF09
:101D2000AD1E7CF26C7916BD88FEBFE74E7B14B207
:101D3000B17E8BF9EDD5ABB50CE5C2F0530232079D
:101D40009065F141B4458086E2946D51AA1D7A6197
:101D500033099B53D81025E084CD246C4E6143B4E5
:101D600080133693B039850D6101276C2661730AA3
:101D70001B1209386133099B53D89058C0099B49FD
:101D8000D89CC28624024ED84CC2E6143624157064
:101D9000C266123627BF914E61CF36BF030560DBA6
:101DA00044F3F6DD79EC1F77BF7D70FBA238390A6A
:101DB0002D2A9779E307C4AE83D2F02E983078EEBF
:101DC00030BF7D3C2F4FB2F4EDA579A658DEB0545C
:101DD000E2AF308AEF5117EBD4C533D5D7C82465AD
:101DE0009E3A7512E5894F89A8BC8FF95EAF56EF10
:101DF0005A83B7D249BB10BD559C64CFB688C097F3
:101E000024D64758A82421F8E116ADCEC7EA5D6B69
:101E1000C7938B4C978BA2F68B488614000CC4C8D2
:101E2000D8380C0A3B2A8618F9B0D893BA7530080E
:101E30001203BD40E9F73C902BDBC9812CB60BD9CE
:101E4000629E6CD07F228BEB42B684278BEE8B6C2C
:101E5000E98BA4CAF266758C6A369A5793966ACE55
:101E60002844E8E06A33530E8B9A2C23C832922C14
:101E7000B3C9924896D164194396B16489254B1C25
:101E800059C69165222CCC3EFE701E591E21CB7C7A
:101E9000B22C20CBA364798C2C8F93E509B23C49FA
:101EA00096DF93E50FF098D129712CBA665E9906FA
:101EB000CA5D53F2BD75856D8C70B82AE8F0593053
:101EC000B217CE52C16A645F0C6620FB12DB387E0B
:101ED0005F669B182745E46AE835F3F8581259669F
:101EE000BA2CFE0DB3287499A8C891E3339A4575AE
:101EF000FC26AE663299ED43991F872E2431B12717
:101F0000CF4E59B74DCCB649ACEF4DCC2E8B2736C2
:101F10001199A5CB44D61D13B3B59089A22B52EBD2
:101F200076C0D3C4EC7B0FAD40D6772666BFA15CEC
:101F30002943E63CC31AF19A416BA2D78C06716F14
:101F4000DA7352F6D9B3E328CB7AC864E17A91E325
:101F50005F438D961C35B4653A2EC18CE15C6C9E56
:101F60005148FB459879FEDA2B52338AF3714520AC
:101F7000BA9A39A8B598C019DAB8A3624CBE4E9F78
:101F8000765DF7B32BBAFB02C99738CA46BF4EB38A
:101F9000E2B8A8501359424349A8A3229EB5A83BD2
:101FA0006B3F5BEB1A0CCF2BAF3B815C6C357375D1
:101FB000EDBE58C325599946C80A44E58F509F760F
:101FC000B5C4B690400129404543AEF07DB8FD440C
:101FD0000641DDED6450D009CD9F440B27E001F4AC
:101FE000A63D3B655F597CE68EDD793BDF99684312
:101FF000A0A719BCA45C868A1C2BC01968E78E892F
:1020000075E46BE7CE8975C2C7F689A4B0EEDC36FD
:10201000B12C7E8760E585FB087FD0D416337A9695
:102020002BDC362A4E7E4ACE4AAE8E8A3510E04FE1
:1020300043C8292B3A31CA60B81ACDD7159305A9E0
:10204000792D8A15890B016B14FE43ADE1B04583F0
:102050002CD350FE24943F05E5C3C76B287F038A29
:10206000355C8F418A103B46E659CCC2E106E163FC
:10207000E67083ECCDB2F8146279F2943433DA4826
:102080006F10C521EE9A59020F9114399A8D46B3FB
:10209000C4D102AB94448F040ECD21607EFE6360F8
:1020A000E0238C7C9823C006C0B75F68D1172BCC87
:1020B000729B9A0F5AE5B27E458E877D46629D7E61
:1020C000E06A0E9B691B8830B9EE85F2B78766819E
:1020D000413FF0CE1CE53279E69EBC02B0E440ED13
:1020E000959082ED136D21053BC05E3659C17B137F
:1020F000ED5401319A3F341712060C8BE78AA36D19
:1021000061E6109BCC1C06F710446138845384B9F7
:102110003F1126B7AB90F68A3C143411A580D850F5
:10212000B388D70F02F7459F510999936616C19B53
:10213000CAE20F86005AB98CE876AD9A11038F6B0C
:1021400056E84E7575E5E5D5CC89FE8A9F084B2289
:102150007C99BC68072C7BE17480E22488023514EA
:102160002E19CF160298FCD5BB9EB4F503F173E689
:10217000CC2972BC176D344790B02546D25E190841
:10218000457BAF0D5060982236049EAF5C16014F20
:102190008763E5CA35181E42C8002D4145DEA5D12A
:1021A00036A999B20D3423E6CE643EA29F8BCE8829
:1021B0007E293A2B1AE84C836D1173E69814B09A75
:1021C000C26031CB89F94CF068E5B290221BAC03B8
:1021D000CD0377C0EBF71A10D47206213A53DD5FB6
:1021E000AD52A7A86733B39923CCB3EA29EA0DEA25
:1021F000AF9883CC6C1EB2E1FC35662E93C8FF5BB2
:10220000C1AF69FC8A60502231A23125A2910851E8
:1022100014A22488A2691A13D4BCD0F9A14B421786
:10222000FB611E3FE7F1FB62FFF7E220FCE26EFF7D
:102230005E8EC9F2C33855564CC73F63CC3731CB9D
:10224000541DFFFFADCA6AFFBE1AD3F13DF793904C
:10225000B95B42F67F4E8363B4C3860D2BC02B213E
:1022600014EE2D10AFACABABDBFA399449526F389A
:10227000A3998648A48B1CE75B8C666D35E3B80890
:10228000FBBDE0FDA5F4DCE709393BECF4E9D370D4
:10229000BF14AF24F852F1CA0E74359396664720E6
:1022A000A92C7E1170334BC822A403783A053CB6A2
:1022B000D79E83F620265A9506AEDD6B3792CF8DDA
:1022C000685D390CA07722C44A0BB6ADACDB6CBAA2
:1022D0006D902D2A8BDF20EA6053CEEB87CC21C096
:1022E0006F8FC0F1940A95603B830849F9B110D70C
:1022F000AFC02A165E295B546E43E648A0420295A1
:10230000CE4C2F152D95D8F0BD1080C3CC18581C7D
:10231000AED61C4405225467C3E5C7B0AB91D903C0
:10232000E10CEF5BE7B74F4F16B2459AE1A1F6F526
:10233000FCCBEDD9FCC363416F4EB62865A9AC9CBC
:10234000C8328BF855C27790D1D2E352569AB62E46
:10235000560997D2D67518BF67F6FFC901B15A6002
:1023600003DDCA1C0DCBD26843597CFEFB747E0191
:102370009D6FA599CB1288F65DDB5615EAA743E160
:1023800035C085B3BBE93C5CBC9BB65881F5B5381C
:1023900015B2C0CDF769C0580ED096FDB401FEA4A9
:1023A000147F44F3D5382DCEC8E3ADF4FEDDB4F68A
:1023B000064279E1F0F7A695FC4EBB6E127E8C5377
:1023C000C1944841E8A2E27D749C0EEDDDFF214DF1
:1023D0002AECB5BAD26D2BCBE2770E4F251F3BA36B
:1023E000852D26151EF5215D5C40436B52AE7A9F0C
:1023F000DEC9A4165BC99F9DEA54BEA4030BCB3E65
:102400007A9D219F574B10D5E9497743F7E4B9BC32
:1024100006D2D78C968F6946A566A68690FE62D9AD
:10242000435E6117C15E5C44435429574AAF15DBD4
:10243000852FA83F45801C4254B68BE1CA2E85C229
:10244000AE24FA83F2B07E4B56CB621A5AC3D3F451
:1024500035CB127A8765194D70B25D0831C7D4BB90
:10246000F498AC2609599D21644511FCB902D6FCAB
:10247000E9886F1F6FACFC2EB9082C5EA8F777C7F0
:1024800037AB9914D21BD2A0CF8145A1769E5BC1F8
:10249000FBCF0EDE2B8B27E1A015CE1F186D2CBABB
:1024A00004AC5AF8B382EF9249C0147C2F6CE785D4
:1024B000ED6272E9F96472FD5291E3C934E8908EDD
:1024C0003FA419B557504B414DB20D15B89309DFD4
:1024D00082EAE4B2F8D20B817BDF66185B0AAE2495
:1024E000434E15D426BF51F033DC29FD577288A91D
:1024F000E05FE4DAC5E4AD8711AF80F7D1D1A497EE
:1025000042044D9F3B7424519CE86DBB477363E9C3
:102510001D5ED143DF252B5ED870F8D0459E73D168
:1025200022205857160FA790B210B7E0C2D0A2438E
:102530003F272B575E4FB6D249A89A39F4EF642B48
:102540004A4287BE4FB65249C89E6D15C19FEA6484
:10255000AB3489F002FFF17497C02D8E99A38DE200
:10256000E9E6E92DD5CCCD3B88EFED7ABCF7945E5A
:1025700091F706AF52F11D1427E5EF929B0F71A35F
:10258000C95DD33FC1E07B0E97FE9B2850E4F8DD88
:1025900068BE458AEC081AA472D9613302DC9564DE
:1025A000B3B6F46AB27946C0D0ACEE142C0DAF9B32
:1025B000103BB6E07AF21B97F61C2EA803931CD4AE
:1025C0000E8B33E6D289C826CAC589A042DAAFABE2
:1025D0000727A2A27253085C2B7F83B4BBBACB2817
:1025E000EFEF1F5C4FE63DBDFF30EA2A991CD52571
:1025F0009B11B4B743D793BBF0B3219EA1992E751D
:10260000279B25A555C96669E9AFC9E6B0D29A648A
:102610007344E9F7C4A6450EA4860EE4A061EDB7A5
:102620003B6C0FDFF6E40537922F2D2A2FAFAB233B
:10263000FFFAC1BF34D065EFB1883C52ADC877D145
:10264000653AEFFB1D20BCE0574135DBE1A2950B5D
:1026500069905493AC7C9597068BA8F43A91C10E7F
:102660002ABD913C6CD871491E6D130133A8319776
:1026700069570D4F07F6026510B94D130589808320
:10268000F4CEC741FA319477C78EB20BAA92ED8F80
:102690002F8238E3EF0B71AB5D0BA5898F6751BBC0
:1026A00068C453127151606E9718FE9AEA891DEB47
:1026B0000ED26483D7802D7F12B848A1CEF4ACF23D
:1026C000DE80CE3BCE4A905F61E532C4EB9C571D65
:1026D0006B80262A12896811458B640A460FDD54E7
:1026E0008F4D1267088AD02BD68E5E1E9B199B14C5
:1026F000FB78AC6EECEB639F881D3076F398DA3193
:1027000099630A467B46E78D7E61F486D110577B3C
:102710000EFB2E42207EF06B32F3BB91F0DF1613DE
:10272000875D98D93F92C77D7031D98E984F47F118
:102730007FE009F64AD0BDAE2CDECE61F8B8B7AE68
:10274000AEBCDCF90DCA6BB4E721124ACA956A54D3
:1027500044BACE7562D5F6430615D5D929FE348024
:102760008418F2CB862AB6FB301418DB342DA71D53
:1027700063DCF9C983C38611EBB819E4BA669BB66A
:10278000FBF0CEB30FF268A57121A05DC1E872A87D
:102790003306060D44114886C448843000CD03E555
:1027A000073202DF0286DC11C16D19500D440C8224
:1027B0007793D2C9348DE2DF6B2051409ECA6133DA
:1027C00002AD79CF52A074597C9D4D50FE042A076A
:1027D0004311370E33D39D8E9DE5C8E5F23FF503D7
:1027E00072C653D605BF972F247B0E4309BA9E7C31
:1027F0008A6245F70AACC93F0EB3A261FC7D9ED147
:102800008FBCD5A19A5D4FB62B0AEA9381D72D7064
:1028100047C11DB86F1B018150C026C7D5D71734DB
:102820002613B58996961534B3622CD0645A444465
:102830003DBBABA08150BCF8905D5240442FD59079
:1028400078B33B3933DA9547D991C99A969A0D1ED8
:10285000B62E4FCD3E4D86EB5AAC81C91D6B80B86C
:10286000849AB38266EF425615F3CC40F13729DBE8
:10287000E1950954D1A155A973F86146F079AF9952
:10288000EE3810D9E8E3A2BC489B084E3793E1AA82
:10289000318DE7FF1D7AD67F075ED17E1F2A77C173
:1028A000ED642259B8FCE51B6CFFD2BBC970A5D4FE
:1028B00093ECC7B86E0A27F062E1106C21E801EED4
:1028C00027E7B7C1B6F92B68D09C77A5A8DD959D01
:1028D0000EC00E7014EC6D3B4D4E786F4349309333
:1028E000E53862C5F7DE2B548572E7931063A000CC
:1028F0007FEE0A214E0326FF4A26B6313F684EE19D
:102900003337D47C3754B9EC6E91A32DD6687EC88A
:10291000C1C1FA70ACA16C46CAA545616F82827FC5
:1029200002A29C947DE0B207836E7B5B63CB66144E
:10293000F74BDC377E5D4B9A7E7C5C397A0DE9F98A
:10294000F5FEB85C58FF1A4702B7B7F557FF00D637
:10295000932D53D465F137736903631D4782407F1C
:10296000E2C17CB99AFC14E4671B1D270F49B784A8
:10297000A96D71715E8B0CEEDACB912524D1FE1A14
:10298000B248130D06DB5A7674BE5ABD6B0DDE4A93
:1029900027ED42F45671923DDB224AB2230B4AB234
:1029A0008FB05049105661894BD7DAD6B0B1F9B41F
:1029B0003A1FAB77AD1D4FEE325DEE8ADAEFAEB166
:1029C000BDC06AE1C163E330298F15438C167112D3
:1029D000C472EAD6C120480CC40299C932480D1409
:1029E00040AB6CA77DC1F6579E36B60BED629E7666
:1029F000509FB47FB5BDC80EDA93670FB16E9B9838
:102A00005D160F954786CC79D0CE5F240DF4795AA8
:102A10001339272FDC36EA949C55D8460D338F3274
:102A2000D846B112DBA87BE10BB02126CBF3341FD3
:102A3000F6CFD38A562101DEA15F174135B48EE36C
:102A4000EBF4010A39CDE80042CE0AA8B32EA69ACB
:102A50003965730DB3A1D73DAE81F645B9704E9A75
:102A60005C0A7173519AF75F40F4F1F8ABE3BE1C56
:102A7000DF6FC29571977930407539709D3356DCA0
:102A8000E49CF6BF17131221711F447651C43BB466
:102A9000E51D3A2097763D0377BD46A762E281EFB8
:102AA0008DCE3925630E9C373AA1179C92A2BC614A
:102AB000A72251C920288B8C717C5E04096881385B
:102AC000564B0478399E8873CEC90322AE2B91A948
:102AD0003B51ACD220BB54CD4022389C46E729263E
:102AE0006FD02977493F85E8D4C7796190078390F3
:102AF000ABB605AEB5C0BD6AE69A651B6DA7FCDA3C
:102B0000C2DF53CBF268FBD2B3876836CC7208EAD7
:102B1000A19D46CC5D097956C79D5C3A11D997E6CF
:102B2000E2443E7641C7C18928579488E0ADDBE88E
:102B30005C49627B48036A6022B26CA70D40C6DC28
:102B40008FEC11CC36641833E1CB099726CC9EF874
:102B5000C844217EF9A28CCCA3ECA65CA446CC7B15
:102B60006AC63C9C510E80FBCCA793999F8631DFAF
:102B70000E630E0DBBFAC2D5BF5E7D71E9C770F35F
:102B8000A29D78D73ED0B299867297AD84C5A958D8
:102B90007AFB6A34F03FAFB647C2029C4721302926
:102BA00018813934DC1E47757C23F2207B180255CE
:102BB000ECE1FC2A125B86D0CC91FE06DE59105661
:102BC00057A3819E121ECEC44C64F2C63143A44C5E
:102BD000DE08064387928DCF1B5B16EF00FFBDAF6B
:102BE000FD458620408A1C83271A2DEFD23B5C329C
:102BF000BB985099247609D9BBD206FA3A44855D30
:102C00006E1E7560496A362BB52D54AE349917DAAD
:102C100016C6B12CD6FEA208A1CD0B63419573A5B3
:102C2000B44B5CFC356D8E3674704801524B296D87
:102C30008BB67C4DDBB1393A360D62A4A330E55337
:102C400089B6E9501AC2132178E75946AA6D0B2CB0
:102C500063D4B6C72CB16ADB1396716ADBEF2D9390
:102C6000D4D0EEE65B46AB6D0B2D12F8DE1353B7F6
:102C700031C6A6B688D5B61196096ADB48CB44A8FA
:102C800033A4C68CB184AB6D632D52B52D166A8DFD
:102C90002DCE12A2B68DB384AA8B67238B465D0C12
:102CA0008E8D57173F80E254906C53D4C5F7932F05
:102CB0003DF94A225F0C7CD9265922D4B6C964D189
:102CC0005822D5B678B24CB1C8D5B6A964996681F8
:102CD00092F63BB24CB4506ADB83EC50D0FA21A898
:102CE00067B687A19C819AC9211A73B205259AC239
:102CF000C89FB80AFE0F38A95F22440052332FC67E
:102D0000310386307F1907D851714672322C9E5993
:102D100010015C2EF215A79AF1CED5909CE46F0FAE
:102D2000D508A6B273D4701271852C890A66D56451
:102D3000F844062897F0B98B52BF80EADC116A97F5
:102D4000E70544BE06A95D77F9FA943F589D3F44D4
:102D50009D3F4CBD6BB85A40A901B56B247F7F1ACB
:102D6000DCB773162AF1D75F8B1589A01FF3F630F5
:102D7000E66312B62478950340F0B4FEE62FEC45E6
:102D80004F9ABFE44B443254D9C4620659A6AA995B
:102D9000BF0E071A4D2B2C8A56E6D989B6E850E8A3
:102DA000451C02EDE142EE54359279A326C44276E9
:102DB0005042661DB8478D0EE860CE54234B3FDA73
:102DC00074E4D222D99BD54C8ADD94B22F4D68632E
:102DD0002B3F9E6C1E0A828CE6E165F13BE27CDCB7
:102DE000DE4510FD0787AEB322945D5707BDF9EEAF
:102DF000BED8752D06D27DD0A853481A9772495671
:102E0000A6F15B2A1F25C283778528B72AA08B20CD
:102E100028D61BD1D6FEA4330C4CDAC5715B07252E
:102E2000D96928D1F943D5B65170DD46BC12DB9281
:102E30006608D66229885FB47BE84154BEC12F750D
:102E4000B3AB7E5F6CA73BF98392F2FB27E5E740CB
:102E500014DA9DC01BECB25EBD8B3681585EC09FFC
:102E60001FD21881E4AEE649CD130086E2FE89AF99
:102E700053AEE6B2F86265A225111747255AEEC790
:102E8000C5C3122D7370714CA2652EE6F95089C02E
:102E900067B03E7FB0BE2C7E9702150FD6CF9994B7
:102EA0008CE74C4AC1A1A1D7E64C7A043E17E0D387
:102EB000AE5ADE0F83F5E0B1C17AF8C5D12E497E56
:102EC00032CE7F10170FD1C38FFFFF08CE9F8F0523
:102ED0004E08953E861FE2B882A77169222E780CB3
:102EE000CF7C1AC3775D9D5B815C97AB1948BD763B
:102EF0000535C5FC55CBD358D0D4F2189EF834868E
:102F0000BFD50CE908B683E6AF6C5F9A0FDABE3026
:102F10007F79FCA06694EDA072D957CA798978DED2
:102F2000FD785E329E9782E7CDC1F3E6E2798FE0CD
:102F3000790BF00331E62F620DFC8D39FE3FCBE3B8
:102F400097CF23807ED33039BB003909C217B23CFA
:102F5000F44ADF7F78FFE15346721C376AD4745815
:102F600053529E0368C7329AF44CCF277B81839BD0
:102F7000F5246827ECF5EEF57AD2D3990EFAA7D7A7
:102F8000DECDDFFE73FE05CF73D9435443674C8C0F
:102F90009BB93A393988BF469B3997F0CCD4A41BEA
:102FA0006EBDFF5EC5D633DCDAB5DDF5EF413346E5
:102FB00063D0EB0D4E53F0EB9C06BDC1A061FC94B9
:102FC000FE7F41E0A7E8C4C5E3F530E90B17F461E3
:102FD000438592808FF329F8AF3E6E06F4ED09E346
:102FE00066DD7D520671E8225BC30474F7BF3708C3
:102FF0009F99E5DDB8E1443078333383F04097EEB4
:103000002E29EC6405A62BBD4404102E532A348CC3
:1030100041EFF5797BC0276813F85B5DF9CBC2956A
:1030200051CA28ED84D88434F023D0CA64E1B22098
:103030007C5676166F738F57E0D3959EE70F16FB7D
:10304000CAEB3D716C6377FD058E4A856005C1064C
:10305000FA1EDEEFCD0CD8A107FE70BAE59CF7C5CD
:103060001740FE967288CF3E6DDE3DDABA60BBF93E
:1030700057248952661ADC26777A66549444D48D94
:103080003B42103BED6BF761720A940297CED2215E
:10309000BFB66C3EB3395CF00D797BF0FBC32367A0
:1030A0004D5D3B7BDEEAB6835FD416738E9F2B1794
:1030B0002F99AA8B8A0AA25728896F62139E4BBE4A
:1030C0007F39C85FFFDA518020BCD7279CF9BC7ECE
:1030D0001C7C05FB5F9B90957C62FD6BFEFC7AED92
:1030E000E889A5595A6D109EF875E3D1D7DA61E3E6
:1030F00031AFC7D3F9E57C860676FEAB937C2F7F94
:103100000E59D891C941F88459D949477372E034AE
:10311000B722F748CE91A34F67272404E10372DB5F
:10312000DFD6E57DDDEA5F17FE10AD4100963ED3A8
:10313000393E728EAC2FDB786C4BF90E5789C77312
:10314000E60CBC75FD919C3EF977CE1FB058ED8919
:10315000DA9B878B3801FEFEDDDB3FBCDD095F5665
:1031600053FDD9AEC6BFFDF0F60FEF55BC51B1F51A
:10317000E4C64EFAFBDF7F24005DDF1FF01FEF3750
:10318000538FF63BDA416FA9A878DA3873666FF48B
:103190009BB740A674969F95CDE39D6C66566424BC
:1031A000E6EF656505E1DBAB6230F4E09F00748D0E
:1031B0009F8EF3FB973FA78D4DD02A3AD3BFFDC317
:1031C000DFEB03B62370F3FEFB97DFDFD9BE3C25B0
:1031D000A1D34E20510ED1DA03DECFB99B7ED9C6E2
:1031E0006C5178A70AD3119F4E77E7EED2DE65DCEB
:1031F0001DF481AE13E8349A20FE40CF63BA420733
:103200003DF4CF850B3217645ED8B219FDF6E1E3C9
:1032100082E53B3BD5C39E075F45C233B33C5B763B
:10322000FCE8792E2D0823BC88C47639A93324FE06
:1032300059B6677AFE66D7FC10F2262DCB93BFE312
:103240008C9F3E2BB367FA3324C7BBD26BB4E950D3
:10325000D5A037EA832CD48D5EE0CFEB1E4E38F438
:10326000A53F40E7F7A16E591A8417BA61A7EEA8E7
:10327000713BBBF2DF7C06F2DFED66D91D79177674
:1032800074E5DF677D11C6971C77EA94E5F5B37E98
:10329000E886EF5DFF60FBF9EDDB43FF12E801AE6E
:1032A0007B4A4A9CDD7B94DF7E7E0B0A3E0BC61771
:1032B000B26E6750ACF72C1F6A40667877F9C4632A
:1032C000C1FE33A41BBAD1B7BFAC97F820E717D221
:1032D0004926A43382473A0FA899FE3AD035FF0316
:1032E000F4843A9D21D9D4532E05F8A7F3FC83FD2D
:1032F0002B0C884C3EFF4987856FFF29A906ED39C5
:103300006BEAC865832640D7A3F7DB6D1FA80C02C4
:103310004D30AF6E0AA235AFF8AC1F743F16F8748B
:103320001D41B818D52C86AF59FC247266A962BA23
:10333000D0735D472F723A5E247C47CA23A13226A0
:10334000CC4A68AF9CA44282FDBA1788F651C812D5
:10335000E843000AEE7F02D7EE3D2418DF192BFC6C
:103360000BE00DE990917D09434FAFBD9BBFFDE799
:10337000FC0B9EE7B287A886CE9818377375723219
:103380008F19353D41A9FC8FFD2D30482C900C71D3
:10339000923A1F74AED3195348E6E656E496932842
:1033A0002B7FCEA8D375A1F5FABC1B379C0800FC77
:1033B0000B92DF57FFE99BFEB7E17BCBE8DF8A1773
:1033C000FC59F8DFC60706540802FFE9CEFF327E3B
:1033D00041265BD897F486E6D6D43F19FF644CFDAE
:1033E000EB933DE2539ECBD46850BAA7F7FA260C74
:1033F000BFE78528E8867DDEC8BDF5D6456BA5D537
:10340000F5D645EEF9E7BB60FBF28F20BFA7FA23A4
:10341000D4B9D78E9E587AFFF2E7B4B109DA8E2C70
:10342000E8E3BD3D696EEA56A7048CD007B409599C
:10343000BFFFD78E1277215BE785B7F355AA831AB2
:10344000B0C9F71B78ADF8E84CCFF46EDDD24DC6AD
:103450005EAF67C1852D17D23D9FECED82E9D09F0D
:1034600064AE3F9783750BEA395DF5EB6243C9049F
:103470006D2CEF017D37AC48122ED36AD80BAE5EAF
:10348000ECC368FC3EE0EF69BAE1C9C8CACE52F8A5
:103490002B4C379C2C1C4E95DA096973CBB7EC8802
:1034A0005276C3339A593A5FCDD569D37AF5CFEEC8
:1034B000BB00205DA94837187A949F9995C9FBA352
:1034C00027F97C870A275316DED19FBA8E9E29BB27
:1034D00056D9CEB7D233D91D251077ACA7E7A22D88
:1034E000E04B2EB0993D6505E9FE3DE543E7D1A9E6
:1034F000FB7B3DA6CEFE251D05741A3962EAD34931
:10350000894B1297FC9C9FDF4D7B417758657CCCA3
:10351000A2CEF4B374D94059B67EA348248952662A
:1035200076B12FE10F55FAFE631B374844BDF89F73
:103530004497C80F5DEB2BE4E172E899F793FDFE29
:103540001EE90DE91943FF5155153F9296402DCFC5
:10355000EC563F406F4C63C045C60C98AAAE3A7219
:10356000A407FDB8EAABD384F8EEDEBF738E1C5916
:103570003C7B7112CDF3E8263FF0FE7FBEFF417821
:10358000B82466F8BA2EEF9748B3334964C11BF8E4
:103590003ED33DFE18CDA717FFF1F2E3D5893DF2EA
:1035A00047A447C1DA1BBD90B16ED693BFC3D953B0
:1035B0003791B5CB26D073FC0B12840177BB600525
:1035C000FB2D7F214B193578FAC86AA7B313362A29
:1035D00026CADF45EFD5B59E3DD52D3E10A279EB2D
:1035E0008BF8ECD330EE2EF4A41313183375C4D437
:1035F00025B3672F3E9293D3054FDEB4B5C2C7B251
:1036000026F2E50BD23558BF8084EEEF5340E578C3
:103610002EF9D8C68D185354B7B707E2FBB1571E21
:103620007BE5BB9D6F5DFC54DBD5FE60110AD3C901
:103630004B9FD36A15CA6EEF4BCFCC8A0CF7AFE025
:1036400085A818A9A41B7FD25B18CDA8E9CB93E667
:10365000AFE61A1A7AB0CF9869D362A2643DD997BF
:10366000F70E641F68C1D70F955CDE09EB8FDFAAE8
:103670009A29D3A306F652FFA0B6B6E75777FF0AFA
:10368000D54DE6AF6F5DF30F6851500E758BCF8E41
:10369000CEDA737D9785A73C47E0A1550FAD7AF848
:1036A000F9D3B95BCF74EE5F1D5D67C3892DE55F0C
:1036B000B16CB7F777EEE05DF5E3755BFFDA51804B
:1036C0005EF2C7E9AE8A575314F8B07B7D286401D7
:1036D000BAC9EB18A4FF1EDBB8A59CD4CE2D2736A3
:1036E0001EDDD5F8CD8FC1F591D168C0DEE9999E78
:1036F0002D9BC333B33C5B76FCE8792E2D08CF7B42
:10370000BE0FBC469B3937A50F7C6C42E682057D17
:10371000E0115A90D93B9ED1A42F4CEF53BE305E9E
:1037200034723B0FC51B532BF376FEC42D5FDE05B1
:10373000CB53837FA07BA4A7331A657A66074E6FAD
:103740003068FCFCF9DEC2DFE9F9FD3DE283DEDF33
:10375000233EE87D3DE24D4EA7410F5A748220BCC6
:10376000D01F3B62AC6B7D34A4B33BF2FAA0E723DD
:10377000A40F7C6C82569339373321EB91337C84D0
:103780009E49CBEC147F82FF4A3C9E33E55BDABB5B
:103790007027FD3AECE7EFD0BDDAAF277CB0FD7AB9
:1037A000C207C54F8FF860FBF68C17B450902C43BE
:1037B0003DD51632D2B23C793B7EFCEA7ADD99F2F5
:1037C000E73C2525DDDED7FE72C23F2B287CFCEFCF
:1037D000EB1D2FBCAF77BCA0FF6FE17F217D416661
:1037E0007A266483C6ED147081CEC9EED8C153EE3B
:1037F00070B16E37DF637AE21F4CCF210EC9504A99
:10380000FFB4FE4C548F06091A5C17E81DEFA3DCC9
:10381000AA4DC6DEF194AF87E6DC89B7CA2DF5F470
:1038200085F7511E69CF782F26B2B59E939DDE2E67
:1038300045BA80D65C16B77EBD0F7D94D581CDEAA2
:1038400022FBA857AB3BD189BF1379BABCDE68EA2B
:103850005D3F2FAE526DECD2DC295EE71AD599841C
:1038600001EC7335EF6D5CE2B7374672A44246AAAD
:1038700055AAF5543875E24A26D56934112E4467A5
:103880002FAE57713A23C7F1F6BA1DE930F9DF8F31
:10389000BD525E0B4E186DBE264F952FDDF8E380AE
:1038A000265C7B4FA1D38D32403F13AAF67ABC171A
:1038B000DC02BFA33A896FA8E7D6AD93CE18D96AC8
:1038C000EA0739D1498AE4D47DD226795B4C93F654
:1038D000DD3756C3ADEBF29F535FC9E2DC9CFB655D
:1038E00069254866B90FAA5ED954AFAAD475F53FC9
:1038F000D7651C4EF2324D2238A7047C96A982E58A
:103900003C6D3E9F1FAF735ADDABD33FD63E9EFF4B
:10391000CBD63BC9B779FB9AC0B26E946EFACA791E
:10392000C1DD99BB17F7E57FC4E9FA8C9F84A3DD5D
:103930000334387AFE53FCC9D99AAECD19A8BCB865
:10394000597A2BF272D48DA8D3DAFF5A13F02B4692
:103950003425A5E4D40CCF8ABA1DEFF67F90DBDACC
:10396000167323AA562105BFAE50DE9DC165DC68E3
:10397000AC6FACE13619546E5D900C62536390FDF0
:103980006EAA7E06F820558AAC0C8F673977A5DBC6
:10399000EA36712A8EDC339A8CA684A314F7D67388
:1039A00035310F67BEEF0DBC25A2F1A79AD64DADFC
:1039B000D2DAF9BE989F127C095F667EC53CBBBC1B
:1039C000F59823DD585559D372F2F38AE2CA66EBB3
:1039D0009F1C2B7638D2A3A869B821E6A4764BFAAF
:1039E000F0252BB80395B3B857BCF56CA5DBE1F413
:1039F000F231F2CA3A29D7208FC2CB17B77A884E54
:103A00002F6F12A4582152FC7A9B3867A513629439
:103A100015B436720E23A7ABD4D5AB7E1DD032A021
:103A20002DE44E488BC8875A446D12AFFB3AEB63C6
:103A3000EF7A384FAB9700D1DF68D2391D100756A7
:103A4000F7FC2EC5D91464198FB4AACFFA21678F59
:103A50007A3D7DFA8FF8AA777C4E3602BDFBA2D75D
:103A60003955EEBEF05EDC20EF1D4FF9349CAF4FB0
:103A7000FEC40E5DF11E69A3FC6EF895981B31DF44
:103A8000DEFBADF67DBEF8638A8094126331763A30
:103A9000759DB8E8BAE5204246B43E6B53D6C17472
:103AA00047BAD540EE3A9CA5470F9F74541CA8B462
:103AB0007226F070A5BE23FA8C844747F435909A9D
:103AC000F7D1D4B6102F2DE430A9793FBAC17F5E6B
:103AD0004EC86114F05E2578AFB3FF4CEDFEF35194
:103AE000C4F65EDCD6CDFE07D3C75F7DF6F21FCAF3
:103AF000BF2BFFF86B6EEBCC98081C8D55F83EE998
:103B00007DD2D49113D7DE585B0BB5A329E87D8D08
:103B10005C5397E7B5614ECA91296D9272721F543A
:103B20003D12579C874093A7D5D3C4726C13F96696
:103B300009C02DB9001C0FAACDDFCCCE46AFE6B42C
:103B4000816E1CD586EFE16671D99CD1D7E687E9F5
:103B50000F4EA858B9F5D10F1ECF7F3C7F8175A1BC
:103B600035D3C42216AA530022BC62EF95A82B516C
:103B7000C713BED50E6BFE5D23460190923A8A268E
:103B8000B30EC301C364B7D16D2C349670867A55D9
:103B9000000EA44EAEE4ACCD741BEDC33ECCE1569A
:103BA000ECC1F0426F0778E179C92F17EA0EE92AD4
:103BB000E406B0B275444E36A98D4ED080D862D698
:103BC00091D2A3C3BD2BDC95CE7B6447B556A37BB6
:103BD00078AB488A8783ED5A01483D6CE5BCD256E4
:103BE000DC4CF9648DE11E4ED2D424673DB73D779D
:103BF000C12E6011248515228E73723AB22155BDF3
:103C0000C31F7F4E9EBF5BE53036C8A55C94B7C628
:103C10001D097DAAA1B289F71F861A26F444B0B304
:103C200083440CA7D739491400BDD1D1094E7A0C71
:103C3000C67C55AD54EBCC656B398E2551E16EEFEA
:103C40009BE085F6BA0B19CEB1EDFDD51F37CD2718
:103C50007551DEB5EC96F519F2933ABD8343426F88
:103C6000E465221329806D5ED406E0A5DA78403E33
:103C7000AE13E4B26E4EAB3B29CD34C9D9132D44FB
:103C80007E47DF6E96421F4542C2904D31BCAD5318
:103C90005ED6787D7C7C236044513EC88B807DA0BD
:103CA000EEF3F2A1CAC1AEA9F073C0D6A78333DB8D
:103CB00047BDBAFEED8CE90DD31AAFD76C59AF955D
:103CC00036B7364BE5482EF476C0638852ABDED16A
:103CD00019B8CE50A9AB98BFE9C1A33810FF95EE33
:103CE0005C769367BD3728BD4DCDBE669F65128B50
:103CF00021CB10A9BDE45E05DBEA255DB622BD221D
:103D00007D35C0010D814A05494A1312A28874D934
:103D10006669B3B44522C0ADC85B9144732A085E9E
:103D20000D7F21FC10E5A0383DA72791DCB6F6CE2B
:103D30002B5EA38FF72D747F5593BC318C0D69A535
:103D40005B031EF5347A59AEB95DBD2636756193B5
:103D5000560EB97052B45E7484E1E443EA0F566CB7
:103D6000E23671EBB9A300907590773E2AF03E924F
:103D700073FECAC28FB9B9634F9640757173994685
:103D800087CA2367DB63873355BA59EE7AF5FB1B85
:103D900097471F8F9F7EB4F4669347E55451AFE277
:103DA0001629177969A6656D935CC7A51AAC50EF03
:103DB0008CA676FB39C08BC68E0EFB6176693BE420
:103DC00024E624961EED801C2E876B157501AE33FC
:103DD000DC8D64658DA14D905F4DE18DB246D9DDDE
:103DE000E606AE816BE4A10980F8D987201BE5A423
:103DF0003AD5CB05A9AD5E3E03A132B561FEEDF02B
:103E0000160E9EEDF3B5F16FE76DCB574D079F553D
:103E1000905D7A0184AC8237703A1E38B78E8F2558
:103E20009FDF86F52A159C1AF9E027E3463897C0EC
:103E3000A5E76E2631A742B9795CE30FB5072BA43D
:103E40009CBFFC717EBB8457F58378609C8CA05F1F
:103E500023E706700278110121BFB25056A7F42261
:103E6000C36A828E93E3A37DD0FD082762DB6C7F5B
:103E70000113E2136CCEA8482DF470FEDEA4E225F7
:103E80004B79B4D1E93040B432158A7AD424836CAA
:103E90007358B94A807A805A0088F44C2EE170A693
:103EA00055512B3BC9708C717DEB26E85D27CFD730
:103EB0009FE42A001AE4CDF24655A3FC3BD53F749B
:103EC0000DBA4F8DC4AAF5001CF4238ED8EE3FE442
:103ED0001787AE0EAC9757A65A532B55952A6B2AC7
:103EE000C75D69AD60ADEE00F07D998F360780D17A
:103EF000DF5B8DE40760E452F352F3EAD101548FA3
:103F0000EAF507F4F5905106136B2A710680E4D4A4
:103F10002D79437823ECAD906B7C56D118168AAF7F
:103F200012070C8EF4F7B30A7CDE9946A885467D0D
:103F30003D6454ABF4D5F53FD6B02040A82F1CFA11
:103F40002592453503EA034683087373355EBEAF99
:103F5000F1F1E54599A8A4DCED84FEC60F1F58BF1A
:103F600084C4901C2A33D2F1BE972BE470D7CA596F
:103F7000C1FE2ADE0764AC4F3CA2AF1175F4D71C1A
:103F80003E2F3B46A7D8077C70ECF39102310FB16E
:103F90000F39C0CA485722314F629F64019FFFD03A
:103FA000951BC33CED1248DC377A3DEDFCA1C955A9
:103FB000F2A186F8EA0551E4D455EAE0DDFEF88284
:103FC00098EF887FC0EBB80EF0C7175381AC482E2E
:103FD000233586C41734553EBA04535528AC105DBA
:103FE0009CAC49D98A88FEB97CD490C86AE2F14E6B
:103FF000C6CD54A14645403F12F36EAEAA5DBF2C1C
:10400000D4467929210B7C3CFFCEF1CF110C4DBA5F
:104010008491D78FE323DF07BE0BE88748C5575449
:104020003AFD12F8451EC0724D222CAA4255238E2D
:10403000A0239489F41C8E14C42300261E5FAF10A5
:104040003C4CAC43E4D773010F0BF23FD309E1289A
:1040500088E2F85AD75EED482521316FB0EAADFA13
:104060004D29EB091E629EC4402E546032CE3DE2C3
:10407000462CD5DAEEFFAD0DE4FD4103229FD7803B
:104080006AC35E920B7E613EAE8D5700625F7FC059
:1040900039994C5873F5254ED6940EC02200C88429
:1040A00066A9177754770E751D9CC9BA79FE917B66
:1040B000D81D992775ACDC4719752B540998F8B2AF
:1040C000A30F7348EF60E572E4F1507EA54C7C5E6F
:1040D00048DBF1826111EA503A20AD09EAAE0747A8
:1040E000DD1DEEF6C922801C32C6D3EA0D6D837A3F
:1040F0002CBF158E50AB37DAA373F972A19B0391D5
:10410000936B95B64A2B74E95CA51BFA7E107FB7BA
:104110004A875856DE89BF3C084FF93848695F27FF
:10412000BC2F080F99C51F06E383F93BA1DE9B4C0A
:10413000C64E78633B5EEA4B70D6E0593A5310DEC8
:104140000BFD1B21EB02EB827A4D7D3AA9593A888F
:1041500031B7C96D729206EF1F6E5587ED7BB27F46
:10416000C052BDE38FCCEA0B2FF5F44DAFCA322914
:104170009DB16886FE01D3A3CEBFA89F5FBF2ED698
:10418000586FBC636C81402278CA0F34C24884C423
:1041900048025E95A190F6F3DF02A1280C85A308E2
:1041A00014091E51A07EA83F1AD0E7FD8168101A9D
:1041B0008C862025FF6F281A86860355148A46317F
:1041C000502719A44623D048340A8D06EC1834161B
:1041D000C5C21E87C6A1F17EFA0968229A842623E9
:1041E0000D8A4753D054340DA8FBA1DFA1E9E81E86
:1041F000A44533D0BDE83E948066A2595079F56855
:10420000364A4449E87EF4004A460FA214F4109A54
:1042100003B71F4673D13CF4089A8F16F0D4FDD033
:10422000A3E831F4387A023D897E0FFFFE8016A2A2
:104230003FA245E84FE8CFE82FE829948A0C68317F
:104240007A1A2D414BD132C02F472B501A5A899ED2
:1042500041CFFAE903F01C5A859E47AB513ACA4058
:104260006BD05AF402FA2B7A11BD041DE265B40E2C
:10427000BD023DFC55B8950DD16582987C0DAD47CA
:104280001B90390836A24D6873A793CEF03A7A0393
:10429000BDC97F6D4116DE1E5B516E10E475FAD705
:1042A00017BCF5BFE4E5FF81FF81FF81FF81FF813E
:1042B000FF9BE0FA8AC6152D2BA834599A3C6D70E5
:1042C0005A74DAA8B4F16953D266A4E9D31E4C7BC0
:1042D000248D364526D2144599D44988C6C8148100
:1042E0001112937F9896D2A60914C232DAA4A011B3
:1042F0000A41A6F8D9221446C1261687917F1209D1
:10430000BF49A57048AE84937F325918210F21CC44
:10431000C650A290480A788686CA57A5BDB5B26035
:10432000A5EED9A455EB571D5A35F979F3F31F3F84
:10433000FFEDEA6F333232A44898B13043FC330EBC
:10434000E638FF1CEF9F0FC39C0B7322CC47FC7316
:10435000BE7FAE8699EE9F19FEF916CCB7FD739B12
:104360002823633BECFFE59F5FC0FF2FFDF36060F8
:10437000CA3232BE827908E645F87F49D6317F08D5
:10438000CFC8F811A617BEBDB0B7C1F4C1B70F763C
:104390000EA62A0266BF8C0CDDA08C8C5432876678
:1043A0006458C98C16A6834C7546462599A3810688
:1043B000A66A9C30099ED0111E44CFD5FE778EF799
:1043C000DB21042170238D30122131E2380EFB7085
:1043D0001BF6E256DC829BB10737E1BBF80EBE8DBF
:1043E0001BF12DDC80595C8F6FE21BF83ABE867F93
:1043F000C5BFE03A5C8BAFE22BF832AEC1D5B80A4C
:10440000BB7125FE19FF847FC43FE04BF822BE80BC
:10441000CFE37FE3EFF1BFF077F89FF81FD8852B4C
:10442000F0397C169FC1DFE2D3F8142EC727F109BB
:104430007C1C1FC34771193E829DD881BFC1A5F85E
:104440006B7C18FF1D1FC25FE183F84BFC05FE1C4F
:104450007F86FF863FC525F800DE8F8BF127781F0A
:104460002EC276BC177F8CF7601BDE8D3FC2BBF07F
:1044700087B8105BF107B800E7E3F7F17B7827DE38
:1044800081DFC5EFE0FFC2DBF136FC367E0BE7E1F2
:104490005CBC155BF016FC267E03BF8E37E34D78BF
:1044A0002336E30D783D7E0DE7601336E26CFC2A7F
:1044B000CEC2AFE075F8659C895FC22FE2BFE217FC
:1044C000F05ABC0667E074BC1A3F8F57E1E7F0B3BF
:1044D000F819BC12A7E11578395E8697E225F869CC
:1044E000BC181B702A7E0AFF05FF19FF092FC27F27
:1044F000C40BF11FF0EFF193F809FC387E0C3F8AF2
:1045000017E0F9F8113C0FCFC50FE339F8219C8271
:104510001FC4C9F8017C3F4EC2897836D6631D9E00
:104520008567E2047C1FBE17CFC05A7C0F9E8E7F2A
:1045300087A7E1A9780A8EC71A9C916160608ECA2C
:10454000C830C1CC89ED981F4E10E61132351919CB
:104550005530CBA6656454C34EFFCE3F676464609C
:104560009823618E9809FBEC8C8C24D893C8FE406C
:1045700046C612FF5CFA5046C67A981FC1DC302F3F
:10458000236337CC6381F96846C6F1273332AEC066
:104590007E0576D1EF3332C48B32324607E65319AB
:1045A000190FC04C26FBD3B02FCFC8580EFB72D8C2
:1045B0003792F98C30373D9F91B107E6C76B3232A5
:1045C0004EC07E12F6932F6664D406E6BA8C0CD9E0
:1045D0002B90BD3065C68C8CB13053FC937C9333EB
:1045E0001EF78A70374047789CF4F324BC890C226C
:1045F0002B2097E8B0DCAF13D18DD7D1AF33D13DAD
:10460000F00EF226F2B62BFEB7923793B707EC40C6
:104610006C426CF391DF56C46601FB115B26F96DA9
:104620004B6CCCDBDA6F7BE283803FAAFD3E22BE7F
:10463000223E3B32A1C38FC1BE25BE0EF8DD30CA7B
:104640006174643B5E7564395E71AC73BCECC874B4
:10465000BCE478D1F157C70B8EB58E358E0C47BAB6
:1046600063B5E379C72AC7738E671DCF38563AD230
:104670001C2B1CCB1DCB1C4B1D4B1C4F3B163B0C52
:10468000BA7ADD4DDD0DDD75DD35DDAFBA5F7475F0
:10469000BA5ADD55DD15DD655D8DAE5A57A5733B04
:1046A000DC3AB56E846EA46E946EB46E0CCC51F090
:1046B0003D42EE06A89257CB6BE497E557E45701CD
:1046C000AEC0570D9C54C9DDFBEBF7DFDC7F63FF09
:1046D000F5FDD7F6FFBAFF97FD75FB6BF75FDD7F42
:1046E00065FFE5FD35FBABF757ED77F35005DF359B
:1046F00070760570B570E717B87B0D686E006D7D3C
:1047000027DEB5F23AF92FF25FE5D772B81C5F4E9B
:104710005B8E37A735A725A739C793D3947337E79F
:104720004ECEED9CC69C5B390D396C4E7DCECD9C3A
:104730001B39D773AEE5FC9AF34B4E5D4E6DCED56B
:104740009C2B3997736A72AA73AA72DC142357CB15
:1047500047C847CA47C947CBC7C8C7CA63E571F24C
:10476000715430C451B1D4586A0C359A1A458DA48D
:1047700046506A8AA1DC4D4D5224CC589821FE192E
:1047800007739C7F8EF7CF8761CE853911E623FEB4
:1047900039DF3F57C34CF7CF0CFF7C0BE6DBFEB98C
:1047A0004DD4D4B41DF6FFF2CF2FE0FF97FE793041
:1047B00030654D4D5FC13C04F322FCBF24EB983FB4
:1047C000843735FD08D30BDF5ED8DB60FAE0DB070A
:1047D0003B07531501B35F53936E5053532A9943CC
:1047E0009B9AAC64460BD341A6BAA9A992CCD140FE
:1047F0000353354E98044FE8080FA2E76AFF3BC702
:10480000FBED1082E8BE06D5CB403D0DAE97E1FB37
:10481000EF8FDE58F628BF3765FB7C61DFE3FF07CB
:10482000EFAFCAA0D728D6BCBDE61D80CFD6B06BEF
:10483000A2D74E5E3B6D6D2F9C4412596878A4A29E
:10484000FF4044D862915884899138596FB2FF4F24
:104850000D640CA50206207A49A4B290D058F2014A
:104860000ACBFB2B635000C51F84868676E5C07497
:104870003D08268EE9D9760141F2982E92088A3FAA
:1048800089E83F5011829650D412449552E8DEB523
:10489000F341CDE9A7A869DF5253CF5053CED2F1EF
:1048A000E7684D85FF177F0E4EC83960A79F0A87BE
:1048B0009B910D54782315769B0ABD4387DCA56533
:1048C0004D0B654DB0C2379C9073C0C21D88C7594F
:1048D000325113D29329D6F193112F41836032E2E2
:1048E0004DF09FCC0AF43B9848264153602A644A15
:1048F000140953211B87F430153DC6D4FF0746CF5A
:10490000C9F87F76D0ADFF2FCB9F1B2A1629E51261
:10491000C4A1071127DF801342298EFCE1E859A1C9
:1049200062C485238906FEE0B9702C255FB4365435
:104930002C9EC60977F02C481E2E5CD24E205206C3
:1049400030DA763E7383F9CC6AE7D3E936612F0912
:10495000662F0DDC6EBF4308843B8437E128F049A5
:1049600009E633AB67ED53FEFBDAA7B44BED45F533
:1049700094FF55D5C5D3C247097C92810FD3BBEABA
:104980005A740F87938954F215A4FA3DC1AADF2304
:10499000E8C304307ED5EFE1D977F099D5CEA7D31F
:1049A0006DC25E12CC5E1AB8DD7E47D05EEBE7CDFD
:1049B0001B9E2748043E5141FAF86F27F8A54E2365
:1049C0008F4A2452C9173D2DD8F009C1864F68E798
:1049D000039869ED56480CE693D0CEA7D36DC25E1E
:1049E00012CC5E1AB8DD7E8710108CC0671A6FFE7D
:1049F00029FCB55D28ECF0D767CE9CFDE9EDC35FDF
:104A00009FFDE9E77A16ED42A2A4A953A78C18F1FD
:104A100076D2D429EA7E50D87A3AF1536DEBA0EAE7
:104A200095CFB66E547DDE09D9C98F5D3BFD63D746
:104A3000F6FB85B1EBFEFFFCF1917F4725C87EFDBB
:104A4000A7B6B88CB1252D2BB23F7BE163CDF32502
:104A500053DCE3FFB63977AFBDE4BEBAB7DFE81F7A
:104A6000FD3D5B58B367EB0D37337054C980E4E507
:104A70002FBDB4E2A5E5252BEE1FA190DFBCF163AD
:104A8000C98FDF1E7E7D338C929D9B7716ED6BFD6B
:104A9000A9ADC4DDD06FC4C851D3FE50F2128C3F13
:104AA000BCF8C2E0122671F2ACE1D13F5D2A395D5B
:104AB0007CBA74EBC5D682925361FBF39B87B7BA7D
:104AC0004BBE45FB27C60FE83FBA44B166E4A38F4F
:104AD000FE4E32A56454623C33453573764943FC3F
:104AE000EDFA7E88FDA924ACEDA78BADA77E79BF3A
:104AF00064DF37F9F643959E23250DEC7722B581C7
:104B0000595A72573276BAB449FD44C9884491EE75
:104B1000B262262A098D385BF27ED185C325DF7CFF
:104B200070E8F035E781D6922AB782EE3771F1D47A
:104B3000927EF18FA99F543F36BB449F18AF1EA0B1
:104B4000E8AF2AA15C6DE1CDAE8BAD25674BEBBC28
:104B5000FBCFFCD056F24DA4EF4E493F5A5EA2C6A1
:104B6000AAFEB3460C5494CC7F441DDF4F5CADC904
:104B70007B7CE2D258239BFB8FC292CAAF2B4AF2B6
:104B8000F38A4A6EB8EA5D7995472A4BC2C3FA1D8B
:104B90006129962DA1FAD38D9899AD2949EC3F92C0
:104BA000EE4F2926152EE02A8F96B69DFEBCE4DC3A
:104BB0004D676B7DC98FEE92736DAEB2CFBC7277CD
:104BC00061F5D19AEF47D0B347168AE3574B35BF0B
:104BD000FB7763A1EE31D5AA015F34F80AE5519164
:104BE000EE4FCFFD545978F65C71B8B3581655782E
:104BF000B6EDC60C794CC39142058318119BA82FC2
:104C000054EBF55306509A05859AA7EEBAFA2B1A7B
:104C10005C85D7146D372FB9BFFE67E127DE73A51A
:104C2000F5477EFE39CF3A6B9BEBC6CBAF8E28940F
:104C300033FD98795344230A474CD18C8C578B1BF6
:104C4000F266DFA63955D587970AB9BF9DBBF9D360
:104C5000F5CAB379CDDF14141F6E735ECFF33EAC8B
:104C6000626F8DD4E9F31E9D36E081C427EF4CCDF1
:104C70001B9434B091AE52A047DB0389B403AADF82
:104C8000B0A28FF695F5EB47FEF47022BFB9EB1397
:104C9000E7FE9B17B7F92E15D937DFBCC9DEA1A9EE
:104CA0007EA81F321A91082115DF524CAC5CC1CA94
:104CB000113529AF6DD6C07FBEF9FDC1DF97DC9AF3
:104CC000F4AF1AC7C41F96957FFDE48983B6439E4F
:104CD00079C7A67D78F86BDFE401ECE7136262E444
:104CE000BA01D5DB0B1F571585BC7EF6B331BBA7C8
:104CF0007F315751F5A71F1D9FB31BC73DE562A725
:104D0000667C1E7DEB4B4653B3C9FCF9D7AFDCF78D
:104D1000EF9FC649CF9E99ABE6B06FF29D4F3F1F04
:104D2000715451E59EA352ECFE6AD0D9E669BBEA04
:104D3000E7ED9E7F19DF4663C7CDDE7D9FE68A6F74
:104D4000D6C2413FEC1E37E0DBC7AE27AC6A2BDC96
:104D50007BE1ABD71DA757C7978C4C1C393231E983
:104D6000897B3E77F5F7A16DB7FEC97E7EF908F520
:104D7000DD67DFB9E8DDECE08331A3ABFA57EE7E07
:104D80005545A966ACF68D2FD4CD959F0EB50F3D38
:104D9000B45B4539FB7FF1B77F0DFF64B16DFC80DB
:104DA000A8419FCEDDDE38B5EADE27399AFD24061C
:104DB0007FE16AD35151DBE9B34D455993A8DBBB81
:104DC000FB3568263C5ABFA67EEF33FD26D7B00AD6
:104DD00044EDFEBCBA2DFA2F15BA59DB8F9AB5A84F
:104DE000EAF811E7F67E47ABD02CB5EE99C2654BD9
:104DF000973DB1F4C9A57FD85DFF3D42B71ACA22DD
:104E0000B79F3F449DCCABFEF9EEF65C74E419DD30
:104E1000E42C66F7A0B31974834AA32A5CBAD6704F
:104E2000EBC71B9F9CDDBE5EFEC53BF3EF360CD986
:104E30005DDD7843BFEB8FE872DEDEF2CD4A477668
:104E4000CD0BBB4591036AAAFA7DDE56E89BE7BA13
:104E5000A6FAA6F56CE1B96FDCAD9147A3FEB1BB34
:104E60007E847B524262455ADEA0A796FCF0B82CA5
:104E7000E9ABDD93D8DB37471DEDDF90F7F80B7713
:104E8000FA1F965CFE77DE7D57A645F63B3869D65D
:104E90006ED55FFAB9F5D513A83CEC9DFCCDB50FE6
:104EA000946FE65D7F63DFAFE77E458F6FAF7D3741
:104EB00062D4C6474AE7E7516DA25DEEC95792B684
:104EC0007F317CD2AD9FE75311797FAE89EEDFF061
:104ED000F330DFF62F2A47DC78EAF3C9EC0686CAFE
:104EE0001EA8F9FC0FFB362C7B6BD2D93B6F64BF3D
:104EF000B63D46C54DAA9A5C73673B37A8AA66C201
:104F00009D2AB43D5A77EC68D84CF53B2667E9C238
:104F1000920BE5A65253DD42792CAB9573A67463D0
:104F2000C6DDD193C70E311D7BAAFF7864FFF9035C
:104F3000D3C52DB23375BED668D3AD11B54DE831AA
:104F400085DEA4593D42C45E71FC6C3A5B7821F663
:104F5000A79FEA5913EE2F16613CE211533CA38838
:104F6000515786B3A69A2AEED6D163CEF9A65B989E
:104F70009E7A55A59B654AAC6E504D9C4855981A33
:104F80005C37155CC30D85C9C7AAAA2647C773A697
:104F900049531AE2475074A4498D54F20637A402CB
:104FA000F20F3DD2A15968264A40F7A17BD10C04EB
:104FB000ED104D47BF43D3D0543405C5230D9A8C13
:104FC00026A18968021A8FC6A138148BC6A231683F
:104FD000341A8546A211488D18C89418148DA2D091
:104FE00070340C0D454A34040D4683D0403400F52E
:104FF000876C5220398A4411281C85A15014826480
:10500000488A24480C298611CDAB416E0810E987E7
:10501000083F84FB21CC0FA17E08F183CC0F523FC7
:1050200048FC20F683C80FD80FB41F283F04868A97
:10503000A2849F8EC6F0338A44BA21D175D548F830
:10504000E6646261251F3204DFCBE71987998C9CE7
:105050003E53D9FAF0BE324D35938F12ED9425228E
:10506000F1CF5B2639FF7C36166EA53C92F608130D
:1050700085FEF3D0F45F2BCD9CBCC068B21A6639B4
:10508000659CA662ED16A389339186CFA18151E478
:1050900083436B51333A8C7C54548D701E00301E08
:1050A0003BB6B692E1501BDD2C19F42BE25879ADDA
:1050B00032188F103CC629FC6B436413B576C65377
:1050C00014879AD079F428CAE0F194AF034FD31231
:1050D00089C37131E9FC8311B93A18E4D0A12F9B3F
:1050E0007934617DD67AEF7AAFD75B59C97259DED0
:1050F000AF3C5F79C8405CD2D71C62E5E9B9E9B939
:10510000E42E192A5E0CB4058402523B2B103CB8E5
:105110002E802A2BBDB0EAF5081D39327B36E2C855
:105120005B11A77720EEC8ACD9DFB4726E80B030C7
:10513000A3D16AE5381D271085DD26D6EC90B4632F
:10514000070BC3ED76FAEDB063052B67E56E95535B
:10515000D7558BAEFA493D23BD940FDA80A933DED3
:1051600064143E85FF4ECE60CC32A60304088D2623
:1051700001847FD84B364933F6767D5EAB88AC6EC2
:10518000D58E15910D9266A9A72B5E8069DF46D555
:105190004436D06D1E69CF78955BD0C864EC99FF1A
:1051A000A9498FFE1CAC6FBD825891808F12768703
:1051B0005ECE82E7B9EEBCBDB88D86F890ADCFA2C9
:1051C0007CA61EF03AE737B3C95EA191B3C1911333
:1051D0000C4D322FF200B8989EF1BDBBDF83588092
:1051E0003EC2C33F3024BF1C0D91F58C3F26DD200D
:1051F0007D0DD3381107B87A90970712FD187710F4
:105200008045F8D37679FC58C0E9B91498FA6EF164
:105210001A20AC05E953260E0C0D965D09D61D1516
:1052200045298EA84DFA42C3DC335130BCB8415EEB
:1052300015E3D4B95567A646D544D5889F79B05CA7
:105240005EBEF82A4587864544D0F4EABC0A4D85FF
:10525000A65689BD61B7236ED16D37E1F5BC9F605D
:105260004FCFB99013CCDF47F9A8B5A8111D45EB76
:1052700049713360966EEEC05A0D727688E7B3A915
:10528000479370D2DAA9B56393D46B0738D16BAF6B
:105290003A7502B8556E15AB6A6E6E7E9965B3B2FB
:1052A0007C3EDF37DE4F7CBE90BBAFDF1518E8E1F8
:1052B000D5885BC18F2618F7DD17A30A97AFD841B1
:1052C000A049D624BBEF98CA2D6767B639B85C6E83
:1052D00013B79EC300C93E122BC11A6A753279B842
:1052E0005C2E97486A6B5F7EF924A773CA49EAB1BE
:1052F00092E65AE5CB1B3904B905F5C8C43D689C54
:105300000FD91BD31E3F42E6F82887DE2355721EB5
:105310008EE5E156B7F89B7544F810712F70B338DD
:1053200079373CC38DAD476E05AB61333D5A0FC134
:10533000D72BE0DDA082474AB209733E5F42825616
:105340002B78D3ED2632138E6A4F0AE46E95D7EB95
:105350007492088994CBE41A28A35EECD4513EECF5
:10536000256F2055B56B4076952F67556E9D335050
:1053700007BA839B8F441F40DF99819184DA486D7F
:10538000C15DF19315A98C43EFD01B4DD9269263D3
:105390005DF127A427A41BA551AA285582EE859765
:1053A00096AEF0F0B1EF0670A2CD684727FD691206
:1053B000669D063448A809895046945CCA7957BD51
:1053C000C9AF9088AFE76454C73051E29906CD92D7
:1053D0009A8D9BB6E496387C94177B312BAF89DA93
:1053E00094999BEED04F4B48CE7ECD47B549C1B77F
:1053F000439AA4B50947B373E02F114535C96A959F
:1054000009B3EF5F2CEB173E502A3B7AACAA9AFD0A
:10541000D4B83E3B27A66A384496D483BDB37D9862
:105420005758C20C81385F0FEAADF0D4366F6AAEC0
:10543000DCEB5799FA272DB5A8CE0F1A747EC071F0
:105440007C92E22856BE6E53ECC9EBF8064DB2834F
:1054500043D9D9D9CFB7B4782EE44749369E3B77A4
:10546000FA1CDD36B8996E6338B7D163D470D35A5D
:10547000294A2E57A9AAAA3096CB753A8C291FF132
:1054800058550CF1B0CE89BDEBD73737EBA0AD54F2
:1054900072ADAD0E4754D4FAAC6689D04D5B450E63
:1054A0007D54CD725F82F747EF75AFC723540AE191
:1054B000FD5E1CA8D4128914069121E0498D977ACB
:1054C000880C01AFD73B9DE5E56D6D9C7FE81D4ED7
:1054D0005DF93D1D598431A1AFAA6A6A12F0D84B1B
:1054E000E8AB629A02958E1FB55C23DF07D96EF197
:1054F00057CF35713EAEA595F4C6219CD48F17BA0F
:105500004220D388ADA59E30507BC689DEE2B437F9
:10551000F0F211D946B7D1CD92199208BA2B5EA8F4
:10552000DF97517D2F317EECA408AC23974B456368
:10553000D17DA27A85D64FD1EAC79B40E73CD6C839
:105540006709895932E441F492663717218757F089
:1055500090C5E3D9E0FCD1A51B37BC6F924746CE7E
:10556000189A89EE4A482E1AC150779BAB7C2C774B
:10557000B7F92593468FA621141E1E2591D372C21A
:10558000E9B5FBCECA7D50CDDA486BF421098DAA6E
:10559000114A422A54E1741B38AA4D167D93930098
:1055A0000A4AA8F5D6F5EBF5BFAC7E56778F6E327A
:1055B0003779566476B682537079DCA96C97D1A599
:1055C0006339E89760FF5A6EAC6E806AB80A5EE98C
:1055D0008F0A9D138A2F1FE35CFBF0C0D8BA35C831
:1055E00072E094AD1902CE6ACDCD3518D2D35353A3
:1055F000059CD5909B6EB0A6E7A616729C976B8310
:1056000079BD7EF66C278C76BF2B667F43AABC0FD4
:10561000A81DE07B1DB79A5B6254A8826D6F34A908
:10562000DC2177C36E87DCDDB97CEA9901D74914A8
:1056300074F50FB82612EC12017B989C52F0F520FD
:1056400082EB70739D814DE712400411F3ADC96484
:1056500065735BCB489FE427E2B2B3A1B38CF0B192
:10566000376FFA5ABC5F9B4C2662383FBD3E10BE76
:10567000C1A38B7C844C2696BD75AB036D32B2F210
:105680005B11013C450915E9C489CA4A82A7FC415E
:105690007662462523E49FC94451D1D142FE353577
:1056A000499A4D46CA175D2DE41F649190B560413B
:1056B000E2ADF46EF2EBEABD809BCB457191E0F474
:1056C00070AE5ED1453F8E7403A947E59EECEA2992
:1056D0003F5E7FF1C082BEF267751E872A19A2EB7A
:1056E000013DA9E3DDDFCFF7253E27C81A4038C1C9
:1056F0007A4EFF05B95C2CC6FC904A094ECE8A5BF7
:10570000F822047A21A4506466AE5BF7C10756AB59
:10571000C3213CCF607DE6BF3E586C351069817176
:10572000F9F2AD5B172F5EBF1EE07F79F8AD888B75
:1057300063AE0FF0DBC7E7747A3CB76F37360A68A1
:105740001FE5D479A4B7C31AC305FCD8B1C40F129E
:1057500049C07F632F103F489A831D6C34EA600470
:10576000471F84A7D3C391086DE58C1C89644F370C
:10577000FB6BB8102E975B0EF537B335B355D3D806
:10578000816915D544817C24F460062A2364B6A976
:10579000672B4B9A63AA221BAE0E6D1177C5109A28
:1057A0000EE84E89905424974586440D88193AF3A3
:1057B000DEE13188C35091A49C9C5FA36BA4AA86B0
:1057C000E6C6FB5E72BC645D50D210FF6983CA3DC1
:1057D000E3C40F972BA118B315FFB899B135CB9837
:1057E00065CC34D6F01638D4ECF104CB69964097EA
:1057F000E00216F67ADBDA5E7E392097F49136FA0B
:10580000E58DA7CF9DADB8DD74B7E9C59748F436EF
:10581000359D8BAFD034C99A642F6D26D1DB24F32C
:10582000F92A2A84C8F70983AAD008914FFA9F8FD2
:105830009AA58BD1C9A13CA51A538DAF1AE7CF27E2
:10584000362720E831BFC4C8A9E01D14570D1DA498
:1058500011FCD0CD0230B28DF5F593F93F6E4EB00C
:1058600059E72CD039492F947A88CFBBD27B31E9C4
:10587000C2F5FE7F81AED71D8836A42A763DA728C3
:105880008984744F12A31249BD9CF2499A49F70CBE
:105890005C983FB7966D62732FB4B509719CE4E0D4
:1058A000E4F5AAF3936FF99B849015727EDC779FE1
:1058B000482464859C2570DF3151ABD74BECDED694
:1058C000D6DADA08A3B696A40DE966ADA2C6F0C68C
:1058D000F05AA5546AB59EA9E88862A92737BD4247
:1058E00013141F41CA76AF9E04AF87AA421C42F927
:1058F00082E902309F5DECD37004615E57AFE85AD5
:105900005D3A64885A7BB65B2EDA2472228FCC8D86
:10591000D291013148CA756EC1A96150B7E542956F
:1059200034C11471A24EF80DA60F4CB9A6A750149D
:105930005202C85057012A9480BE4641A35B7804A6
:105940005A984E279737350547859C25F555C763E7
:10595000EFF452DF59EE18449556E7E46671C387B9
:105960002B95015AB20EBFACACC5109F2ABE7F5515
:1059700056CAE5B382EA472523674924DF539E5A76
:10598000989B3ED925F510E3F5165F04A01A76C35F
:1059900037434DCD8367510803D476A371F2569BEC
:1059A0003E8B54AFD946A351389E7584442B89D978
:1059B0000EC3389D7A96653B489D3A126452A98A77
:1059C0001F7C17E7E38774FEA03887BE0F646C471F
:1059D000FFF348095D004F049018AEA870437F1292
:1059E000C8480C0762C96824BDCBC7FF09072B75DF
:1059F000AD6172BF97A0EA4383A67AC8EF59D0DBA6
:105A000024F041B7E54147E91E7BA4BFADCF223961
:105A1000D3496F3F78A45F3DD82C61E55EDCB3CD00
:105A2000C912714BE5EEAD326B2A3237B5D13DE389
:105A3000047AA6B22F9F92E5D3477AC76B2AA06A51
:105A4000A9AA62847F6D3DDC90B39359D20B3FD5F8
:105A5000FFC5E4EC86158928AAD3FF5652E53AA083
:105A60009EABE0AC622E921BEC6F0BA8A326885A6B
:105A70001177070698550077ABE74EE89DD0CE0F1B
:105A8000F0782A3BBDC7230DC6F75345463641CAB9
:105A900082508A80CA1DD92060188E68A2D5023D26
:105AA00070AE07A87537B1DA9302BD536732EA1DAD
:105AB0007A074575D69F348560FE77DA38CE842E16
:105AC0002022C10B93F82218FF32C48E0C95D15FAF
:105AD0008830C4CAEAD5C1EF2360E20AF9DECE718C
:105AE0002A5545C5D1A3E430FE1CC462A3AC49B815
:105AF000D165B47B85785653A1E71E80C35BB71A86
:105B0000D81AF7B7CE0A6787570340864A151E7E14
:105B1000146D4427F8A37BCAFF9FF6DA3CBEA96A3E
:105B2000ED1F7DD6DA3BD9699B36692950A09030AC
:105B30004955B045102A962605041415545454B0FE
:105B40006592A9B465500A94EE94A9A8D4A0C75749
:105B50003D8A168FE7381C077046049242B57814C8
:105B60005B8F03886802ADB44790A40D25699BEC58
:105B7000759FB5938E78EFFB7E3EBFFBD7BDEF7A66
:105B8000B2D7DAD96B7AD6B39EEFF7DBB5DFCB0E9F
:105B90001FB658D6ACB14BE3258BC43F1DCEE2A750
:105BA000E4285123D165F375EB3A27BACC1EE3BA4A
:105BB0001D9C41CADDFC726CAA5D991F0AC9291798
:105BC000F16287B9B46CAAE3CA7ED946142B2B0DB7
:105BD00084E3DAB3D7A1D641347792AD10DA154217
:105BE000409354C37F35B05F655F4ED16A6F2A9B87
:105BF000C6EAD130B0EA9D45184684B8F06C453D00
:105C00008C0BE5BAB12DEC235CD2CD3107A0F50A9F
:105C1000EF6C61CE96E133DC2011C470746DF294A8
:105C2000CFEA93CE27B689A9C8FC508196453BE8B8
:105C30003DB322B3E2705678BE91FBE584F1E1FDFD
:105C4000F5EA378BF3D878941915B501F56C9DD624
:105C5000713A01B3156B0124906C861C8359C0B551
:105C6000E6442256EE76B919B73D3DFD0D372202C6
:105C70002AAC537FDEDF697E54FF7A37929BCE9346
:105C80009B9FE7C8E8DAA7F3B7AB661B654248F508
:105C900027DC434342307C5F3ADD4EFD51A1853421
:105CA000610C157AE5FA26D38811369B8211CFCC88
:105CB00064CCDDA5DFE869CF4E8763E6CC34F86CB1
:105CC0004B5B2D60EC92BA894895B3CA79C1CD8BF4
:105CD000D5CA585656CFF53FC49885C00029E6244A
:105CE00048A07BCC3DFBD7492E93032514C0609080
:105CF000E5A142670FF75F086EDCD81D5E03EAEC92
:105D000005D569F682FC5D3CCE78FF98D389E7A380
:105D10002EC75C3278479CCCBE22DE0BCBAD8E9278
:105D200062A7C5EA705A386B5C19EF704A12A66D0B
:105D3000F9D3FB084020C9BDDE66C3E4CB70A63BA7
:105D400023592DE2A3E139AE269555ADA51895430B
:105D5000305ED5AAAB01846E1054EDDDCAC7E8DC15
:105D6000A8C56A8FC20AD97E7F00571114C4C60322
:105D700018231314A279E18AFDF598DBE598A4199C
:105D800090C973DDA7B7C939E5F54947332A32D53C
:105D9000FE2C35BBDB2184DCC0B35BE9E044AD19EC
:105DA0000AD0E6E00A63712D93CB6C2FB017BC3E8E
:105DB000A73EE9ABB13EBDDB2483055241002DE98E
:105DC000A71DAFCB37F6DCBF33F3BD704CB76953BB
:105DD00024F75535F4C366D0417FDA8FE851C311FB
:105DE0008A392FA35087DC0A4A7990A32087E4845C
:105DF000BD723AADD6B43409AE4D09AF6A41DEE0AA
:105E00001479021FD74F061861DEBB6788D9A6DE5A
:105E1000C7110B41E6B4C966971A2C68C93A439C6E
:105E2000A0D51EE657ADEAF57CCC0C6DCB61B9422E
:105E30003EC4929377ECB020517C1A4E0FBCE31D08
:105E40005D3810690F366E9871AB64F3FC8E789EE6
:105E5000C4E7AF2F9DF151A9FC4A76881D428A49BB
:105E60008281A6899625F9C1439802F3593230837D
:105E700097DB6484C4CBAC16997F0FC218D8018518
:105E80008598D01A3DEECBF6F4A44C0979D9135B72
:105E9000CED616B3540FBB293490DDEC984C94DA6F
:105EA000E4FAA4FAA4D308DA032CC80A0AA82CC876
:105EB0005BD09157DB2E0DF3E479ED9C86659BC595
:105EC000797AC4E9B6A79801F531100885BEFC8936
:105ED000E3ECC77BB93E06A410FDE92A93DBE0DDC5
:105EE000DEE204594E326DDAA4B0478BC7DFC8D367
:105EF00053B699DC455BFCBAF5A599554E4B20A0ED
:105F000028996837B3E5B2BB7C3F6253E1E280F782
:105F10005FEE96DDD9FBF1C06CAE9C9D5D5151E00A
:105F20009D7F26D5C3335CB665EFA9C8F41ACE0CA5
:105F3000AABCC96CF6788CEC22266B6CACC2E4254A
:105F40006697279203B14DBFF54F62767B5D7D1258
:105F50002B66C7D919F6A92318B417E0DF48741DBA
:105F60005681F9D5D71DEBB81AA2EAB5F5C81F318D
:105F7000C88C4C6CEBF8E0EDD16F18C474D8E4B069
:105F80002C56C28C1B4B4ABAF6CA5B8BB1C93A5C21
:105F90009FB470B7C5C9E35175ACFB7C4B8FF53A24
:105FA000F3BEDD2EF4427644FB1949BE12B335EC44
:105FB00015DA3066613731BFC91DD90BE75AACA677
:105FC000CE9936F5710738017460C10D2AFABBEC21
:105FD000A2022F8087073BA25CCBB5CB2905D44317
:105FE00085F1CB8B9623D7C6319CC1D6317DCB763C
:105FF000DEC3317C34C30DDDCB15F89F8CAE4596E6
:10600000B122CF1C9C6C93DB59CA11EEC8EA44BF85
:1060100015BF1CCEEA1A051804E720880350E8488B
:1060200032C93833A8DF3921C8C063AC4FAA4D3E0E
:106030009A518CB8F6183807230BCBB2AAC75E3C2E
:10604000A713CD86C6C92AD8857F553A133AFD2DA8
:10605000670EB4720CA68599F0811C74C28A355FF4
:106060000097F9E8C3AD5B8F1CA9AD6D6CE4797E38
:10607000EAE40CD808135193E3B86EC2882BCE4BD8
:1060800010A6410C30434CF36376CF26440EE6A2B3
:106090001771BB07116543156D33B4DF4E9BD8AA4A
:1060A00061468B57C7A67022406F0C68BCE772141C
:1060B00037BF8E1BEB518E5296C0ACED980E41054A
:1060C000DB89E761EC2BCCEC20429E453F74677086
:1060D000006A2B8FA9F78F94665C53C298A060E288
:1060E0005B1563BA9905FEF06D9B594EF62CBF3ACD
:1060F0009B976A8C8A9DA19BC92C2DB2BE99E92CD5
:10610000C829617990D1438905F52CB6335B1C937E
:106110009DECDFB8737B0932591FF16EB463426A9C
:106120000ADBBF26B2FE376C1BCE9EC6CF27F9EF27
:1061300073948736E138AB2785CBCEEB019EBAFC52
:106140005E8EF2FE8A5AF7FD492EB83844D1F9E343
:1061500051E7D5E54EB3AFD939B496084B1E8393BA
:10616000494E140937AEAD927B44FFCB4DCD839998
:106170004EA616B3CB28C105331FEC659BD4E80AA5
:10618000F87E7B96C3C13E6063C2FE6F82C3AA6E77
:10619000EB23FEEBD96FF51B8A158545EED104FD87
:1061A000430FFF95BF46B289BDCEDCEE1DB60F4A48
:1061B000CB4D872D0AB38C7FE895724C4239E0F1C4
:1061C000BADCE38F5D7BBABEA111DCCD97381C959C
:1061D000F4502064F232C5F4BBCBCC6FAB5D878E3C
:1061E0008239D9FCA5D989397E9BBA4F061EFC5746
:1061F0004C12A4544CD16B9D12DC886D25889015EF
:1062000056097E716A7198C0643399B18687201BE4
:106210000DC9BEDDF6703B821A370971B00793D9FC
:106220008D0CD0335F298A1BCC17AD14B11F072208
:106230006689C5F9F27C87B59D8F6CE918541DE815
:106240006D22263DAA61557A7D925FE7D3B789B565
:10625000C9E539AC0BF2C99FE35FC7E7135242BEF1
:106260008C0A248D267E1D9FAF800297A11E6BBDD8
:106270005EA79B7E4B7805EE830F55F9E32EF8D78A
:106280006448C9423F12B54510FA0AEB34D2D1F442
:10629000DAA473499775416848DCB1364031D81D9E
:1062A00045C162EBE61169BF28D6DAEAF50E33176D
:1062B00075F469C0002EDC2753490FA479CD61D451
:1062C000233F11A7E43438CBAD0ED5186CB1093893
:1062D000B2974A19C9C998F55DCE56CBCF2BF25467
:1062E00053FF732E27E1DC0BE74E90A38CDF749CE9
:1062F00007195CB1FEC033087B1A51AF7E67EFB25D
:106300006F99877974C165881FBE82D14F99760BCA
:10631000EAC853EA538D356152D054A7F66AF7DEC6
:10632000BBF75EC7D436D6C2FE836BB4444C21D5CE
:10633000A829984F094A3C2B44F241549562FF1F0B
:10634000B87629E2BF567087B1BFB1F8696CCF70DB
:10635000A7783A6F532EA0778318BBC4DCFE064F94
:106360000E0B845A5D3F6D5CFDA5C565C976543B37
:106370001CD3ECEBB6CBB1ACB937A3D3A4FA11550F
:106380009AAA9BBF3A5A51E1C635ADAC2A70846DCA
:10639000E6C7559A0A03677483404EE887EA1ECC25
:1063A000C8B4FB4D0A3B236F61E75CE7DEBACF520E
:1063B000B1F76D72D67C277C003FC12F2733328B1B
:1063C000EF66083D3BCAF1C36C013BDA52BA661F67
:1063D000CBDC3D51D70247357F7D31505BEBAB6E57
:1063E000A96AABF223C528F292720CB84ED11EDA1C
:1063F000142CD217E5E58D5FC7427EE40727DBE961
:106400000B6EA9711C731CB1FC71C697C6D299683A
:106410008799D6F3AF040A5532500989A09F368C6C
:10642000BFD3E96EBF31ABDFE7EC929C0E7C8A13E1
:106430004CA65183CBC81D801C80D41517EA75610A
:10644000F0AF9C03808D52F95B40B320BEF07E0319
:106450008AD235B9257C2CE34DA611232449D2B626
:10646000AC67966A1613148257FDC477D7B20AC573
:10647000E26C6DE1E1F678EAEBCF9F47626CA9B27E
:1064800094C852C0E0950239E5C72C5F58CC60DB58
:10649000EFBEE0F536799B5A598BF26B9857AB2DCE
:1064A0001ED3C07A2D1BE5038F0A5C3D85AD789223
:1064B0002183B1931BC36B68B33057F059180F0B8E
:1064C000603E0EF1A2A539598E2A2CB6AE18AC86C4
:1064D00094487A5FA9577BC848729078611F8C46B0
:1064E0006B41C4738BA815C76F02DD2CD5C75DD473
:1064F0006A6DF057CCE23F1236D992DCF1EE967617
:106500007C73DC525E3B3AD60C75597FAE558238AF
:106510001DE786711D9AEF0FAF1FC5EB6878171442
:1065200055FD18C8D037A2639DF3671AB24D264BAC
:10653000D4B21DB045A892EA256F9ADBEC743FEB0C
:106540006610CC09400082C1D680DB0D2008A53C36
:10655000ED9980AA8C77854C57A8FA560419E86003
:10656000A68561F0B9A9FE512769E7819E7A0A3DA7
:106570004AD8178FB5F537B64B654495F50D7805B4
:10658000F9ED12002AC6ADE1D6CB788297ABC609E9
:106590005CE9C76C180F63DB35174B4EC7331881A6
:1065A000F71B426C7E8BF38FF3F9AA4C85D9E693E7
:1065B000E98E599E6EDE78D8896B5AA5F77B176DE8
:1065C00044E6A6782A21A4CE2E551380978B0B641F
:1065D0001FA28D584637AFDAB42FA97E27EA3FE7CE
:1065E0009D6FD8CB1E55A79DF5CEFCA9B25585450C
:1065F0003AEAAB8559D63BB0C2AE2AB43367DC5811
:10660000FCBD6AFFE6FFA83AE6F88C70E6BB5916B7
:106610009BAC7CAE9406D7CB671A9D278F4A2FD6AA
:106620003BAA329D69D5A80E4B4630E6966D2A00EE
:106630000C8C6533BD61A7DB1D0CB2F1FE540F83DA
:10664000BDB37C410C0112A15FE7D9555FCF9D908E
:10665000288FB40B03529FC4F34BF51D59AB4DF477
:1066600034B09FE45B582DFB8D7F9AED2A950F2F58
:1066700019C792597F1CC947FCFAD0C58B3E9F09A8
:1066800033BEB1B1AD8DB12387963E97536EF0B650
:106690006AE22F0EA8AB4F023018BADD1F33782DF7
:1066A0004E88E835AEE13FCD6E633BCFBCEDBBE03D
:1066B0007FDBF74DA84D3FE66B9F5E7E99E9DBF4EB
:1066C0004CEFD32BE164AF6F4FB848EE27B5E75FCF
:1066D000A6C58D90E2579B816C696296AE048226B6
:1066E000075CA739CD3FACA892AE94CADFA5361A95
:1066F0000252282C0470E810F3F8A7E17A830CB258
:10670000C4263B629BEEDBFF41B01E89388CD1DF93
:106710005A6D1CB036A773C992269FBB36B22ADECB
:10672000CF92E77DFADAE40CA7C569D8450611C512
:10673000CD261E89EC9A831714D95F8254F084E722
:10674000D8069D09483DF11D828388AFB0EE9BDCE1
:106750007D1B7AF6A7A3405BE0127287139CC64AA2
:10676000B16B9FC7D806EBD43705C7C09FEA3B8BF8
:10677000F42BEA18CB153DA560473C9623EEB917DC
:106780000AEDE9DD3F46944AE5A690BC0975DC6256
:1067900049B59C444CBBC1065CC7B94757ECD5A36F
:1067A00044085968EF0F306EC108025F66E746285B
:1067B000F7B0BBD805F491B068177031D4E0705EC3
:1067C0009A317DC3C873CC0AAB7DFBFA9D280C0EB1
:1067D00045421FD314DBD627446BA17A0EC774B58C
:1067E000AAAF1C809F78747E1A22CAC42381B1DEAE
:1067F000B50A678B48A966E5B888C27E1AF4D77BCC
:106800009F7AA8F0B07762A154E97BA3A29E6BBEE9
:10681000DF5FEDC25EC4A0A57AC63731D533D23F63
:106820002BBE29294397A19B591AAC0A7E7EF8C436
:1068300085E66FFC5FB1A3CC6BFE2AE7899CC79C01
:10684000E3CDAEA47AAB050C4C8FE018848E735F59
:106850006DCC5B7CD07260C2C157653F52DBA660D5
:10686000366A677335CEB3F951027D86FDB2D2D850
:10687000F6C8B4B64CB6DFC19817424C7EF2E28B34
:10688000212D671C7E561A7AE3D5D95950CB03289F
:106890003CD78FBC54515E241FC61D3883AE505860
:1068A000B1631D1B8F7DD7B1558D5E6F07DFA1953D
:1068B0001417D8FD3A8C29C6FA0F84AF13ADC6E37E
:1068C000ACE8C0858D33844579B239B1F6C13D95C8
:1068D0009F54E3A83F58EC518E3A8E3D1FDABF47D4
:1068E0002913F9E0DFFA8B6D467E975CAFC3F3D5D1
:1068F0003CBCEF0DD9665055568700A26C28074660
:10690000F76CB06D0F1CC1E416C2091E7406E49248
:106910002EEA2130C9A84F360F82D41A93DB0040EB
:10692000744E74B516C1C7F3CA8BB0F5FFB3300D02
:106930000AD1D33388009C0248ADD57269783E06EF
:106940004878B14E4616627034A3457BA3B69F5675
:10695000EEAAAD4EE60E090AF95AE8E1551733B929
:106960004D6E3E1FB90C1AE19CB67B6F0B1C4B722F
:1069700022F978D0EAE1377CEA3B333E0949308995
:1069800010EE1657C7F21C8337004A8FF5C388BB39
:10699000F18B8D5BF37729B0F98AFD5BA9A2BDACC1
:1069A0003D4B9D5082F68A39847BB67428B40BF235
:1069B000656EA988BCBD966AD3D15E362337A76AB7
:1069C0006EE3056337AC29C160576D242040BDAA32
:1069D00022A5EC04E3FCBECFD6B5DF8C8A3E900D39
:1069E000526E6C19E70FAAA8E4FA4A408B9CD35E5A
:1069F00076973B3B9C95B03FA7A7FEB647AA85E795
:106A0000ABC7DBEE8B169FB46A13EA0DCB69E3F9D3
:106A100062C77B47AA0E21EA3903146036653B1C26
:106A20002E956544EC3FC6DEE71CC0958773C078A1
:106A3000767BBB602438A660728599897264B72121
:106A4000B45B22B6177B5C43D87A8F2E188FBDAA11
:106A5000FE86D8763CB307DB202B7E5A6E6B6E6CBD
:106A6000163695C87F611B432D17D836C5A060A880
:106A70009827F8DC0549A9743A7FDC773CE0DD779C
:106A8000781FF336B97D5C7F99C52EBB9630C9312E
:106A9000D395AA37695C7D1D26074C7CA1C896D189
:106AA000CF82673023BF5BD911B60571EC04DB568A
:106AB000E527363734617FFC40EB8B5F2380DB3486
:106AC0006A664F63E7D8C34CC8365D85E878231300
:106AD000E6C24FF080F195FA807A8E0ACCF28751A7
:106AE00053AB31455952BD4AA6195001AF74B0A8F5
:106AF000453DBDABA42469B3D166C56B91DC42466C
:106B00004A6931634B583E7360F89238A4714379F7
:106B1000BC2C59F48320401AFBFA376CF3EDACDE41
:106B2000873D6798A418FE33A8C673B2FEA77A38CB
:106B3000873B9866B2A3C1C8FAFD706D37E7989D90
:106B4000BE517E8FEF42AD1E245F2AEB53CFB1EFD3
:106B50001A69C254E01CD0A68F5C2F1637E3AE77BB
:106B6000B27C58692BD39F580B5CE6700097B10834
:106B7000D307708089BF438BAE11F6B9C1EC9CE896
:106B8000DC288E8EC32492D84CEC33E16DA1B41A6C
:106B9000208FCC84249C9E0E3543CD4EE665BBD819
:106BA0003E568FF3AB90454D61140066A468047D9A
:106BB000D67591FD3DEC9CA7AD2DD4F87279875226
:106BC00031D442996B6F17F6E989B6404FFC69EBF7
:106BD000A5A34295544284A326BC278105F0101C2E
:106BE000C51991FC361A1565C50A0F1627F61A98AD
:106BF00007F1F10C18D13A4B5555733363325E9956
:106C0000498D4F3A4477F4196010FA4EF1ADA080E7
:106C1000B370E7DE76B5DF163180B973AB3AE38B3C
:106C2000F66A786DA956F04221A4C1F514F7747381
:106C3000FF3A4F6C02454948E8F4243393C01F5D86
:106C4000CE57016FEC4A826776E8C468B4019A5F58
:106C50002A30423C4AAA2990891BCAF2C891393984
:106C6000662C1B0BFD5EEED177508E317741297A71
:106C70001F0A959460F221CB85998C42B13AB37D7D
:106C8000078FDBB1CF92C6FB649BD11800135E6EF9
:106C900035EBA2D20BF1469638CC4CCA7BF62A2DA6
:106CA000187723FE9F672E4C108E5E2C54F959D90D
:106CB000A290B6D6DFCF8FBC1A500187B34DF859DA
:106CC000C3FA863867B1418EA98EA987A67C32D5D2
:106CD000FEC5DEA9C2AC33EABC367CD6F3F99E2AE7
:106CE000CEC3B4BEFF65DA3AC76BADB74EC3D4416D
:106CF0000E0985D8EB0812076B11D697DCF4C1C1D9
:106D0000F40997687019D1036A8AF24DE884A7DA0A
:106D1000C2F58C31EB19DB19CCDC8789590DE00AFF
:106D200035334DE8A42B7C86119655C462F17BCB9C
:106D30006D26C886323859AFE02DDA65BC6EB59C39
:106D4000CBF7FB83C921D4348FD195822AE08D52B1
:106D50006AD59551BCF8FAAB765CD4C55C6A7537D8
:106D60006FB5DAB2F64F6276FF00E637F82DD52A16
:106D70008699B91F64E842185EE807F7CAB014B3F1
:106D8000FE289A5A1C4EF61CA982D518F45F6E8E06
:106D900027A698A14B18068E53E43976915D60A71B
:106DA00015622A1F649A255F6ADBDC028DB56DB51A
:106DB000ACBED0E37570648A2C2E280585AA40E904
:106DC000FEAD037631E35973151C03D42919290745
:106DD0005592630B63407C096704EF5DAFE8419C0B
:106DE000A10784BB3E629162F0F26B46A23083B58C
:106DF0002BDFB7F7BB4D395B8654086EA9504A228A
:106E0000771847604FB26A3624362F0B083664B6BF
:106E10003398ACC184DC75202D65452A4C04B4122E
:106E2000B683ED52A5A68F75508ED6FCF578AB379C
:106E3000B2AEC7D18237E03886FC7171D6DE1C3B1A
:106E40000AD9149473629CD6680A180206AE5422BA
:106E5000530CFBA76D42EED805B3208783C80939D0
:106E60009C5330E3CCB24DDE637196BBA70BD305C8
:106E70002274962074B72B04B9A7BE8505016D5303
:106E800068639BDFDFD9434144E7AB8F561FD54A88
:106E9000034D21E578F0EBE0D7810C648E0071ABF7
:106EA000DA2B08120DB903CEF9255C356D6A869987
:106EB0001047C536F4D2E632F3EDBA0A7212ACBF0F
:106EC000C29D00B3BD0EAF23BF0AE2640021589EED
:106ED00023BB58B69A1D61796C807CB80D1DD141D9
:106EE0009213307E3C771DACA3A023217C08444143
:106EF0000C6FDBBF5F66CD6A7BD3A4CCA9A6A906C5
:106F00006BEC14DDD492D98F4D094570D9C6588BDE
:106F1000630593DDAFEC79FF5286139C239DB61673
:106F20009076652BF271353F5D08802F58217C00EB
:106F3000593AB79633DCE04A7A0E10FE3CF15BD446
:106F40002CBD91F543324DC3DCC98121F0286CA2E0
:106F500081F6FD5D0E0FF2842114AB1F9084677BD8
:106F6000924A341D5E84E77D2AF5B3465541F835D3
:106F70008F2CFC74C1A1A9CBFA3660806E83E9DF47
:106F8000B1FA5FF18677B567A092650278934B8F6F
:106F90006E8E313639593DFAA36A86D5B3268FCF26
:106FA00066704ED40394F6D565C3B85B8A04CC49A9
:106FB0005E0A313BF7F05BD09E53D91997238A14B0
:106FC00030785B4CE1B0B59B80694F4CE07C36DF9C
:106FD0006D2AB0477675633A44FA6D783CD88C27B1
:106FE000C43F922A90782C19D923D2AF1FAB17C077
:106FF000EE36EC9B39EC67AFE036B485C9D184F846
:1070000033040D5E03DE8916CE50A7582156C00505
:10701000F02327B4E0F339FB4A39FF9D47870BA8DB
:1070200029E2448E3A8A74CEA32AF3BB2F5732AAA0
:1070300032BFA42154C6044CC4D77195B961588697
:10704000FC9C1D5B14875C1249B09C84340380E473
:10705000A66E90F9F9FF28F75633BF2920073100B3
:10706000A938A610114AB6005944BF0F5894F62B00
:107070002A72E4A5FE02FB8C7B12CD636DCB6DA959
:10708000B64CF4C3E3C5D3BBF106780E57589C1237
:1070900016834194B64965863243AC218017EE854C
:1070A00070CD2D881B5AE57621262CAC799DC5E242
:1070B00035B893DD194ED9596C3BEC74580D8810D6
:1070C0008E110BC844263CFEE3F93F9BC566527BFC
:1070D000C20B21BA6D8872F424D8458BFECC703374
:1070E0002E5700DF60240D3082752FAE3448E3B098
:1070F000017C9C3842D7A39FA9D869B7784ABAF7D0
:107100002A21D1DAEFE4533F992B871C3107A7A13D
:1071100054B136CFBA3C3FDB18925D0B4393985580
:10712000281CF3F598ADC2D742A1C96AB1396C9851
:10713000D35FA30531BFDD48ABD67A38D76EE436CE
:10714000A22F4135D3A98F4E89524617376A03348F
:10715000802768A12DAAE02B7D5BA41660DA166D4E
:107160000BDE3D1BCAE0259C8AB283E7DC0131D6E9
:10717000E7796E5898AC1AEE62819378B27DF84C3C
:1071800087A5100BD0F37CFA814853360A49D6C440
:107190005B7B3F9E3CA9ED1CCEE276EED0D9D0D9E8
:1071A00043679D168568681CB98E1860109CEE1E9A
:1071B0005DC20483171909AF97DF7723A997BAF641
:1071C0002B10505B27944AB2DC1E5095D53A728042
:1071D000411374F3AA07099B53899E4679BDFBDED0
:1071E000F3F9CEFCF67D758DC1A7F7EB0D7177C471
:1071F000EAF5FDF5693150052E9073647D30275412
:107200008CB04260BB30354D82970E8412440D83A2
:107210001009E8DD0502F86321891A1965D3149372
:107220002F68C0ABA621015E859F361746CF1EFA98
:10723000BD70096AB4DEB9AF5FF573E9FAB7665F8E
:10724000FBFD8C4BA941538027A2D61BF794D38416
:1072500000D8A0353AF10A0DDEBCF7DCA69AD46D51
:107260001B3C4621097169421F98C10DABA0BCFEB1
:107270006446ADBBDC8CFF4DEE2757E5945B6C821A
:1072800053E384B03A39E911D966715A9C3C7F794D
:107290003BD179C1F095E10729201522FDB92A2EAD
:1072A000BA3966F0CAA5106590890B8322285A2640
:1072B00086924337B5ACF215B17022A2B6A024185D
:1072C000B02EB6159714EC2CD809419BB2C45621A8
:1072D0007388A9EA2AF0371BAE3008FA118081C4FE
:1072E000240C24032B386614F509E293E96C81DD44
:1072F000C9EBD79796DAED51514F3D156760500BAA
:10730000DB91100AE032E4A12FE61130C2DCD73560
:107310001DCF5688B12C7231541F83039E64A5B8CB
:10732000C51686BAF392391BF3AF1FCA578B80F983
:10733000D7CA1ACA1BE4CBA1FAC0E596FA00C4C3A7
:107340009D38CF0E1AD0BC1D13102EB27743ABD888
:107350002A1CD5CA947B14CDD86F26543E75DBE821
:107360003B6E9A32C89A9C9594C5B21C598E050EF4
:107370002B5AD661B4F42C28949C2F82B02F7AFF1C
:10738000F44F759F2A55558CCD61568FB7DE3BF56E
:10739000BD2FDE1B4B72883BEA3228989F5281B585
:1073A00051A9504A2E47217AF0F4F682B8F78C0D95
:1073B000C8AAD7DA1EDE0C539E363F0BCFF6F598DF
:1073C000DA5C99E5329B287F2AB7C82DB699704CB4
:1073D000EB9EEC861A38825A7A4E95FA7E2C596DBD
:1073E0004DAC9FC68B5FFF806C4897BCD8AE64AD38
:1073F0007EF66FCFDB3C53031BD8294FD2A4A449A0
:10740000C993061EED37591A21D4D37387161C3A37
:1074100072E86CC6D983674FE624D5F5AB4B353F90
:10742000B2DAEFF561F1A205DA5C180A03124DD861
:1074300044A8366CD5BAA53D9BDD6EAF5751909EE2
:1074400011EA016913350197068E8CE2E2C2C2C1CE
:10745000834D2683218C881228855F31B1BD6194CC
:1074600021580894DADEDDF352C95AA9C004617EBE
:1074700044878B11656ED867AF31B92D3364814D68
:1074800046BA01566070C739636D62C401982B9F7C
:10749000C4635AF03861E8DA86C2509CC68B9557AF
:1074A000BB2BE26ABE3879BCE60F6FC05DE04EF1DF
:1074B000646659ACC8C7D444391B1B4B0DEED89C2D
:1074C0005873898ECC1566477F4BBE37795993AB7D
:1074D0008915FB154751EAF7D7FE688D87F6A39407
:1074E00080D30617E3DD26AF81DF0E7F98157E027D
:1074F00016E745870740141A5C85FF0D5E9B5C37D5
:10750000E07214DE23241CE9F305FDC2E814A6F59D
:10751000927A49543BD179A3F3C64A8B73FF948086
:1075200018105BC44279BDBC49D619D47CC253D86B
:10753000241BB551AFC4F38DEF6A8E909191CD525B
:1075400089159C2A126B208249AAF652344D289341
:107550006586A94705196D272856C2FEC25E625787
:10756000619C8674A5265C1CE0C6D6F5ADAB5AEBD3
:107570005A356DD121DA4C9B25089B162D0E8DA016
:107580000A13A6F387BDB03A6CD0BD243BCBD1AA79
:10759000DDDFB83D67FE7DFCFB2F9115AC16ABC956
:1075A0006C320F42FC678219F9A7441182421049DC
:1075B00002CD093D5690CDF21ED92B1720E1833C18
:1075C00018772B3961CBC62818F078CCF62B2233EC
:1075D0001964EB05ABC7F6360444770EAB0DBACB96
:1075E000D794AF2FDF68EACB4C6D70886E4265D9B7
:1075F000A4FA6781E193D9964D946DE65A83227F70
:107600002AB479123D32E4C88185CF16EE9FF9C6BF
:10761000D43DD64368216B90A31411EAC8D20793D6
:10762000193D9C8C0967FBC3E60179A8176AB30E64
:10763000DA169E75FD2A177089CB82460C07D7D8BB
:107640001097EAC324AE3120592ACA918579026085
:10765000B60D86F5F1BAAC3448C18CDB82CAA330D2
:10766000C57F911D66871C725139C1BB321FF782DD
:107670005607E9E85F355E11C7A581B5F85995232E
:10768000CD05068D1113DD63AC0603F5923D5EC496
:10769000657D60362BACF6BAECA16C859EEB33555C
:1076A0009BA70F1A98A13E0943D1AFEE53EB534B62
:1076B00005A4D92437CB61EE401B1508E9D78FE329
:1076C00048920C061182E8E639F5E2B9A6652A86E9
:1076D000302E301A4E3C0F812BCBB9AAF62C035515
:1076E000BFD2BBF4EDB1D8BA49A6B3E76426A27500
:1076F00019A143830839601D77D1A41ED7C0FAB2FF
:10770000312EC115DF2DFDCC307BB62C5B2C61E911
:107710006C412FDF52D3BBB33821D7E8B0FDE2FC78
:10772000FD6C9DDBF39FCBDE303B586020C2B20F77
:1077300002939FF9FAEB6B059FB08A3C6F73BBF91C
:10774000998F630C7814640E5D03638AE2F331E66B
:10775000C71D64D9ABC2431F59DD067EBFC3D145E7
:10776000BD992E4C1B1D25C84E63DCBE66C7DA1AB8
:10777000DAB6FA9DFEF6EF221A3F2A61DC04450CC8
:107780006A95AC0EE9E70A178EB4A2A25A6F58297F
:10779000B7B0B39CC1D4E2ED40411F361767995989
:1077A00047947B146DA31E2DB9D1E445DA7123F9FA
:1077B00041D80C689CC104E43DADE2F796E714C1E2
:1077C0002E7821B2BBA1E33A2E7EFBC3DEB644ABDA
:1077D000C99969B3D82C157226AC46853C03155C53
:1077E000CED18B69FB271FE4D961939DB2D3E2B65A
:1077F000B4EF1B117CC427378ED17D724DF6CC9926
:1078000036A69A0B313A738F611F0897843AF14B71
:10781000684829119F1FBA7F8FC3143005325D2637
:1078200026BF9C5F3EADDC6AAAD1ECD3203F85DC4D
:10783000F65B35E99FC3B7AD9AD69BF97FAFA1B58B
:10784000992114CC56B01A67D135F441C4D9FCC77C
:10785000CE724CEECDDAB9EAEFF7C735FE7A46FEC6
:1078600011500A57858A82411E46962DDB18B9BCF5
:1078700079A7600BD31B463188B86C841674555BAE
:10788000F6C7FC6241A1A1389FB6CD72A4459B907A
:107890005342D5203830500CFC2FBC187D9EE7ABEE
:1078A000D5E1CEC675FD8B48E2197041706B104E64
:1078B0004015DC061F0A4E3343AE2A4C39915EF563
:1078C000C1CC199F589CB0C709F1547B0C2C828500
:1078D0005872E46C3FA6B3DEE27533671063AA8387
:1078E0007DBB0A2CB285C57D9375C6EDBDAC541722
:1078F000D8736C56708E760EDA6330F21CD041630A
:10790000A3A284B3CB64E2EEC4413B0ADD9066D10E
:10791000190699924D275D3BEC0D9E1A17271A37D1
:107920009A190AC0C8095ABDC62E188BE85E0463AE
:10793000FAC12EE886CF9EF9F3175681349186DA84
:10794000A165C29FF4B70542C1CB4A2CE35C262057
:107950003F481D991BC9546F5191526CB13C575E01
:107960005DEDF13066802D5C082107D2D03F008BA1
:107970005AB2B3DF79E7B7DFCE9E55824E356BF64C
:10798000C05DD01F312A20A15C564FAEB06259961F
:10799000B3B33B57E619B6076AFCD33D7B3C469729
:1079A000D5657358F17675B8AA5165066B1823E84A
:1079B00039EA0E7B98CD47FF2C57F8BF1D7B335813
:1079C0000A9ED119C6508F6240B996BC5298ABD16D
:1079D0004C2A723A4FA84011265008933C8400313B
:1079E000393B0329AB3C53217F2E1F936D68CFCBCE
:1079F000FB0D01AE4A1D86240C5693BBDC5BBE0F0B
:107A0000CDEBF2BA6A5C6E8C4CD8CCAA752E676648
:107A100039B2D1D4FEDF2683CB667223508536314E
:107A20002806014FC00DEF3A20A0E198726ED6E60D
:107A30006279826547197244C8C846B2E88F6CC43F
:107A4000A959CD31F50B78E0BB8F261F526E2CBEA5
:107A50003A6F6BB53853977DAD7CF05698649BB206
:107A60006B6ADA8C7DB7ECB9D336CBC24AE49CF2B0
:107A7000C5E5763909A3D7C27162559DCFC124737C
:107A80006A618B2261FC64D6868FA2F8FD5DEF9E51
:107A900060EE2AC59999AF97963BBDDEFAFA295355
:107AA000C68E2D41E628048BD50049F0197C05D7F8
:107AB000A7FD714692CA4DB28C68B6F4ED5B0D839A
:107AC0005077DCEADD39A101F8DD0799AB835F7BF4
:107AD000DE4F2B7B9D5545FACE9CF17ABBF60DC24D
:107AE0009B2A290933282F0E87D95CDCA5DF8AE081
:107AF0000D5FD83EE6C55D8A64ADD4D57D9B102070
:107B0000A0F2733AF6A7B3F53DF74727F518151914
:107B10001F2E41F5F5972F77ED4E822810D92B882F
:107B20008A7DCCE76B6C6C6AF2717D5371A7471448
:107B3000C7720CAAFB0BEC09C4592D0B5D71BE5525
:107B40008DC7023E16D59156712075EB6F0DECDE98
:107B50009D99D9D818EE3522FE166284E33AFA933D
:107B6000936FBC31D3D288E8D5318A27A9852FBA43
:107B7000E9233F1FD7006E7358EB15FBCB6EC5EDA5
:107B800038F36EADBED6E8D3F962FD5C3306413200
:107B90001A3F860E028642C3175F4EAFB6562DF5CA
:107BA000E8ED77CCE4399D86968E282C807D305880
:107BB00001559F7258017A7725BEF6498A00BE8A20
:107BC0003159AF0B1EA14A6C0B4C0B82BE4D9FF975
:107BD000FC6B3517F6573ADB72307AC024BF915DE3
:107BE000C7EE64C636788973B1CE8BB9FB2DBC2B3A
:107BF000FE8E6D0810BBE32C0FB972589CCBE8A128
:107C0000F81F2CCE287309949BBFED250F94C7AFA6
:107C10002B674FB24CF92696C46C39B69C1DA81937
:107C200060E52C0B4EAEECEDE520C642DFC3BFC3D2
:107C30004A28D4DEEFC77D08D06EFD46A3D3E9F114
:107C4000D4D7F3FE52BC410F62DE8837DF5E7CBEC4
:107C50006030A1295339A7D8D90B78123D725AAC9C
:107C600099743008214E27A556ABD3C9573030053B
:107C7000E78750702C5DF6188B4C6236734FF11706
:107C8000490417B47B6A8DDCA7DB8D19C83AF9C7A4
:107C9000A47E9D44252C7DFAF4EBB765CBD1A34D92
:107CA0004D21445700FE03E790B73230031544C519
:107CB000C489D9D9265320C05586AF770479D58D8C
:107CC00079C67D0CE32FC8022CDD9261F9BB435DC0
:107CD0005440939C92935AE13B978F35368E618343
:107CE000D17AF19BC6B4C0ECFB3A62FACEE8CAB2D4
:107CF0000BCFD7792A9B5ABF8873BCB87A2B32C86E
:107D00009FE11BD8FDEC71A5B074DFCC3AD31D8E7A
:107D100004B59F74EBF7B26493D74BCF5EE5E9E50A
:107D2000125C6A2410F703232A6040B935B1C3B846
:107D3000C3581CE9BC62FD2E84FDA7FA67F06B8373
:107D4000D1974059F2D7E212851496EAD4C3777AD4
:107D5000D0C60E3A8AC6BC393465E8FA85A17AF1F4
:107D60001C8FDFD7701A6D3766413FF4AF44E9BD11
:107D70002171A3B871D88357DDBFB7267CF276C3D3
:107D8000F25CBE3DDF6E33F435F56D004BFFDF1A5C
:107D90004E14D80A6C5CC3A101EFD51DCFE2D0AB65
:107DA00023C83D1343161EBF3C58855E4E84EDD458
:107DB000865BA565B23CF6B27A4385F21E079EA6A5
:107DC000029E82F9DC499B648DC13462376156DFC3
:107DD000E9B1A206DAC289E3847627D4F85557DBE5
:107DE000C23D114BEB11FFE3C7F957ADDA27E27340
:107DF0007DB7EEB988ED9860AC12ABBC8DEAA26796
:107E0000181A03889DFD1AD48FF9E5127A6E408600
:107E10001118D854FD70B693500459FEDDBB799EFD
:107E2000B923F1D7218B85CB33E519E5735DC7AA5B
:107E3000A3FA941CBE1FB924AC8C69181FABDA2FAF
:107E4000B886B2A1EC75B94E46ED73D898B98B6F70
:107E50007C84C5D96EE38F49019DBFE7FDBA4DAA69
:107E6000B8DA2CCE471FDBBA71E0D99EFD724768A5
:107E7000B888176DE9D9BF401EE2A2A1C79F00567E
:107E800095CE47D9081C03EF5AD29E49A8D3ECC619
:107E9000AAA47A608765A745E1D17122052F8432B3
:107EA0008C5426A03E706DA950A4C080BA8084B3C3
:107EB000DA600A423BAD83A4D57BB3629477C98371
:107EC0007F4CFB2A723033A6B74E278A20AACEC534
:107ED0000457BE5C609F7468F0BF23FAC26F4055C0
:107EE0001953EE9064C13C74D8D091E2D8E1E9DA3C
:107EF0008CE156DDF487474E9B322D7D877547C652
:107F0000B737703E1370B806B488781D2A16B76864
:107F100088C1E9B1A82306DC281E12A01724426FED
:107F2000E8037DD5ACEE0F03500106A21298D09560
:107F3000C1300486C230181E991D0557C188C85B20
:107F40000A5C0DD7C0B5301246C175908A9606A35B
:107F5000E17A1883AC76038C83F1A8145170234C1A
:107F6000809B908FC2732662602C78C82C980493F3
:107F7000311CA9DDEC66980AD3603ADC02B7C20C6A
:107F8000B82D32E776B8036676EC1F05B3E04EB83D
:107F90000BEE86D93D66A7C23D38BFD3DAC7DF0BEB
:107FA000F7C19CC8FBFDF0003C0873B19D070F753D
:107FB0009B9B8DD937BFDBFC051D2B2C8445B0184E
:107FC000DB8761092CC5B9F7C33258DE63EF159022
:107FD0000B2BFF64FF3CC847B55C05ABD5796B60E4
:107FE0002D3C028F5EE1792AAC834258DF63FE06A6
:107FF000D81859A5489D7D3F6C8262ACAF9C9D8A84
:108000003A628312D8DC65FE16D80ADB607B97C81B
:10801000712B851DF0183CDE63F613B0539D53D6CB
:108020006DFF27C1DE637614EC42127A1AFE82736A
:108030009E81FF8267E139781EFE0A2FC08BC88AB5
:108040002F75F3FF652847B57905FE06AFC2DFE15E
:108050001FF01ABC0E6FC09BF04F780BDE8E9CE7B2
:108060001D7817F6C23E780FDE870FE043F8083E12
:10807000C6999FC07EAC3F850311FB0C0E627D0844
:108080000EA37A3A91068FC0D1C8FC4AF81C21573A
:1080900085C0FC12FE055F213F1F876FA01A6AE0B2
:1080A0005BF8377C07DFC30FF0239C8093F0139CB1
:1080B000829F91BB7F815F9128DD7006CE422DD4D7
:1080C000C16FA897F5D080BAF93B9C870BF0075C8D
:1080D000040F78A1119AC00797A0192E831F75B5B8
:1080E000055A11C0415470851300218412818844BF
:1080F00043B444223A1245A2490CD1935812470C7A
:10810000C448E24902E94512496FD287F42549A4DF
:108110001FE94F06906432900C2226622683C91014
:1081200032940C23C3C9556404492157936BC8B5D5
:1081300064241945AE23A9240D6D34B99E8C2163A6
:10814000C90D641C194FD2C98D6402B98964908924
:108150002493588895649149643299426E2653C994
:1081600034329DDC426E2533C86DEA5C6EB7933BBA
:10817000C84C328BDC49EE227793D9E41E722FB9BA
:108180008FCC21F79307C883642E99471E22D924E8
:1081900087CC270BC842B2882C260F932564295917
:1081A000469693152497AC2479249F1490556435F2
:1081B0005943D69247C8A3641D2924EBC906B2913E
:1081C00014914DA498C8C4464AC866B2856C25DB94
:1081D000C876524A7690C7C8E3E409B293949127CF
:1081E000899DEC224F91A7C95FC833E4BFC8B3E4AF
:1081F00039F23CF92B7981BC48769397C8CBA49C83
:10820000EC21AF90BF9157BBD8DFC93FC86BE47575
:10821000F2067993FC93BC45DE26EF9077C95EB2F7
:108220008FBC47DE271F900FC947E463F209D94F7F
:108230003E2507C867E42039D46DFE61E2204E5226
:10824000418E90A3A4927C4EBE2055E418F992FC76
:108250008B7C45BE26C7C937A49AD4906FC9BFC9C5
:1082600077E47BF203F9919CE836FF24F9899C229C
:108270003F93D3E417F22B7111373943CE925A5200
:10828000477E23E7483D6920FF21BF93F3E402F9CD
:10829000835C241EE2258DA42932D7472E91667275
:1082A00099F84980B49056D24682244414C2908CE6
:1082B00009A554A022D5502D95E8AB4447A36834B6
:1082C0008DA17A1A4BE3289F6DA0461A4F13682F91
:1082D0009A487BD33EB42F4DA2FD687F3A8026D3C7
:1082E0008174103551331DAC8E1C82F5503A8C0EC2
:1082F000A757D11134855EAD7EBD865E8BED483AC1
:108300008A5E4753691A1D4DAFA763E8587A031D6B
:1083100047C7D3747A239D406FA2197422CDA41647
:108320001AF6D84AB3E824DAF5FC93E9147A339DB7
:108330004AA7D1E9F4167A2B9D416FA3B7D33BE846
:108340004C3A8BDE49EFA277D3D9F41E7A2FBDAF1A
:10835000DB2C6E73E8FDF401FA209D4BE7D18768B2
:1083600036CDA1F3E902BA902EBA62E462FA305D2A
:1083700072C5D7A57499FA6D395D4173E94A9A4778
:10838000F369C115A3B8ADFAD3AFDDADA79EFFFF6A
:10839000AD6CE80782D9EE6D6C609F7BD97176A8D1
:1083A00001E6650F1356CE5FBBD6BAE8E1FCD50BEC
:1083B000178F494B4BBB6ED1E2BDC7BC356D76798B
:1083C000B75D7EC90E2FDBA1DC6ED86337BC628738
:1083D000F7EDF201BBFC99BD708B3D79ABC5D1CBFC
:1083E000324F6F89D65B7AF5AA0BD585BC414B48D5
:1083F000B0DC91587729C5BBD45B73015B43F23C79
:10840000D31AA1A5D75FF0E1F6423CAF5F33B4F4D5
:108410009A691C91189718EC352E7152A2C564E028
:108420006BF58AED582E75AFE57842EA3FCBE0ABAD
:108430004B5F357F75F92B7F436E99FB5453831E39
:108440009F647C46E29381CF6DA79ACA58C35CAC07
:10845000A12116FF8FC267223EB7E3330F9F95F825
:108460006C3AD58447CE7632FC091E92FF56CE3246
:108470007B4E4D7F3BE49CDFC5A7D62965B44EF10A
:10848000069556CB7DA2E5EAB8FC037F3FB5DC0E2E
:10849000859691DA03AFE19B517D7B03DFCCEADB6C
:1084A0003FF12D8DBFD57DEAD5D96F6BAAF4D9E107
:1084B000D3FC030B4E3D3BE1233BAC6B9FBD57B45C
:1084C0007C17DBBE40F84F648DF09FC832EA1FCBAB
:1084D0005F622DAFC5654FE93561011E849D581E51
:1084E0006CFFE597817F79656E10AB95BC2AE0D56E
:1084F000AAA895B95105B951AB72EB726B044B1F29
:108500002D0E5AB094792B4E2C4F312DFAA086BEE9
:10851000F561D0BF00E77754131684AD8CFA97A7A6
:10852000182A73CB046CBD62EED25FBD82A5B7463C
:10853000DDC5DB7F7799AE7A43E9A95C1C955B26A4
:108540009E588EA3722BD79769F08DF897E3066338
:10855000F87C6CAFE36B04C34B942FFDCD6B0CAF79
:10856000BB54F0C62CD578A5D4388B2B2635CA72CF
:10857000972EFB712DFEF8ECB2F813CB432BCB44B6
:108580007C9B5EBDA1E4947CD12F57E656EE0C6235
:10859000B3B2B2ECFCCABADC0DB91BFE869B036E0B
:1085A000BA2188D5C6326DDD063C40DD4674A05741
:1085B000DD4EFE5A86AF71E88358A32D8B6D80C8BF
:1085C0003F2BFE33F07F75853A3AAF4CEB5F7E125E
:1085D000AF253831DC4E0C9F4E7D3DD96487F67A4D
:1085E00062595FFF72715DE53A74B1DBC489C17095
:1085F0009B1F39EE59358F6FD2FEAE2D952E497FD8
:10860000D34D8F12A4286960F483DA07B53EB57E96
:10861000503B179FFC7058E7CE9D3BCFB44CFBD826
:108620001576318ED79FC785DBF6D547A8ABFF55AA
:10863000DBE70A9B10D347FB54CC7B318E9883DA5F
:108640009131D978CFEAFAA1721CFFA5F6CB18595F
:10865000BA20FD47FB758C2B6663DC7FB4FFD17EAF
:1086600012F77B4C6BCC27719FA8FFF2BB049B9F3A
:108670008C077579E5C66C8364795F97ED8BB614CA
:1086800046615D975306C78597BFCA2D24B9DE980A
:10869000429AEB351442AE37413D4B798A21B5B74A
:1086A000BAA92135565D239C89A95727630EC5FBBE
:1086B00097E76CCD0DE1053EC66FF1F1F38FD73D25
:1086C000B6E131BCC3C730E08FF1A18F55AEE48174
:1086D000AD6C6ACDF51DC47AA52FBF10726A16D98C
:1086E0000D9B1A5695C1A982B25E1D6BF26D866D07
:1086F000C28F7907725FC87BA0C0480F146036F440
:10870000AACBE5F7BEF2C4F28E14C9C3E5F3F8AC08
:108710003C9CA5EDE8EFB1939D6D5237F3F3CDE6A8
:1087200094097FBAD986DC070AD2FE0F37CAE7E977
:108730007D456AAB895D56D6BB336DBBEC1EC373FA
:10874000F5C0CE0772BD51695AFC4738D07BF38F14
:108750002AE4D1396F74593407A09AE2BD3B661EF2
:10876000C8F5FE58168D1B6198CA62FCCB6BCCEA2B
:10877000B2615638508071CB355EDBB1D281DCD42A
:1087800041DDFA37607F5A4C97FE6EE73ED0158187
:10879000051C81ABF0D405BC7755C7A90BD453AFEA
:1087A000F285BDBC06D340CF1D4B37E47AB5E9DE78
:1087B0009551B96A6C2B73D3BDFC8341FDA0E7AB27
:1087C00097C5F27133D0D24D2B396A5384CA3CEF2E
:1087D000D09895DC9612AFC6CEF25207F051C6285B
:1087E0007CB5BDB9322F55DF8A951458D9EC4EAC03
:1087F000CCE31BA518CEE755E34D4A3356AD2850C0
:108800005AD5C385D39A4F4CD31ED8F04241AA788B
:1088100060C38682531BB0B4A7E2069E8A1B23273F
:10882000D8A09E60A38FAF37776E4A061E2156CD23
:10883000E4F6D0F34319FFDB4319D543197A1CAA98
:10884000326F46C4D2853CEF55E1D3C5AC2C2479B8
:10885000FF83031A3B0FA88D1C50C3B7E5BBA46967
:10886000731E2BC84D156D6F16E41A053BE4165A9E
:1088700073D304BB35174F051DD998EBE38B444EDA
:1088800065E87A2A84B2B70F7EC405B7E62EB5A68E
:10889000D106EB89E595EB2D1FC48659CB10EEFB75
:1088A0007BAE91F2ECE8EC596AD8A7A9B4EFAE7CA4
:1088B0004AFD37AF01CAC0BE2BCF0EF9C7C0ABD936
:1088C000903730D5AF66CCF2E4E479CD402B0B3E47
:1088D000B7D166422B577D5E429B29FD7C336D16D6
:1088E000E8E75B10631B724F15D4F1EE3ADE876E3A
:1088F0008B954D767338912A8BE635AF1E882B34D5
:108900000D0C35FB066E58746AC1BB6AC9BE57E0D0
:10891000FD5C83D0A5EFC22ED50876F262FE5B9F88
:10892000747A1E17D6A2C859530C5CBDF2EB726A5A
:1089300062DA47642BD1DDFFF78FC9B7434E835608
:108940003D9A1D5EB0431132C66F05032B9FB407DD
:1089500073ED64E5816DA74AD1E505A7169D7AFE02
:10896000B71EBE3540654943EFCACD0D85957FC31F
:10897000F6553BBC68874FF26B891D1AEB42754A6E
:108980001DB31BDEB3EFD9D7BAAFD56E6C03B00BF6
:108990008D0D30EF586E8DF6243FF24455648C1ED9
:1089A000FBBC263BF5D973F937BBBEA975B7CF9E83
:1089B000DCD4FA92CF3E91EB93BD0847D90D4DF62A
:1089C000349FDDA47E48556B8B5ACF54EB6CB5CEEB
:1089D000571790F9C8BAC2517628B4B4E9ED46B534
:1089E00036AB751AAFDFCD6FD08885F3D08338559D
:1089F0000147F9266E4AF1CE6BB0E61FC73B0DFA70
:108A0000B79DCED9BAED0791FAB76DDDFE83860624
:108A100079897CD4863F4AEAC789588E15D57C93DC
:108A20009FD3BC3E7947E18F226D2E4CDE91FCA393
:108A300086F29EC8476DE4A3A47EE4D3DE29AA791A
:108A400031BF61707272A8C1F623D01F296D68FB17
:108A500091D01F059A5F060D734F35D96F6BAA5BD6
:108A600037EC3D94DD06492CC4DC28F79569782E57
:108A700046FED7AD4F912BF1804BC19BB6D4EC1D78
:108A800079FEC0A9A683E73F3BD514E9E7E9DB31CE
:108A9000220E4744778EE0D541FE37BF8EAFE4AB60
:108AA0007C74D9A3EBBDC969B16F3D5A5778FE51AB
:108AB000EC3CD5947AE1892E7F5CE8951D76D94906
:108AC000A1656A9C9DAAB5A8D6BAC2ECA971FE059B
:108AD000B8C935A8DE5707F19579CDBC11BCFD7931
:108AE0006EE1EB699E8D4B7FF546D7ED42D776A5BB
:108AF000AA818BE4668DE6C0B3A79ECFAF7B21C56C
:108B0000DC9E8FBAB4CA17F807C3EECA17BC42522C
:108B10009AFAC7E88D3EF0FCA905F8E6C1DEF04000
:108B20002FD95D96C0B33C415D69E089E5965763F6
:108B3000CBFAFA974F67958F5DFDD83A3B709084DA
:108B400065237F77E7C0044B6F0D1F267E5AF969B6
:108B5000975EFB48357F32D4FA765EE7631EF23FBC
:108B6000C96ADDB55BCDD286C6CA4B98FCCD959758
:108B70002BFDF6C22DF6E4ADF6C26DF6E4ED6550C0
:108B800078E992775C61D3A59ACB75CD27B64CD89E
:108B9000527759ADFDBCB6375D2AF45DAA69FB93E7
:108BA0001EDFA5D4CF71C14B9125E1233B7C6C27FF
:108BB0009EFC8640978DE636D999EFC016CE338558
:108BC0002DFF2F6C83BAB725897A2C4623D2CBF19F
:108BD0001DC85E5B524CFCDEB60473B66EF901A88C
:108BE0007FCBD6ADA77F20786B914F34F249A0BFE1
:108BF000E4EC880BF19CCECBADC9C7E9072E9DCA2A
:108C00003D70F9549EBDF5D2188FA72E3FC536652D
:108C10007F4DFD1CDB7EBE6A6541DDCA4505FB4E0E
:108C2000D6ED3D886AB7775EF3C9C4CA82E6D389B8
:108C300095ABF04C98A94A9958A778834A6B0007DE
:108C400026633918E28982ABC8DEC1984AAB73F05B
:108C50005BBA61B5B8BA72B565663CA78DE0444BA6
:108C6000AEFA921AE7DF12FED0DED6E579AF5F9951
:108C70001CF29754AE0E62B5E6FC9ABAD51B56A309
:108C800008AE465F5673115C5DB9F162DD86C8E8D7
:108C90008D7FB6CAC4BA95393B86745FB77BCB6FFC
:108CA00003D3E1B6A6D6553E3C7F5D7E798A747BC0
:108CB000F2BCBAD5A6B9F18FC53F1EFF44FCCEF871
:108CC000B2F827E3EDF1BBE2BB74AEC7BF76FC5C44
:108CD00086DD4FE0B0C7E2E7860B54A29BB6BFAF7C
:108CE000F9269FAF6CF0D9E16D3BBC63D9147BA032
:108CF000F9546E03844EE59D6AB6375F2AF4E3CDDE
:108D00001E687E20AF66519DBFF25DEFD2BAB79369
:108D1000E7996E49C0EFDEB6039746AD3C7079D453
:108D2000CABADC3FB3BC0257C3B0CA8232FBBB270E
:108D3000569FEEFAE415FC5128BD53A32B2BF5AF3B
:108D4000D60927564FC87BEB9D74E99DBA903778BA
:108D500000773D908BBB9572AF88CF7EF912723B46
:108D60000032BA4AE778F2BC84DB13ECB6D5F6B62B
:108D70003575EF94EDAADEB0FAD4EA0638FFAE4AB4
:108D80001FC868B86376757CFB8014293224DCC365
:108D9000B7B5768C3E5806BC127935B8FD2F6F6595
:108DA00064C5F6707327B80776087BF0D6DB7CF9CC
:108DB000DDDBEC80E8B3934B85104EFD6D13B6619F
:108DC000EAF3DACF6B3B5C2A247FDAD305762B9B60
:108DD000EC019F7D93BA476C935DECAE46239B5AA2
:108DE0005FE62CD05ACE49A2F5155F7EDD8BDE11F1
:108DF0006F15058A329FACD1A070068A7A8A370A2D
:108E00006244BDD5BE836A67E54AECADCC3DB0E0B7
:108E100085450FE41A49FE5B4575458B9EF4265E39
:108E200021FDC88EF65997FF74E1FC06D4AA53B908
:108E3000A7FEDE402C677B9D7AAD81F2E68D069120
:108E400037FF6CD061935FD6F7446E7F4C9D13B9AA
:108E50004A70426E435219A08EE772B0B636BF8791
:108E6000F1AC7B6FBA01F3387449FDB2AFFD5EDB44
:108E700095DA1EE41DE98A27928F6DE171EFB75EE6
:108E8000FEC0AE84DF0FB45EFECCCEF87BDDFB29E6
:108E900012E6E17D894B120B128B130F26FE0BDFBE
:108EA000B8B59357BE1D9A0F7C74EA72DDFB3A7712
:108EB0006573BE3D0AD507B39EEB84BD1FBE277305
:108EC000A5C0F7AB3BBEAFB4DF18F9BEB272E58107
:108ED0005C9CDF391B9AEB3EA9ECFAEFC38E7FD680
:108EE00059390546B3D50649A36F9D5F58F6CA8721
:108EF0009F7FEF3E7FA935C442AD97CEBBBFFFFC3D
:108F0000C357CA0AE7DF3A3A698E9022B4D21AFAF6
:108F10001AB5D1B97402ED4F83C44D3E276F9367E4
:108F2000C826B294DC4DACE43A3290C41205BC7051
:108F3000167E847FC161F810FE097BE039CCBE52F9
:108F400090A11056C10A580CD9F000DC03B360069A
:108F50004C83C960810C48871BE07A488551700DAD
:108F6000A4C070180A83C1048320197A9613FE9F47
:108F70004F1E716E7CE7A39776ED5AB5AD61E33F66
:108F8000D62CCF8D7A785ECE8C070FDCFBFC5D276C
:108F9000EE583663CAF49C9B3F9AF4BBE5E3896FB5
:108FA000DCF4D98D7F8CBF69DCAB63878CF978F4F6
:108FB000436949A9B5A30E8F7CEDDADDD7945FFD37
:108FC00076CAE7231AAE4ABCEA96E1DB877D35B460
:108FD000EFD0E5432A070F1BFCB8B9D9F4B0E9E795
:108FE00041F70CFA7EE07D037F495E9AEC1FB06387
:108FF000C0A0011FF7BFB3BFB7DF53FD6EE8F77323
:10900000D2D6A4D4A45FFAEEEC9BD9B7A9CFEB7D5E
:10901000B2FB24F5F9AEF7AEDE77F48EEB5D9DF88A
:1090200074E2BD89C989B5BDDEEAB5B65766AFE859
:109030005E2712FE9EB02661724262C26FF1FB9102
:10904000C272E26F888F893F6B3C607CDAB8C2786D
:10905000B3D1646C33FC68F8C0B0CB9067B8CD7006
:10906000AD21DAF07BDCBFE2DE8A2B8BCB8FBB330A
:109070006E6C5CDFB8B658776C65EC9BB1F6D84780
:10908000621F8C9D147B75AC3136A077EB8FE9DFC6
:10909000D3BFA0DFAACFD3CFD14FD28FD227E9053C
:1090A000FDC59853315FC4BC1F531EB333667DCCDE
:1090B000C331B363B262526306C5E863DAA27F8F3D
:1090C000FE29FA58F427D1AF473F175D1ABD2E7A13
:1090D00069F49CE85BA227445F1B9D1C1D17CDA271
:1090E0001AA36AA37E883A167520EAEDA8F2A8A70B
:1090F000A3B6451546AD88CA8EBA2B6A6AD484A831
:10910000515183A3FA444547293A9FAE5E775AF7F7
:10911000ADEE0BDD67BA7DBA7FE85ED4EDD26DD7D8
:109120006DD4ADD22DD1CDD3DDADBB4567D18DD3BF
:109130008DD40DD17368617265645F6D656D6F72FA
:10914000795F736372617463687061645F7265678D
:10915000696F6E5F72785F736176653A20756E6CC9
:109160006F636B0A007368617265645F6D656D6F34
:1091700072795F736372617463687061645F726552
:1091800067696F6E5F74785F736176653A20756E9C
:109190006C6F636B0A007368617265645F6D656D07
:1091A0006F72795F736372617463687061645F7218
:1091B0006567696F6E5F736176655F68656C706522
:1091C000723A206F70656E20747820616464723D1D
:1091D00030782530366C780A007368617265645F98
:1091E0006D656D6F72795F736372617463687061CE
:1091F000645F726567696F6E5F736176655F6865EE
:109200006C7065723A206F70656E207278206164B0
:1092100064723D30782530366C780A00736861726C
:1092200065645F6D656D6F72795F7363726174639E
:10923000687061645F726567696F6E5F74785F7292
:109240006573746F72653A206C6F636B0A007368A4
:10925000617265645F6D656D6F72795F7363726172
:109260007463687061645F726567696F6E5F72785E
:109270005F726573746F72653A206C6F636B0A007E
:109280007368617265645F6D656D6F72795F777227
:109290006974653A20206C6F636B65645F74782035
:1092A0002D3E20746D7020736176650A00736861CD
:1092B0007265645F6D656D6F72795F7772697465F1
:1092C0003A20203078253034783D30782530327897
:1092D000203078253034783D307825303278200AB7
:1092E000007368617265645F6D656D6F72795F7739
:1092F000726974653A20206C6F636B65645F747883
:10930000202D3E20746D7020726573746F72650A33
:10931000007368617265645F6D656D6F72795F6916
:1093200072715F656E61626C653A0A0073686172A2
:1093300065645F6D656D6F72795F77726974653AA8
:1093400020206C6F636B65645F74780A00736861DA
:109350007265645F6D656D6F72795F726561643AA5
:10936000203078253034783D307825303278203000
:1093700078253034783D307825303278200A005214
:109380006573657420534E45530A004163746976D2
:1093900061746520415652206275730A00446973F6
:1093A00061626C6520534E45532057520A00456E4A
:1093B00061626C6520534E45532057520A00416349
:1093C00074697661746520534E4553206275730A43
:1093D0000053657420534E4553206C6F726F6D209F
:1093E0000A0053657420534E4553206869726F6DAF
:1093F000200A0053657420534E4553206C6F726FE2
:109400006D200A0053657420534E455320686972DD
:109410006F6D200A000A427573204D6F646520202D
:10942000202020202025730A00526F6D204D6F648C
:10943000652020202020202025730A0052657365B6
:1094400074204C696E65202020202025730A004975
:109450005251204C696E6520202020202020257349
:109460000A005752204C696E6520202020202020C1
:109470002025730A005265736574204952512020DB
:109480002020202025730A00534E45532052657337
:10949000657420202020203078253032780A004161
:1094A0005652205265736574202020202020307889
:1094B000253032780A00436174636820534E455367
:1094C00020726573657420627574746F6E0A005340
:1094D0006574207761746368646F672E2E2E0A00AE
:1094E00055534220696E69740A00555342206469DD
:1094F00073636F6E6E6563740A0055534220636F29
:109500006E6E6563740A00496E666C617465206CEA
:109510006F61646572002E000A00466574636820FE
:109520006C6F6164657220726F6D0A004D6F7665B5
:10953000204C6F6164657220746F207772616D00DA
:109540002E000A000A00205F5F5F5F5F5F5F5F20A1
:10955000202020202020202E5F5F2020202020207F
:1095600020205F5F202020205F5F5F5F5F5F5F5F85
:109570002020202020202020202020202020205FAC
:109580005F5F5F20205F5F5F5F5F5F5F5F0A00205C
:109590005C5F5F5F5F5F20205C20205F5F205F5F1C
:1095A0007C5F5F7C205F5F5F5F207C20207C205F92
:1095B0005F5C5F5F5F5F5F5F205C2020205F5F5FBD
:1095C0005F5F5F5F20205F2F5F2020207C2F2020A7
:1095D0005F5F5F5F5F2F0A0020202F20202F205C1D
:1095E00020205C7C20207C20205C20207C2F205FA1
:1095F0005F5F5C7C20207C2F202F207C202020207F
:109600007C20205C5F2F205F5F205C20205C2F206F
:109610002F7C2020202F2020205F5F20205C200A2C
:1096200000202F2020205C5F2F2E20205C20207C1B
:1096300020202F20205C20205C5F5F5F7C2020208A
:10964000203C20207C20202020602020205C202026
:109650005F5F5F2F5C2020202F207C2020205C205B
:10966000207C5F5F5C20205C200A00205C5F5F5FE5
:109670005F5F5C205C5F2F5F5F5F5F2F7C5F5F7C65
:109680005C5F5F5F20203E5F5F7C5F205C2F5F5FE1
:109690005F5F5F5F5F20202F5C5F5F5F20203E5C2D
:1096A0005F2F20207C5F5F5F7C5C5F5F5F5F5F2080
:1096B000202F200A0020202020202020205C5F5F17
:1096C0003E202020202020202020202020205C2F31
:1096D00020202020205C2F20202020202020205C03
:1096E0002F20202020205C2F202020202020202020
:1096F0002020202020202020205C2F200A000A008B
:109700002020202020202020202020202020202059
:1097100020202020202020202020202020202077F2
:1097200077772E6F70746978782E6F72670A000AE7
:109730000053797374656D2048773A202573205360
:10974000773A2025730A000A416464722030782534
:1097500030366C780A0042616E6B203078253032EA
:10976000780A0042616E6B73697A65203078253023
:10977000366C780A0042616E6B636F756E742030D0
:1097800078253032780A005374617475732030780C
:10979000253032780A0050657263656E742025307A
:1097A00032690A0054582062756666657220253059
:1097B00032690A005258206275666665722025304B
:1097C00032690A0053796E636572722025303269FE
:1097D0000A0011241FBECFEFD0E1DEBFCDBF14BE03
:1097E00088E10FB6F89480936000109260000FBE7D
:1097F00011E0A0E0B1E0E6E6F2ED02C005900D92C6
:10980000AC3AB107D9F71DE0ACEAB1E001C01D9256
:10981000AD3FB107E1F70E94C9500C9432690C9436
:109820000000CF93DF9360919D03635067FD92C06A
:1098300080919A03CDEAD3E0C81BD10980919903A6
:109840008D3209F074C0683009F082C083EC8093D7
:109850008D038AE5809300011092AC0188818076A7
:1098600021F0CE010E94254E4EC046E953E02A81E8
:10987000809396039981992321F48093970382E042
:109880003EC0953019F420939E0339C0963051F5AF
:10989000382F8B81813021F432E182E890E019C0C9
:1098A000823021F432E180E790E013C08330A9F4E4
:1098B000222321F434E080EC90E00BC0213021F42D
:1098C00036E18AEA90E005C0223039F436E184E9D5
:1098D00090E090939C0380939B0380E48093AC0181
:1098E000832F11C0983019F440EA53E007C0993033
:1098F00019F42093A00303C09A3009F481E0509337
:109900009C0340939B03982F8F3F39F4888187FDF8
:109910009E8180E88093AC0107C08F81882321F469
:109920008E81891708F4982F9093010111C08091BE
:10993000AC0187FF0DC0CE010E9440518F3F21F442
:109940008EE18093000104C0882311F01092010180
:1099500010929D038091000184FF3FC0809101011E
:109960008F3F09F43AC0682F893008F068E0861B01
:109970008093010180918D0398E8892780938D035E
:10998000AEE8B3E06623B9F0962FE0919B03F09127
:109990009C038091AC0186FF06C084918D93319623
:1099A0009150D9F704C081918D939150E1F7F093D4
:1099B0009C03E0939B037727C62F693040F48EE821
:1099C00093E00E94164DCC5FCC3028F401C0CEE16C
:1099D0008FEF80930101C093000194E189B18471FC
:1099E00031F49150D9F790939E0390939803DF91AF
:1099F000CF91089580916900826080936900E89A10
:109A00000895A82FB92F80E090E041E050EA6095DA
:109A10006F5F58F42D9138EF82279795879510F056
:109A2000842795273F5FC8F3F3CF0895EADF8D932E
:109A30009D930895CF93CFB7CF93DF93C3954C9B5E
:109A4000E9F74C9B11C04C9B0FC04C9B0DC04C9B2D
:109A50000BC04C9B09C04C9B07C04C9B05C04C9B4A
:109A600003C04C9B01C081C06F93C0919A03DD2756
:109A7000CF55DC4F2F9320E400C065E04C9B03C022
:109A80002F916F91DECF0F931F934F9345E55F9317
:109A900055E53F933BE014E009B104712EC06A958F
:109AA000C9F03150D8F109B1047101130BC0089409
:109AB0002795299320E4555500F46A9569F701E04C
:109AC00069B10BC0102F66E02695299320E4555507
:109AD00018F3E2CF0FEF69B10000162F455500F0E3
:109AE000404066E014710030E2F221F0000009B15C
:109AF000047103C009B10471A9F0011309C00894ED
:109B0000279568F200C06A95A9F700E069B1E5CF32
:109B1000102F66E0269528F20000ECCF11E01CBB68
:109B2000002717C03B503195C31BD04011E01CBB30
:109B30000881033CF9F00B34E9F020919803198176
:109B4000110F1213EDCF093651F10D3211F0013E14
:109B500039F700939F033F915F914F911F910F91B0
:109B60002F916F91CCB3C0FD69CFDF91CF91CFBF63
:109B7000CF91189520919F03222369F310919D03A3
:109B8000112329F534302AF130939D032093990352
:109B900010919A033BE0311B30939A031AC0009155
:109BA0009D030130A4F40AE53091000134FD12C098
:109BB00000930001CDE8D3E011C0052710E000C0FC
:109BC0000BB919C0052710E0221F00C01DC04AE5CF
:109BD00002C032ED432FC4E1D0E032E01AB114618B
:109BE0005C9A0BB11AB954E120E869E420FF05271B
:109BF0000BB92795179500C000001C3FF0F666953D
:109C0000A8F7A1F720FF05270BB9279517950000A6
:109C10001C3FC0F629913A9541F70B7E10919E03A7
:109C2000110F0BB9C651D04011F01093980311E0F9
:109C30001CBB00611AB11B7E402F4B7E55E05A952C
:109C4000F1F70BB91AB94BB986CFDF92EF92FF92B9
:109C50000F931F93CF93DF93EC01DD24898186302E
:109C600009F090C0D092BF03D092C9038C819D812E
:109C70009F938F938A819B819F938F9384EC90E035
:109C80009F938F9302E010E01F930F930E94B557AC
:109C900081E090E0A0E0B0E00A8004C0880F991F46
:109CA000AA1FBB1F0A94D2F78093C0039093C103ED
:109CB000A093C203B093C3032C813D813093C503AD
:109CC0002093C40344275527BC01CD010E949F68FF
:109CD000DC01CB018093BB039093BC03A093BD0335
:109CE000B093BE03D092C603D092C7031092CC03A8
:109CF0001092CB032DB73EB7285F3F4F0FB6F894B5
:109D00003EBF0FBE2DBFBF93AF939F938F938091A4
:109D1000C4039091C5039F938F938091C00390914A
:109D2000C103A091C203B091C303BF93AF939F93AC
:109D30008F9381EE90E09F938F931F930F930E94D8
:109D4000B5576D2D85E00E94D25A6091C4038D2DC8
:109D50000E94D25A8DB79EB70E960FB6F8949EBF4A
:109D60000FBE8DBF8091B7039091B803A091B90346
:109D7000B091BA030097A105B10509F0D6C10E94C0
:109D80004259D3C1873009F079C083E08093C8037A
:109D90008A819B81AA27BB27AC01332722272093E6
:109DA000B7033093B8034093B9035093BA038C813F
:109DB0009D817C0100271127E22AF32A042B152B11
:109DC000E092B703F092B8030093B9031093BA037B
:109DD0008E818093C903E114F1040105110509F492
:109DE00042C02091C0033091C1034091C203509101
:109DF000C303C801B7010E94BE68DC01CB01009714
:109E0000A105B10581F50E945E599F938F938091C2
:109E1000B7039091B803A091B903B091BA03BF936F
:109E2000AF939F938F938091BF0399279F938F93B5
:109E300089E291E09F938F9382E090E09F938F93CC
:109E40000E94B5570E9442598091BF038F5F809353
:109E5000BF032DB73EB7245F3F4F0FB6F8943EBF08
:109E60000FBE2DBFB1C06091B7037091B803809150
:109E7000B9039091BA030E942853A6C0883009F014
:109E8000A6C083E08093C8038A819B81AA27BB2751
:109E9000AC01332722272093B7033093B8034093B4
:109EA000B9035093BA038C819D81AA27BB27822BCB
:109EB000932BA42BB52B8093B7039093B803A09357
:109EC000B903B093BA032E812093C903BC01CD011D
:109ED00024E630E040E050E00E949F68DC01CB01C6
:109EE0002091BB033091BC034091BD035091BE0350
:109EF000BC01CD010E94BE682093C6038091C703B8
:109F0000281721F0622F82E00E94D25A8091C60366
:109F10008093C7036091B7037091B8038091B90330
:109F20009091BA030E94EE596091B7037091B80303
:109F30008091B9039091BA0361157105810591056E
:109F400009F442C02091C0033091C1034091C20383
:109F50005091C3030E94BE68DC01CB010097A105AC
:109F6000B10591F50E945E599F938F938091B7033D
:109F70009091B803A091B903B091BA03BF93AF9386
:109F80009F938F938091BF0399279F938F9385E62B
:109F900091E09F938F9382E090E09F938F930E9434
:109FA000B5570E9442598091BF038F5F8093BF03D2
:109FB000682F85E00E94D25A8DB79EB70C960FB6D7
:109FC000F8949EBF0FBE8DBF3FEFD32EAEC0893039
:109FD000A1F481EA91E09F938F9382E090E09F93B8
:109FE0008F930E94B55781E08093C8030E94645408
:109FF0006D2D83E00E94D25A94C0843009F04DC088
:10A000008A819B81AA27BB27AC0133272227209373
:10A01000B7033093B8034093B9035093BA038C81CC
:10A020009D81AA27BB27822B932BA42BB52B809332
:10A03000B7039093B803A093B903B093BA03BF9347
:10A04000AF939F938F9387EB91E09F938F9382E0E1
:10A0500090E09F938F930E94B557E090C003F090DB
:10A06000C1030091C2031091C3032091B703309143
:10A07000B8034091B9035091BA0360E070E080E00A
:10A0800090E00E94A4562DB73EB7285F3F4F0FB611
:10A09000F8943EBF0FBE2DBF48C08B3031F487E02F
:10A0A0008093C8038FEC91E007C08A3071F486E09A
:10A0B0008093C8038EED91E09F938F9382E090E0B0
:10A0C0009F938F930E94B5572CC08C30D1F48EEEA5
:10A0D00091E09F938F9382E090E09F938F930E94F3
:10A0E000B55788E190E02DE00FB6F894A8958093DD
:10A0F00060000FBE209360000F900F900F900F90A4
:10A10000FFCF8D3091F48EEF91E09F938F9382E09B
:10A1100090E09F938F930E94B5578A818093F503B7
:10A12000DD240F900F900F900F908DEE93E09093A1
:10A130009C0380939B038D2D9927DF91CF911F91D5
:10A140000F91FF90EF90DF9008958FE3E7EBF3E03E
:10A1500011928A95E9F71092B7031092B803109202
:10A16000B9031092BA031092BB031092BC03109271
:10A17000BD031092BE0381E08093C8031092C9030F
:10A180001092CA031092CC031092CB038093F50374
:10A190000895CFEFD0E1DEBFCDBF0E94E25183E052
:10A1A00091E09093FA0D8093F90D0E946A5F0E94EE
:10A1B0009E590E94395C0E947C520E941D5E0E9442
:10A1C000345E82E390E00E94295F0E94A5500E94C5
:10A1D000165E0E94FA4C0E949C5E78940E948F5CEE
:10A1E0000E949F5C8FE092E09F938F930E947F5923
:10A1F0000F900F908091C803863019F00E94114C87
:10A20000F9CF60E085E00E94D25A0E94355A0E9440
:10A210005B5A87EB93E00E94CF5C0E949F5C0E9498
:10A22000BD5C0E94615C0E94475E89E192E09F9361
:10A230008F930E947F590F900F908091C8038730B1
:10A2400019F00E94114CF9CF83E292E09F938F9313
:10A250000E947F590E949E590E94345E0F900F9079
:10A260008091F503882329F082E390E00E94295F22
:10A2700004C00E948F5C0E94615C0E94A550AECF1A
:10A28000EF92FF921F93CF937C01162F8091C90309
:10A290008617C8F4862F99279F938F938091C903BF
:10A2A00099279F938F9385E392E09F938F930E94CA
:10A2B0007F591091C9038DB79EB706960FB6F894D3
:10A2C0009EBF0FBE8DBF8091C8038330B1F58091D2
:10A2D000C903811B8093C90399279F938F93812F73
:10A2E00099279F938F938091B7039091B803A09182
:10A2F000B903B091BA03BF93AF939F938F9388E74D
:10A3000092E09F938F9384E090E09F938F930E94BD
:10A31000B557EDB7FEB73C960FB6F894FEBF0FBE2B
:10A32000EDBFC12FC150CF3F41F0F70181917F01B7
:10A330000E9460540E944A54F5CF812F9927CF91F3
:10A340001F91FF90EF900895EF92FF920F931F934C
:10A35000CF937C01C62F8091CA03861708F4C82FBB
:10A360008C1B8093CA0399279F938F930C2F1127DF
:10A370001F930F9387EC92E09F938F9384E090E07C
:10A380009F938F930E94B55790E02DB73EB7285FFB
:10A390003F4F0FB6F8943EBF0FBE2DBF9C1750F431
:10A3A000F801E954FC4F8689D7018D937D019F5FA9
:10A3B0009C17C8F38C2F9927CF911F910F91FF9075
:10A3C000EF90089582E08093C00088E98093C100F7
:10A3D00084E18093C4000895982F8091C00085FF88
:10A3E000FCCF9093C6000895CF93DF93EC01888152
:10A3F0000E94EC5189918823D1F7DF91CF91089584
:10A40000CF93DF93EC01FE0184912196882319F00C
:10A410000E94EC51F8CFDF91CF910895CF93C82FD0
:10A420008A3019F48DE00E94EC518091C00085FFC4
:10A43000FCCFC093C60080E090E0CF910895FC016E
:10A440001082758364837383628341834783468369
:10A450000895FC0190818181981718F080E090E0C8
:10A4600014C0A481B5816D938781815019F48181D5
:10A47000A81BB1098783B583A4839FB7F894808113
:10A480008F5F80839FBF81E090E099270895FC0152
:10A4900080818823E9F3A281B3812D918681815047
:10A4A00019F48181A81BB109B383A28386839FB766
:10A4B000F8948081815080839FBF822F99270895CF
:10A4C000FC018081882319F48FEF9FEF0895A2810A
:10A4D000B3812D918681815019F48181A81BB10926
:10A4E000B383A28386839FB7F89480818150808351
:10A4F0009FBF822F9927089511B812B887B1856739
:10A5000087B987B1857F87B988B1877988B988B1DC
:10A51000856088B984B18F6084B985B18F6085B951
:10A520008AB1806E8AB95E9A8BB18F758BB90895A6
:10A53000EF92FF920F931F93CF937B018C019F9318
:10A540008F937F936F9380EF92E09F938F9380E23E
:10A5500090E09F938F930E94B5578DB79EB7089652
:10A560000FB6F8949EBF0FBE8DBFC7E181E090E0AB
:10A57000A0E0B0E00C2E04C0880F991FAA1FBB1FDB
:10A580000A94D2F78E219F21A023B1230097A10521
:10A59000B10561F087E093E09F938F9380E290E0B4
:10A5A0009F938F930E94B557449A0BC0449889E0BB
:10A5B00093E09F938F9380E290E09F938F930E940C
:10A5C000B5570F900F900F900F90459A4598C15036
:10A5D00068F68BE093E09F938F9380E290E09F93E7
:10A5E0008F930E94B557469A46984298429A0F9088
:10A5F0000F900F900F90CF911F910F91FF90EF90C0
:10A6000008958091B1019091B201A091B301B091F0
:10A61000B4018093AD019093AE01A093AF01B093CC
:10A62000B001BF93AF939F938F938DE093E09F937F
:10A630008F9388E090E09F938F930E94B5578DB7DA
:10A640009EB708960FB6F8949EBF0FBE8DBF0895B3
:10A65000EF92FF920F931F937B018C019F938F9337
:10A660007F936F9381E393E09F938F9388E090E0D3
:10A670009F938F930E94B557E092B101F092B2017F
:10A680000093B3011093B4018FEF81B92898299AF0
:10A690002A9AC801B7010E9498528DB79EB70896B2
:10A6A0000FB6F8949EBF0FBE8DBF1F910F91FF9004
:10A6B000EF9008958091AD019091AE01A091AF010E
:10A6C000B091B001BF93AF939F938F9387E593E0D1
:10A6D0009F938F9388E090E09F938F930E94B5574C
:10A6E0008091AD019091AE01A091AF01B091B00108
:10A6F000BC01CD010E9428538DB79EB708960FB6B6
:10A70000F8949EBF0FBE8DBF0895EF92FF920F93F6
:10A710001F937B018C019F938F937F936F938EE7A1
:10A7200093E09F938F9388E090E09F938F930E9494
:10A73000B557E092B101F092B2010093B3011093CA
:10A74000B40111B812B82898299A2A9AC801B701F9
:10A750000E9498522A9800000000000000000000AB
:10A7600000008DB79EB708960FB6F8949EBF0FBE37
:10A770008DBF1F910F91FF90EF9008958091B101CF
:10A780009091B201A091B301B091B4010196A11DC5
:10A79000B11D8093B1019093B201A093B301B09326
:10A7A000B4012A9A4098409A2A98000000000000BC
:10A7B000000000000000089580B19927089583EA01
:10A7C00093E09F938F9388E090E09F938F930E94F4
:10A7D000B5572A9A289A11B812B80F900F900F9077
:10A7E0000F900895EF92FF920F931F937B018C01BE
:10A7F0009F938F937F936F9388EB93E09F938F93B7
:10A8000080E190E09F938F930E94B55711B812B8E2
:10A810002898299A2A9AC801B7010E9498522A9822
:10A8200000000000000000000000000080B12A9A33
:10A83000289A11B812B82DB73EB7285F3F4F0FB610
:10A84000F8943EBF0FBE2DBF99271F910F91FF9027
:10A85000EF900895DF92EF92FF920F931F937B0189
:10A860008C010E94F253D82E0894E11CF11C011DAA
:10A87000111DC801B7010E94F2532D2D3327322F2D
:10A8800022279927822B932B1F910F91FF90EF90F6
:10A89000DF9008958091B1019091B201A091B30130
:10A8A000B091B4010196A11DB11D8093B1019093A7
:10A8B000B201A093B301B093B4014098409A0895B7
:10A8C000299882B9299A089582ED93E09F938F93F6
:10A8D00088E090E09F938F930E94B557299A289A19
:10A8E00011B812B80F900F900F900F900895DF924B
:10A8F000EF92FF920F931F937B018C01D42E842F34
:10A9000099279F938F931F930F93FF92EF9287EE58
:10A9100093E09F938F9380E190E09F938F930E94A9
:10A92000B5578FEF81B92898299A2A9AC801B7019B
:10A930000E9498522998D2B8299A0000000000007D
:10A94000000000000000289A11B812B88DB79EB719
:10A950000A960FB6F8949EBF0FBE8DBF1F910F9140
:10A96000FF90EF90DF9008958F929F92AF92BF92E9
:10A97000CF92DF92EF92FF920F931F93CF93DF93CB
:10A980006B017C01480159018A01BF92AF929F92ED
:10A990008F925F934F93FF92EF92DF92CF928AE074
:10A9A00094E09F938F9388E090E09F938F930E9411
:10A9B000B557C701B6010E942853A70196018DB76C
:10A9C0009EB70E960FB6F8949EBF0FBE8DBFF701CF
:10A9D000E601C80DD91DEA1DFB1D2C173D074E07CA
:10A9E0005F0730F5D8018C91299882B9299A2F5F99
:10A9F0003F4F4F4F5F4F2C173D074E075F07A8F49F
:10AA00008091B1019091B201A091B301B091B401D4
:10AA10000196A11DB11D8093B1019093B201A09345
:10AA2000B301B093B4014098409A0F5F1F4FD5CF48
:10AA300082ED93E09F938F9388E090E09F938F93B4
:10AA40000E94B5570F900F900F900F90299A289A57
:10AA500011B812B8DF91CF911F910F91FF90EF9035
:10AA6000DF90CF90BF90AF909F908F9008958F927E
:10AA70009F92AF92BF92CF92DF92EF92FF920F938D
:10AA80001F93CF93DF936B017C01EA0148015901C9
:10AA90003F932F931F930F935F934F939F938F93A6
:10AAA0007F936F9386E494E09F938F9388E090E088
:10AAB0009F938F930E94B557C701B6010E9485539B
:10AAC000A70196018DB79EB70E960FB6F8949EBF5C
:10AAD0000FBE8DBF87017601E80CF91C0A1D1B1DF6
:10AAE0002E153F054007510738F5FE01E20FF31F11
:10AAF00080B180838091B1019091B201A091B301A6
:10AB0000B091B4010196A11DB11D8093B101909344
:10AB1000B201A093B301B093B4012A9A4098409A2D
:10AB20002A980000000000000000000000002F5FD5
:10AB30003F4F4F4F5F4FD4CF83EA93E09F938F9364
:10AB400088E090E09F938F930E94B5570F900F90ED
:10AB50000F900F902A9A289A11B812B8DF91CF91CE
:10AB60001F910F91FF90EF90DF90CF90BF90AF902B
:10AB70009F908F9008958F929F92AF92BF92CF92A5
:10AB8000DF92EF92FF920F936B017C0149015A0112
:10AB90005F934F933F932F939F938F937F936F93E5
:10ABA00082E894E09F938F9388E090E09F938F9347
:10ABB0000E94B557C701B6010E9428538DB79EB7B2
:10ABC0000C960FB6F8949EBF0FBE8DBF8C0C9D1CCB
:10ABD000AE1CBF1CC814D904EA04FB0408F042C030
:10ABE000C701B6012FEF3FE040E050E00E94BE6891
:10ABF000DC01CB010097A105B105B1F4FF92EF9202
:10AC0000DF92CF9288EA94E09F938F9388E090E060
:10AC10009F938F930E94B5578DB79EB708960FB636
:10AC2000F8949EBF0FBE8DBF299802B9299A8091D2
:10AC3000B1019091B201A091B301B091B40101961C
:10AC4000A11DB11D8093B1019093B201A093B301F6
:10AC5000B093B4014098409A0894C11CD11CE11CE7
:10AC6000F11CB8CF82ED93E09F938F9388E090E042
:10AC70009F938F930E94B5570F900F900F900F9056
:10AC8000299A289A11B812B80F91FF90EF90DF908F
:10AC9000CF90BF90AF909F908F900895262F33272D
:10ACA000322F22272827392761E270E147E050E060
:10ACB000C901880F991F37FF04C09C012627372739
:10ACC00001C09C014150504057FFF2CFC901089587
:10ACD000EF92FF920F931F93CF93DF939C017B0121
:10ACE00080E090E0EC018617970750F48901F801A5
:10ACF00061918F010E944E562196CE15DF05B8F363
:10AD0000DF91CF911F910F91FF90EF900895EF92F7
:10AD1000FF920F931F93CF93DF937A01C0E0D0E0AF
:10AD2000C417D50750F48B01F80161918F010E947F
:10AD30004E562196CE15DF05B8F3DF91CF911F91C6
:10AD40000F91FF90EF9008952F923F924F925F9254
:10AD50006F927F928F929F92AF92BF92CF92DF922B
:10AD6000EF92FF920F931F93CF93DF93CDB7DEB790
:10AD700023970FB6F894DEBF0FBECDBF5B016C0109
:10AD800039014A01170128011B821A8219820E9487
:10AD900085539F928F927F926F92DF92CF92BF9254
:10ADA000AF9286EC94E09F938F9380E490E09F9322
:10ADB0008F930E94B557860175018DB79EB70C968B
:10ADC0000FB6F8949EBF0FBE8DBFE614F7040805BA
:10ADD000190508F046C0E114F1040105110581F1DF
:10ADE000C801B701A20191010E94BE68DC01CB013C
:10ADF0000097A105B10521F5EA81FB81FF93EF934F
:10AE00001F930F93FF92EF92F9818F2F99279F93B2
:10AE10008F9383E095E09F938F9380E490E09F93DE
:10AE20008F930E94B55729812F5F29831B821A8235
:10AE30008DB79EB70C960FB6F8949EBF0FBE8DBF10
:10AE40000E94DC53682F8A819B810E944E569B830F
:10AE50008A830E94BE530894E11CF11C011D111D40
:10AE6000B4CFD801C7019F77A070B0700097A1053B
:10AE7000B105F9F4EA81FB81FF93EF931F930F93E0
:10AE8000FF92EF92F9818F2F99279F938F938FE3F2
:10AE900095E09F938F9380E490E09F938F930E941F
:10AEA000B5578DB79EB70C960FB6F8949EBF0FBEE0
:10AEB0008DBF0E94DF538A819B8123960FB6F89441
:10AEC000DEBF0FBECDBFDF91CF911F910F91FF90DD
:10AED000EF90DF90CF90BF90AF909F908F907F903A
:10AEE0006F905F904F903F902F9008956F927F9258
:10AEF0008F929F92AF92BF92CF92DF92EF92FF928A
:10AF00000F931F93CF93DF936B017C0149015A018B
:10AF10003801C0E0D0E0860E971EA81EB91EC814E6
:10AF2000D904EA04FB0488F400E010E020E030E0FB
:10AF3000A301C701B6010E94375540E050E0B301BC
:10AF4000CE010E948756EC01EACFCE01DF91CF916E
:10AF50001F910F91FF90EF90DF90CF90BF90AF9037
:10AF60009F908F907F906F900895CF93DF93CDB790
:10AF7000DEB72D813E816F817885809102019091AD
:10AF8000030182239323892B69F040E850E088EF86
:10AF900093E00E94D365BE01675F7F4F88EF93E027
:10AFA0000E94E965DF91CF9108952F923F924F92D1
:10AFB0005F926F927F928F929F92AF92BF92CF9249
:10AFC000DF92EF92FF920F931F93CF93DF93CDB752
:10AFD000DEB723970FB6F894DEBF0FBECDBF2B01AF
:10AFE0003C0149015A0118011982CC24DD242115A4
:10AFF00031054105510509F4A3C0780120E030E096
:10B00000F601E20DF31D8FE090E09B838A8381912E
:10B01000280F311D8A819B8101979B838A8397FF2B
:10B02000F6CF232B19F491E099837BC0E981EE23BD
:10B0300049F08BE795E09F938F930E947F59198287
:10B040000F900F90C601AA27BB27840D951DA61D42
:10B05000B71DBF93AF939F938F938EE795E09F9318
:10B060008F930E947F598DB79EB706960FB6F894BE
:10B070009EBF0FBE8DBF8701EFE0F0E0FB83EA8348
:10B08000F80181918F0199279F938F9385E895E02F
:10B090009F938F930E947F590F900F900F900F9066
:10B0A0008A819B8101979B838A8397FFE9CF8BE8F5
:10B0B00095E09F938F930E947F590F900F90870187
:10B0C000EFE0F0E0FB83EA83F80191918F01892F93
:10B0D00081528E3578F4892F99279F938F938EE82C
:10B0E00095E09F938F930E947F590F900F900F9040
:10B0F0000F9008C081E995E09F938F930E947F593C
:10B100000F900F908A819B8101979B838A8397FF81
:10B11000DBCF83E995E09F938F930E947F590F9037
:10B120000F90E0E1F0E0CE0EDF1EEE0EFF1EC60136
:10B13000AA27BB2788159905AA05BB0508F45ECF89
:10B1400023960FB6F894DEBF0FBECDBFDF91CF912F
:10B150001F910F91FF90EF90DF90CF90BF90AF9035
:10B160009F908F907F906F905F904F903F902F9027
:10B1700008958F929F92AF92BF92CF92DF92EF92FB
:10B18000FF920F931F937B018C0149015A010E948A
:10B19000855367017801C814D904EA04FB04A8F5B3
:10B1A000D701C6018F709070A070B0700097A10594
:10B1B000B10591F4FF92EF92DF92CF9286E995E08C
:10B1C0009F938F930E947F598DB79EB706960FB6B7
:10B1D000F8949EBF0FBE8DBF0E94DC53182F0E94B3
:10B1E000BE53812F99279F938F938EE995E09F936C
:10B1F0008F930E947F590F900F900F900F9008949B
:10B20000C11CD11CE11CF11CC6CF84EA95E09F93C0
:10B210008F930E947F590E94DF530F900F901F91D0
:10B220000F91FF90EF90DF90CF90BF90AF909F90E5
:10B230008F9008951F920F920FB60F9211248F9343
:10B240009F93809178049091790401979093790469
:10B2500080937804892B79F484EF91E090937904BA
:10B260008093780480917A0490917B040196909366
:10B270007B0480937A049F918F910F900FBE0F9063
:10B280001F90189589E0809381008FE39CE990934B
:10B29000890080938800109285001092840010929B
:10B2A0007B0410927A0484EF91E090937904809368
:10B2B000780482E080936F0078940895CF93DF93B1
:10B2C0008091780490917904AA27BB2724EF31E07C
:10B2D00040E050E0FA01E901C81BD90BEA0BFB0B77
:10B2E000BE01CF010E94E068DA01C90120917A0411
:10B2F00030917B04820F931FDF91CF9108950F93BC
:10B300001F93CF93DF93CDB7DEB707E010E00C0FAC
:10B310001D1FF801819191918F0140E850E0BC011F
:10B320008CE794E00E94D365B8018CE794E00E941A
:10B33000E965DF91CF911F910F91089581E080938E
:10B340001A018093190108950F931F930E940153CE
:10B3500084E391E99F938F9380E890E09F938F938C
:10B360000E94B55700E410E020E030E04DE355E0E6
:10B3700060E070E180E090E00E94375510921A0181
:10B380000E945A530F900F900F900F901F910F91A2
:10B3900008950F931F930E94015385E691E99F93AF
:10B3A0008F9380E890E09F938F930E94B55700E4BD
:10B3B00010E020E030E04DEF54E060E070E080E02D
:10B3C00090E00E943755109219010E945A530F9035
:10B3D0000F900F900F901F910F9108959B01AC015A
:10B3E0006134710581059105A8F0809119018823C8
:10B3F00089F05F934F933F932F9386E991E99F9351
:10B400008F9380E890E09F938F930E94B5570E949E
:10B41000C9591CC0213480E1380780E0480780E02A
:10B42000580700F180911A018823E1F05F934F9350
:10B430003F932F9389ED91E99F938F9380E890E05C
:10B440009F938F930E94B5570E94A45980E090E08B
:10B450002DB73EB7285F3F4F0FB6F8943EBF0FBEE3
:10B460002DBF089581E090E008950F931F93809180
:10B4700019018823E9F48CE192E99F938F9380E886
:10B4800090E09F938F930E94B55700E410E020E076
:10B4900030E04DEF54E060E070E080E090E00E942A
:10B4A000B45481E0809319010F900F900F900F908A
:10B4B0001F910F9108950F931F9380911A01882374
:10B4C000E9F48EE492E99F938F9380E890E09F9354
:10B4D0008F930E94B55700E410E020E030E04DE388
:10B4E00055E060E070E180E090E00E94B45481E0BB
:10B4F00080931A010F900F900F900F901F910F9152
:10B50000089560E070E080E090E00E94F253809344
:10B51000FC0461E070E080E090E00E94F2538093D0
:10B52000800562E070E080E090E00E94F25380933A
:10B530007E0508954091FC0460E070E080E090E0BA
:10B540000E9477544091800561E070E080E090E0D7
:10B550000E94775440917E0562E070E080E090E0C8
:10B560000E94775408956EEF7FEF80E090E00E9494
:10B57000F25380937D056FEF7FEF80E090E00E94B3
:10B58000F25380937F0540E064EE7FEF80E090E02F
:10B590000E94775440E065EE7FEF80E090E00E94EB
:10B5A000775408951F93CF93C82F162F80911901B8
:10B5B000882381F080E892E99F938F9380E890E060
:10B5C0009F938F930E94B5570E94815A0F900F90BE
:10B5D0000F900F90812F99279F938F9382E090E097
:10B5E0009F938F938C2F99279F938F9381E090E067
:10B5F0009F938F938DEA92E99F938F9380E890E0D9
:10B600009F938F930E94B5570E9401538DB79EB7A9
:10B610000C960FB6F8949EBF0FBE8DBF8091B501FA
:10B62000882311F00E94B35A45EA60E070E080E0A0
:10B6300090E00E9477544C2F61E070E080E090E051
:10B640000E947754412F62E070E080E090E00E9419
:10B6500077545E985F985D9A2098289A8091B501FA
:10B66000882341F0239A2B9885E88A95F1F72B9A45
:10B67000239809C028EC30E084EF91E00197F1F7BE
:10B6800021503040C9F75D985E9A209A2B982398F4
:10B690005E9A5F9880911901882381F081EE92E98A
:10B6A0009F938F9380E890E09F938F930E94B5576C
:10B6B0000E949A5A0F900F900F900F900E945A5329
:10B6C000CF911F91089581E193E99F938F9380E833
:10B6D00090E09F938F930E94B55781E08093B501CE
:10B6E00060E00E94D25A0F900F900F900F90089533
:10B6F00040917D056EEF7FEF80E090E00E947754EF
:10B7000040917F056FEF7FEF80E090E00E947754DB
:10B7100008955E985F985D9A2098289A28EC30E00A
:10B7200084EF91E00197F1F721503040C9F75D981F
:10B730005E9A209A5E9A5F980895EF92FF920F9317
:10B740001F93CF93DF93EC018B017A0180911A0153
:10B75000882389F08CE293E99F938F9380E890E0AF
:10B760009F938F930E94B55781E090E00F900F90C8
:10B770000F900F9077C00E94015360E070E180E06D
:10B7800090E00E94F253853A29F00E945A5381E0DA
:10B7900090E068C061E070E180E090E00E94F253C8
:10B7A000888362E070E180E090E00E94F253F8014B
:10B7B000808399279F938F9382E090E19F938F934B
:10B7C000888199279F938F9381E090E19F938F9336
:10B7D0008DE493E99F938F9380E890E09F938F93FC
:10B7E0000E94B557F80180819927AA27BB278C01B1
:10B7F0009D01A70163E070E180E090E00E94375571
:10B800004AE560E070E180E090E00E9477545E9845
:10B810005F985D9A2098289A8DB79EB70C960FB6C0
:10B82000F8949EBF0FBE8DBF8091B501882341F073
:10B83000239A2B9885E88A95F1F72B9A239809C0CB
:10B8400028EC30E084EF91E00197F1F7215030408F
:10B85000C9F75D985E9A209A5E9A5F980E945A5343
:10B8600080E090E0DF91CF911F910F91FF90EF90DA
:10B8700008955B9A539810928605109285052B9A2D
:10B88000239881E090E090938805809387055F98E6
:10B8900010928A05109289055D985E9A209A1092FE
:10B8A0008205109281055E9A10928405109283059C
:10B8B00010928D0510928E0510928C0510928B05BA
:10B8C00008958FE793E99F938F930E947F59F8948F
:10B8D000539A5B980F900F9080E197E20197F1F7F0
:10B8E0005B9A5398789480918D058F5F80938D0536
:10B8F0000895239A2B9885E88A95F1F72B9A239837
:10B900000895239881E090E09093880580938705BF
:10B910000895239A109288051092870508955D98DE
:10B920005E9A209A8BE893E99F938F930E947F59A8
:10B9300010928205109281050F900F9008955F98E4
:10B9400010928A05109289058DE993E99F938F9350
:10B950000E947F590F900F9008955F9A81E090E0C8
:10B9600090938A05809389058EEA93E99F938F933C
:10B970000E947F590F900F9008955D9A2098289A01
:10B9800081E090E090938205809381058EEB93E9AE
:10B990009F938F930E947F590F900F900895FC0101
:10B9A00081859285A385B48580509048A040B040A1
:10B9B00041F45E9A109284051092830581ED93E91B
:10B9C00009C05E9881E090E09093840580938305A0
:10B9D00082EE93E99F938F930E947F590F900F906F
:10B9E00008955E9A109284051092830583EF93E97F
:10B9F0009F938F930E947F590F900F9008955E98A8
:10BA000081E090E0909384058093830584E094E93D
:10BA10009F938F930E947F590F900F9008958823D2
:10BA200019F08BE191E008958EE191E0089588236B
:10BA300019F082E291E0089587E291E00895882369
:10BA400019F08BE291E0089581E391E008958091EF
:10BA500081050E94175D9F938F9385E194E99F93E1
:10BA60008F930E947F590F900F900F900F908091AD
:10BA700083050E941F5D9F938F9389E294E99F93B2
:10BA80008F930E947F590F900F900F900F9080918D
:10BA900085050E940F5D9F938F938CE394E99F939C
:10BAA0008F930E947F590F900F900F900F9080916D
:10BAB00087050E940F5D9F938F938FE494E99F9376
:10BAC0008F930E947F590F900F900F900F9080914D
:10BAD00089050E940F5D9F938F9382E694E99F935F
:10BAE0008F930E947F590F900F900F900F9080912D
:10BAF0008B050E940F5D9F938F9385E794E99F9339
:10BB00008F930E947F590F900F900F900F9080910C
:10BB10008D0599279F938F9388E894E99F938F933E
:10BB20000E947F590F900F900F900F9080918E057B
:10BB300099279F938F938FE994E99F938F930E9406
:10BB40007F590F900F900F900F9008951F920F92B2
:10BB50000FB60F9211242F933F938F939F93EF93E0
:10BB6000FF938091B300835F8093B300809193052E
:10BB70009091B601981710F43F9801C03F9A9F3FEB
:10BB800019F41092B60103C09F5F9093B6018091A3
:10BB90008F05909190059C0101969093900580935C
:10BBA0008F05809191059091920528173907B1F47E
:10BBB00080919405E82FFF27E95CFE4F8F5F80930B
:10BBC00094058081809393051092900510928F05C3
:10BBD00080919405803411F410929405FF91EF91B7
:10BBE0009F918F913F912F910F900FBE0F901F90BB
:10BBF00018959093920580939105089580E098E0C0
:10BC00009093920580939105089580E092E090933F
:10BC1000920580939105089580E094E090939205B9
:10BC200080939105089580939305089580919305DD
:10BC30008D3FE1F710927000089580E094E09093BA
:10BC40009205809391058FE780939305109290055C
:10BC500010928F0581E08093B10080917000826026
:10BC60008093700078940895F894809173008860B0
:10BC70008093730080916800886080936800789456
:10BC800081E090E090938C0580938B050895F89463
:10BC900080917300877F80937300789410928C0555
:10BCA00010928B050895F894549A80918E058F5FB9
:10BCB00080938E0588E190E028E00FB6F894A8956F
:10BCC000809360000FBE20936000FFCF1F920F9201
:10BCD0000FB60F9211242F933F934F935F936F935F
:10BCE0007F938F939F93AF93BF93EF93FF934B9962
:10BCF00012C086EB94E99F938F930E947F590F9017
:10BD00000F908FEC94E99F938F930E947F590E942C
:10BD1000535E0F900F90FF91EF91BF91AF919F9164
:10BD20008F917F916F915F914F913F912F910F90E4
:10BD30000FBE0F901F90189580EE94E99F938F93FC
:10BD40000E947F59549AF8940F900F908AEE94E9CC
:10BD50009F938F930E947F590F900F9049E024EF9B
:10BD600031E084EF91E00197F1F721503040C9F7BD
:10BD70004150A9F747983F9854988AEF94E99F93C8
:10BD80008F930E947F590F900F900895AF92BF92AA
:10BD9000CF92DF92EF92FF920F931F93CF93DF9397
:10BDA00087E095E99F938F930E947F590E94776067
:10BDB0000F900F9021E0C22E91E1E92E91E0F92E33
:10BDC00085E1A82E81E0B82EF501C191D1915F01E6
:10BDD00000E010E0F7018081918108171907A8F4AD
:10BDE000FE012196D490C8019370892B41F486E11D
:10BDF00095E99F938F930E947F590F900F908D2DFF
:10BE00000E94A3610F5F1F4FE5CFCA9482E090E0CC
:10BE1000E80EF91EC7FED8CF8091BB01882321F41C
:10BE200080E00E94A361F8CF0E94806088E195E9DC
:10BE30009F938F930E947F590F900F90DF91CF9126
:10BE40001F910F91FF90EF90DF90CF90BF90AF9038
:10BE50000895CF938AE195E99F938F930E947F592C
:10BE60000E948F5C0E94F15C0E94C65E2B980E942B
:10BE7000815C0E94FF5C0E949F5C0E94BD5C0E94EE
:10BE8000615C0F900F908CE295E99F938F930E94D5
:10BE90007F59C0E00F900F9028EC30E084EF91E0E4
:10BEA0000197F1F721503040C9F780E495E99F935D
:10BEB0008F930E947F590F900F90CF5FCE3160F328
:10BEC00082E495E99F938F930E947F590F900F9082
:10BED000CF910895CF93C7E284E495E99F938F9320
:10BEE0000E947F590F900F90C150C7FFF5CF86E495
:10BEF00095E99F938F930E947F590F900F908FE841
:10BF000095E99F938F930E947F590F900F9088ED32
:10BF100095E99F938F930E947F590F900F9081E234
:10BF200096E99F938F930E947F590F900F908BE615
:10BF300096E99F938F930E947F590F900F9085EB06
:10BF400096E99F938F930E947F590F900F908EEFE9
:10BF500096E99F938F930E947F590F900F9080E0F6
:10BF600097E99F938F930E947F590F900F908FE2D4
:10BF700097E99F938F930E947F590F900F9087E7C7
:10BF800091E09F938F938BE791E09F938F9381E351
:10BF900097E99F938F930E947F598DB79EB706961E
:10BFA0000FB6F8949EBF0FBE8DBFCF9108958091BC
:10BFB000B7039091B803A091B903B091BA03BF93AE
:10BFC000AF939F938F9387E497E99F938F930E94FA
:10BFD0007F598DB79EB706960FB6F8949EBF0FBED9
:10BFE0008DBF8091BF0399279F938F9386E597E933
:10BFF0009F938F930E947F590F900F900F900F90F7
:10C000008091C0039091C103A091C203B091C3037A
:10C01000BF93AF939F938F9383E697E99F938F93FB
:10C020000E947F598DB79EB706960FB6F8949EBFB3
:10C030000FBE8DBF8091C4039091C5039F938F93D2
:10C0400085E797E99F938F930E947F590F900F90F8
:10C050000F900F908091C80399279F938F9387E843
:10C0600097E99F938F930E947F590F900F900F90A5
:10C070000F908091C60399279F938F9386E997E944
:10C080009F938F930E947F590F900F900F900F9066
:10C090008091CA0399279F938F9384EA97E99F938E
:10C0A0008F930E947F590F900F900F900F90809167
:10C0B000C90399279F938F9384EB97E99F938F935D
:10C0C0000E947F590F900F900F900F908091CB039B
:10C0D0009091CC039F938F9384EC97E99F938F93D8
:10C0E0000E947F590F900F900F900F90089560E07D
:10C0F00070E080E090E00E948A610E94A66008954E
:10C100000E947861089581E08093BB0108950E94A8
:10C11000F8600895AF92BF92CF92DF92EF92FF92B4
:10C120000F931F935B016C01C801AA27BB277C01F9
:10C130008D01C601B5010E943B611F910F91FF90D7
:10C14000EF90DF90CF90BF90AF9008951092C5010F
:10C150001092C4011092C0011092C1011092C2014C
:10C160001092C3011092BC011092BD011092BE0149
:10C170001092BF0160E070E080E090E00E942853E0
:10C180000895EF92FF920F931F93CF93DF93EB01EC
:10C1900000E010E00617170768F47C01F7018191B1
:10C1A0007F010E9460540E944A540F5F1F4F0C177A
:10C1B0001D07A0F39E01442755278091BC01909153
:10C1C000BD01A091BE01B091BF01820F931FA41FBA
:10C1D000B51F8093BC019093BD01A093BE01B093A5
:10C1E000BF01DF91CF911F910F91FF90EF900895C4
:10C1F00040E02091C4013091C501F901E950FA4FA6
:10C20000808383E02F3F380739F460E074E087EFE4
:10C2100095E00E94C1600FC02F5F374069F460E075
:10C2200074E087EF99E00E94C1608FEF9FEF9093D9
:10C23000C5018093C40141E08091C4019091C50182
:10C2400001969093C5018093C4018091C0019091A3
:10C25000C101A091C201B091C3010196A11DB11D00
:10C260008093C0019093C101A093C201B093C30118
:10C27000842F99270895EF92FF920F931F93CF93E6
:10C28000DF939B01AC01EB01C901AA27BB27E20E9A
:10C29000F31E041F151F8E159F05A007B10708F593
:10C2A0008091C0019091C1018C1B9D0B2091C40114
:10C2B0003091C501F901E81BF90B2817390718F46B
:10C2C000E950F24F02C0E950FA4F80810E94F860B5
:10C2D0002196CE01AA27BB278E159F05A007B1077F
:10C2E000F8F2DF91CF911F910F91FF90EF90089599
:10C2F0006091C4017091C50184E0613078071CF43D
:10C3000087EF95E004C06050744087EF99E00E9489
:10C31000C1600895DC01CB011092C6011092D101D9
:10C320001092D2011092D3011092D4011092C70141
:10C330001092C8018093C9019093CA01A093CB01C8
:10C34000B093CC010895282F3327442755276091B7
:10C35000C601062E04C0220F331F441F551F0A9426
:10C36000D2F78091D1019091D201A091D301B091E7
:10C37000D401822B932BA42BB52B8093D1019093C6
:10C38000D201A093D301B093D401862F885F80930C
:10C39000C601803178F08091C701E82FFF27EE0FAA
:10C3A000FF1FE158FE4F0190F081E02D099580912B
:10C3B000C601EFCF08958091C9019091CA01A09163
:10C3C000CB01B091CC01BC01CD0108958091D10188
:10C3D0009091D20108952091D1013091D2014091E4
:10C3E000D3015091D401082E04C056954795379536
:10C3F00027950A94D2F72093D1013093D20140932C
:10C40000D3015093D4019091C601981B9093C6011B
:10C4100008950F931F938091C801882331F00E94E3
:10C42000836080E10E94EB6127C00E94E6618C017D
:10C4300081708093C80183E00E94EB61C80186701F
:10C4400090708230910581F08330910518F4892B2A
:10C4500021F010C0049751F00DC08091C601877083
:10C460000E94EB6181E003C084E001C089E0809319
:10C47000C70102C00E94CE651F910F9108950E94CE
:10C48000E6618093D90180E10E94EB6182E08093B4
:10C49000C701089580E10E94EB6183E08093C701AA
:10C4A00008958091D901882319F48093C7010895D4
:10C4B00081508093D9010E94E6610E94876080913B
:10C4C000C9019091CA01A091CB01B091CC01019614
:10C4D000A11DB11D8093C9019093CA01A093CB0106
:10C4E000B093CC0188E00E94EB610895CF93DF9375
:10C4F000C091DB01D091DC010E94E66121E0C930EE
:10C50000D20718F4CE5FD04055C021E0CD30D2071D
:10C5100050F4CC0FDD1F81709070C80FD91FC75029
:10C52000D24081E042C021E0C131D20760F4CC0F9B
:10C53000DD1FCC0FDD1F83709070C80FD91FC15253
:10C54000D44082E032C021E0C531D20768F443E034
:10C55000CC0FDD1F4A95E1F787709070C80FD91F87
:10C56000C556D84083E021C021E0C931D20768F424
:10C5700034E0CC0FDD1F3A95E1F78F709070C80F53
:10C58000D91FCD50D14184E010C021E0CD31D20778
:10C5900078F425E0CC0FDD1F2A95E1F78F719070BC
:10C5A000C80FD91FCD59D24285E00E94EB6102C06D
:10C5B000C2E0D1E0D093DE01C093DD0187E080933B
:10C5C000C701DF91CF910895E6EEF1E0119283E08B
:10C5D000E530F807D9F3D0F3E2E2F3E08FE111920E
:10C5E000815087FFFCCFEEE5F3E082E111928150AC
:10C5F00087FFFCCF0E94E6619C018F7190708F5F76
:10C600009E4F9093E3018093E201C90175E09695F6
:10C6100087957A95E1F78F718F5F8093E401C90167
:10C62000892F9927869586958F708C5F8093E50179
:10C630001092E1018EE00E94EB618AE08093C701D5
:10C640000895EF92FF920F931F93CF93DF93ADE086
:10C65000FB0111921192A150A7FFFBCFA0E0B0E027
:10C66000A417B50738F5EFE0EE2EF12C01E010E04D
:10C67000EC01899199270097C9F08F309105B1F0AD
:10C68000FC01E80FF91FE60FF71F32979701281BEF
:10C69000390BC901980102C0220F331F8A95E2F7B6
:10C6A00080819181820F931F918380831196A417BB
:10C6B000B507F8F220E030E0ADE0FB018081918128
:10C6C000280F391F21933193A150A7FFF7CFDF9196
:10C6D000CF911F910F91FF90EF90089540E251E0AC
:10C6E00066E073E086EE91E00E94216340E250E054
:10C6F00062E473E082E293E00E942163089588E09F
:10C70000E6EEF1E0819322E0E537F207D9F3D0F3CA
:10C7100080E990E029E0E6E7F2E0219301968F3F7F
:10C720009105D9F3D0F331E08831930750F427E035
:10C73000FC01EA51FE4F2193019631E088319307C5
:10C74000D0F321E08032920750F428E0FC01EA5156
:10C75000FE4F2193019631E080329307D0F380326F
:10C76000910550F425E0FC01EE5DFC4F219383E040
:10C77000E134F807D9F3D0F30E946E6385E080932B
:10C78000C70108958091E501882381F443E150E0D9
:10C7900061E773E08EE593E00E9421638BE0809374
:10C7A000C7011092E0011092DF0108950E94E66136
:10C7B000982F97708091E101E82FFF27E756FE4FF1
:10C7C0008081E82FFF27E25AFC4F908383E00E948C
:10C7D000EB618091E1018F5F8093E1018091E50140
:10C7E00081508093E50108956F927F928F929F927E
:10C7F000BF92CF92DF92EF92FF920F931F93CF934E
:10C80000DF933C016B014A01C0E0D0E0F1E0BF2EB4
:10C810000EE010E07B010E94E66181709070002EB6
:10C8200002C0880F991F0A94E2F7C82BD92B81E028
:10C830000E94EB618FE0B81669F0F7018191919148
:10C840007F01C817D90730F0B39401501040FFE0C2
:10C85000FB1508F72B2D3327F901E20FF31FEC0D21
:10C86000FD1D349780819181C81BD90B8FE090E02A
:10C87000821B930B02C0D695C7958A95E2F720E0FC
:10C8800030E02815390560F4F30181918B1519F416
:10C89000209741F021972F5F3F4F28153905A8F3C6
:10C8A0000E94CE65C901DF91CF911F910F91FF903A
:10C8B000EF90DF90CF90BF909F908F907F906F9080
:10C8C00008950F931F93CF938C0143E150E061E7EC
:10C8D00073E08EE593E00E94F463803198F4E09178
:10C8E000DF01F091E001E00FF11F80838091DF0113
:10C8F0009091E00101969093E0018093DF0121E0A7
:10C9000030E055C0803159F50E94E661C82FC370F0
:10C91000CD5F82E00E94EB6140E04C1798F420E08C
:10C9200030E0E091DF01F091E001E00FF11FDF0165
:10C93000A20FB31F319780818C934F5F2F5F3F4FC2
:10C940004C1778F32C2F33278091DF019091E00171
:10C95000820F931F9093E0018093DF0128C0813103
:10C9600039F40E94E661C82FC770CD5F83E006C02E
:10C970000E94E661C82FCF77C55F87E00E94EB6118
:10C9800020E02C1790F4E091DF01F091E001E00F3E
:10C99000F11F10828091DF019091E0010196909348
:10C9A000E0018093DF012F5FECCF2C2F3327C901EB
:10C9B000CF911F910F9108958091E401882331F464
:10C9C0000E946E6385E08093C701089582E293E040
:10C9D0000E9461649091E401981B9093E401089592
:10C9E0002091E2013091E3012115310541F48CE001
:10C9F0008093C7013093E0012093DF01089586EE14
:10CA000091E00E9461642091E2013091E301281BD2
:10CA100031093093E3012093E20108958AED91E01A
:10CA200040E250E0BC0168597E4F885B9E4F0E94F7
:10CA3000F4638093DA0188E08093C701089540E2AF
:10CA400051E066E073E086EE91E00E94F46321E03D
:10CA50008030920719F41092C70108958F3F910515
:10CA600009F0B0F40E9487608091C9019091CA01D9
:10CA7000A091CB01B091CC010196A11DB11D809375
:10CA8000C9019093CA01A093CB01B093CC01089542
:10CA90009093DC018093DB0186E08093C7010895C9
:10CAA0000F931F93CF93DF93AA27BB272091C90130
:10CAB0003091CA014091CB015091CC01FA01E901BA
:10CAC000C81BD90BEA0BFB0B8B01BE01CF010E94E7
:10CAD0008A60DF91CF911F910F910895CF93DF93DB
:10CAE000C091DA01C43018F4DD2721962FC0CE3171
:10CAF00010F00E94CE650E94E661BC012C2F332706
:10CB0000A9014250504057FF03C0A9014150504075
:10CB100055954795E901C170D0702296242F33278F
:10CB2000022E02C0CC0FDD1F0A94E2F781E090E0F4
:10CB300002C0880F991F2A95E2F701978623972351
:10CB4000C80FD91F2196842F0E94EB616091DD01EF
:10CB50007091DE01CE010E9450658091DD019091BF
:10CB6000DE019C01442755278091C9019091CA019B
:10CB7000A091CB01B091CC01820F931FA41FB51FD0
:10CB80008093C9019093CA01A093CB01B093CC01CB
:10CB900085E08093C701DF91CF91089581E090E017
:10CBA000F8940C943269DC01FB014115510549F000
:10CBB0004150504029F005900D92002029F0F8CF07
:10CBC0001C9205900020E9F7E61BF70B3197CF0187
:10CBD00008959C01AB01B9018091F90D9091FA0D76
:10CBE0000E94F3650895ABE0B0E0E9EFF5E60C9440
:10CBF000FE683C014B015A01FC01178216828381B9
:10CC000081FD03C08FEF9FEFF5C1F3012381F40194
:10CC100023FD059123FF01914F01002309F4E7C192
:10CC2000053239F423FD059123FF01914F010532AF
:10CC300031F4B301802F99270E941468E6CFCC24E9
:10CC4000DC2C5C2C3AE0FFE1FD1518F1802F9927D0
:10CC50008B32910591F08C32910534F4803291053C
:10CC600079F0839799F015C08D32910561F0C097E6
:10CC700081F461E0E62EDE2831C052E0F52EDF2897
:10CC800004E0D02A2BC018E0D12A28C040E1D42AE1
:10CC900025C0D7FC2CC0802F80538A3088F4082F01
:10CCA000D6FE06C0539EC0011124502E580E16C049
:10CCB000C39EC0011124C02EC80E50E2D52A0EC05A
:10CCC0000E3229F4D6FC93C180E4D82A07C00C3672
:10CCD00019F490E8D92A02C0083649F4F40123FD7A
:10CCE000059123FF01914F01002309F0ACCF802F64
:10CCF0008554833018F08052833038F444E0E42EB9
:10CD0000F12CAE0CBF1C8FE316C0802F9927833601
:10CD1000910559F08436910524F48335910541F14C
:10CD20005CC08337910579F058C0F50102E010E04E
:10CD3000A00EB11E808189837E010894E11CF11C44
:10CD400001E010E012C0F50122E030E0A20EB31EB7
:10CD5000E080F180D6FE03C0652D772702C06FEF1B
:10CD60007FEFC7010E9409688C013FE7D32214C0FE
:10CD7000F50142E050E0A40EB51EE080F180D6FE41
:10CD800003C0652D772702C06FEF7FEFC7010E94B8
:10CD9000FE678C0150E8D52AD3FC0CC08C2D992756
:10CDA0000817190738F4B30180E290E00E94146874
:10CDB000CA94F4CF0115110509F40FC1F701D7FC8E
:10CDC0008591D7FE81917F01B30199270E94146854
:10CDD000C110CA9401501040EDCF043611F009364D
:10CDE000A9F5D7FE0BC0F50134E0E32EF12CAE0C13
:10CDF000BF1C60817181828193810EC0F50102E0C8
:10CE000010E0A00EB11E808191819C01442737FD66
:10CE10004095542FCA01B9013FE6D32297FF09C0BC
:10CE200090958095709561957F4F8F4F9F4F40E80B
:10CE3000D42A2AE030E0AE014F5F5F4F0E94416884
:10CE40009E012F5F3F4F082F021B53C0053729F467
:10CE50005FEED5222AE030E027C0E9EFDE228F36F0
:10CE6000910571F08037910524F488359105A9F07A
:10CE7000BEC08037910539F08837910531F0B7C0D1
:10CE800028E030E011C0F0E1DF2AD4FE03C024E046
:10CE9000E22EDE2820E130E007C0D4FE03C096E099
:10CEA000F92EDF2820E132E0D7FE0AC0F50104E0C8
:10CEB00010E0A00EB11E60817181828193810CC04F
:10CEC000F50142E050E0A40EB51E808191817C0105
:10CED00000271127C801B701AE014F5F5F4F0E94C5
:10CEE00041689E012F5F3F4F082F021B8FE7F82EEE
:10CEF000DF20102FD6FE0DC02EEFD222051548F4EC
:10CF0000152D8D2D992784FF04C082FD02C03FEEB0
:10CF1000D3222D2D332724FF0DC0FE01E00FF11D7C
:10CF20008081803319F449EED42208C01F5F22FFAC
:10CF300005C003C08D2D867809F01F5FED2CFF24FE
:10CF4000E3FC12C0E0FE07C0502E1C1520F45C2C40
:10CF5000511A500E1C2D1C1538F4B30180E290E0DC
:10CF60000E9414681F5FF7CF1C1518F48C2D811BCD
:10CF700001C080E0C82EE4FE10C0B30180E390E061
:10CF80000E941468E2FE15C0E1FE03C088E590E04F
:10CF900002C088E790E0B3010AC08D2D867849F081
:10CFA00080E2E1FC8BE2D7FC8DE2B30199270E947D
:10CFB0001468051538F4B30180E390E00E9414680A
:10CFC0005A94F7CF0150FE01E00FF11D8181B301AA
:10CFD00099270E9414680023A9F7CC2009F415CEE4
:10CFE000B30180E290E00E941468CA94F6CFF30186
:10CFF00086819781EFE02B960C941A69FC010590CD
:10D00000615070400110D8F7809590958E0F9F1F4A
:10D010000895FC016150704001900110D8F780958F
:10D0200090958E0F9F1F08950F931F93CF93DF93BB
:10D030008C01EB018B81992781FF1CC082FF0DC001
:10D040002E813F818C819D812817390764F4E88106
:10D05000F9810193F983E88306C0E885F985802F7B
:10D060000995892B39F48E819F8101969F838E8348
:10D07000C80102C08FEF9FEFDF91CF911F910F91F9
:10D080000895FA01AA27283051F1203181F1E8945E
:10D090006F936E7F6E5F7F4F8F4F9F4FAF4FB1E0AB
:10D0A0003ED0B4E03CD0670F781F891F9A1FA11DA6
:10D0B000680F791F8A1F911DA11D6A0F711D811DA7
:10D0C000911DA11D20D009F468943F912AE0269F6C
:10D0D00011243019305D3193DEF6CF010895462FCB
:10D0E0004770405D4193B3E00FD0C9F7F6CF462FAC
:10D0F0004F70405D4A3318F0495D31FD4052419315
:10D1000002D0A9F7EACFB4E0A695979587957795D1
:10D110006795BA95C9F700976105710508959B0158
:10D12000AC010A2E06945795479537952795BA95E1
:10D13000C9F7620F731F841F951FA01D0895629F7A
:10D14000D001739FF001829FE00DF11D649FE00DFF
:10D15000F11D929FF00D839FF00D749FF00D659F60
:10D16000F00D9927729FB00DE11DF91F639FB00D5F
:10D17000E11DF91FBD01CF0111240895A1E21A2E6E
:10D18000AA1BBB1BFD010DC0AA1FBB1FEE1FFF1F6B
:10D19000A217B307E407F50720F0A21BB30BE40BBB
:10D1A000F50B661F771F881F991F1A9469F7609502
:10D1B0007095809590959B01AC01BD01CF010895BC
:10D1C00097FB092E05260ED057FD04D0D7DF0AD0D5
:10D1D000001C38F450954095309521953F4F4F4FA6
:10D1E0005F4F0895F6F790958095709561957F4F04
:10D1F0008F4F9F4F08952F923F924F925F926F9261
:10D200007F928F929F92AF92BF92CF92DF92EF92D6
:10D21000FF920F931F93CF93DF93CDB7DEB7CA1B57
:10D22000DB0B0FB6F894DEBF0FBECDBF09942A8882
:10D23000398848885F846E847D848C849B84AA842A
:10D24000B984C884DF80EE80FD800C811B81AA81B7
:10D25000B981CE0FD11D0FB6F894DEBF0FBECDBF82
:06D26000ED010895FFCF6F
:10D266005AFFC300000002000000000E520000003A
:10D2760000FF7F8F0B3511A60501014F4E004F466B
:10D286004600534E455300415652004849524F4DB1
:10D29600004C4F524F4D007F8B97A4AFBBC5CFD9E3
:10D2A600E1E8EFF4F8FBFDFDFDFBF8F3EEE7E0D770
:10D2B600CEC4B9AEA296897E7165594D42372D24EA
:10D2C6001C150F09050301010103070B11171F2880
:10D2D600313B46525E6A76312E3000322E360009D8
:10D2E600623F624A6251627F631F6576620E656EB7
:10D2F60065E462C263F064DC641011120008070979
:0CD30600060A050B040C030D020E010FBB
:00000001FF
